:020000040000FA
:100000000EEF00F0FFFFFFFFC5EF0DF0FFFFFFFF5A
:10001000FFFFFFFFFFFFFFFF90EF18F027EF0CF04F
:100020005BC002F30301036B5AC004F3056BB1C05C
:1000300006F3076B94C008F3096B45C00AF30B6B1A
:10004000B3C00CF30D6B3FC00EF30F6B0001B75143
:10005000BC6FBD6B060ED890BC37BD37E82EFBD702
:10006000B851BE6FBF6B050ED890BE37BF37E82EB4
:10007000FBD73D501F0BC06FC16BBE51C027BF5196
:10008000C123BC51C0250301106F0001BD51C12126
:100090000301116F00018A51BC6FBD6B070ED89030
:1000A000BC37BD37E82EFBD78D51BE6FBF6B060E38
:1000B000D890BE37BF37E82EFBD78951C06FC16BD0
:1000C000050ED890C037C137E82EFBD701014A5141
:1000D0000001C26FC36BC23BC33BF00EC317C251DA
:1000E0000F0BC313F00EC2178751C46FC56BD890A6
:1000F000C437C537D890C437C537D890C437C5374B
:100100009051070BC66FC76BC451C627C551C72393
:10011000C251C627C351C723C051C627C151C723E7
:10012000BE51C627BF51C723BC51C6250301126F5C
:100130000001BD51C7210301136F7AC016F37BC0C4
:1001400017F376C018F377C019F335C01AF336C029
:100150001BF300019C05D8A405D072C01CF373C02A
:100160001DF305D0000E03011D6F000E1C6F000E65
:100170004F6E1200000ED46FCE05D8A402D01E0E12
:10018000C727010ED56F95D0BB98BB9AD551C8250E
:10019000AF0F34EC19F0BB8A0001CE05D8A40FD004
:1001A000BB98BB9AC7510F0B34EC19F0BB8ABB9AB2
:1001B0000001C7390F0B100F34EC19F00ED0BB98AB
:1001C000BB9AC7390F0B100F34EC19F0BB8ABB9ADE
:1001D0000001C7510F0B34EC19F0BB8ABB88000E2D
:1001E0000001D36F61D0C651C503D551CF6FD06B1D
:1001F000F350CF27F450D023FF0ECF25BC6FFF0E56
:10020000D021BD6FC4C0BEF0BF6BDFEC17F0D3517F
:10021000C225D16F000EC321D26FBC51D127BD5171
:10022000D223600047F3F6FF60004BF3F7FF000EA8
:10023000F86E08006F00D4FFD4F0CCC0CFF0030EEE
:10024000CF17D4C0D0F0CF2B02D0D890D033CF2F3F
:10025000FCD70001D051D46FCDC0CFF0030ECF1723
:10026000D4C0D0F0CF2B02D0D890D037CF2FFCD72E
:100270000001D051D46FC905D8A404D0C551D519F7
:10028000D8B4D48FCA05D8A403D0D505D8B4D481A6
:10029000CB05D8A402D0FF0ED41BBB9AD45134ECAA
:1002A00019F0BB8A0001D32BC451D35DD8A09BD7D2
:1002B000D52BD551C55DD8B067D7BB881200D66F96
:1002C00091D0350EC26FFA0EC36F0B0EC46F010EC4
:1002D000C56F020EC66F3F0EC76F000EC86F010ECE
:1002E000C96F000ECA6F000ECB6F000ECC6F000EF0
:1002F000CD6FF6C0CEF0BAEC00F01200350EC26F32
:10030000FA0EC36F0B0EC46F010EC56F030EC66FDE
:100310003F0EC76F000EC86F010EC96F000ECA6F87
:10032000000ECB6F000ECC6F000ECD6FF6C0CEF07E
:10033000BAEC00F01200350EC26FFA0EC36F0B0E4E
:10034000C46F010EC56F040EC66F3F0EC76F000E5F
:10035000C86F010EC96F000ECA6F000ECB6F000E82
:10036000CC6F000ECD6FF6C0CEF0BAEC00F01200EC
:10037000350EC26FFA0EC36F0B0EC46F010EC56F40
:10038000050EC66F3F0EC76F000EC86F010EC96F16
:10039000000ECA6F000ECB6F000ECC6F000ECD6F3B
:1003A000F6C0CEF0BAEC00F01200350EC26FFA0EB5
:1003B000C36F0B0EC46F010EC56F000EC66F3F0EEC
:1003C000C76F000EC86F010EC96F000ECA6F000E16
:1003D000CB6F000ECC6F000ECD6FF6C0CEF0BAEC36
:1003E00000F012000001D651000AD8B4C1D7210A8A
:1003F000D8B4A1D7630AD8B481D7260AD8B461D7B4
:10040000D4D7C46F0001C451D8A4BFAF1AD0BCC0A8
:10041000C0F0BDC0C1F0BEC0C2F0BFC0C3F0C01FBD
:10042000C11FC21FC31FC02B000EC123C223C32381
:10043000C0C0C6F0C1C0C7F0C2C0C8F0C3C0C9F0D8
:1004400008D0BCC0C6F0BDC0C7F0BEC0C8F0BFC0B9
:10045000C9F0BC51BD11BE11BF11D8A409D0000E06
:10046000BC6F000EBD6F000EBE6F000EBF6F12009E
:10047000960EC56F06D0C52BD890C933C833C73385
:10048000C633000EC615C06F000EC715C16F000E33
:10049000C815C26FFE0EC915C36FC051C111C2117C
:1004A000C311D8B40DD0E7D7C52B010EC627000E57
:1004B000C723C823C923D890C933C833C733C63329
:1004C000000EC615C06F000EC715C16F000EC8150F
:1004D000C26FFF0EC915C36FC051C111C211C31144
:1004E000D8B407D0E1D7C507D890C637C737C837C3
:1004F000C937C8BF03D0020EC561F5D7C5A1C89FD3
:10050000D890C533C5C0C0F0C16BC26BC36BC0C04F
:10051000C3F0C26BC16BC06BC051C613C151C713CE
:10052000C251C813C351C913C451D8A4BFAF01D01D
:10053000C98FC6C0BCF0C7C0BDF0C8C0BEF0C9C03E
:10054000BFF01200C2C0C9F0C3C0C8F0C15104E17D
:10055000020EC05DD8A03BD0C0B139D05A0EC4192C
:10056000D8A435D0C0C0BCF0C1C0BDF009EC19F0B2
:100570000001C919D8B414D0C0C0BCF0C1C0BDF0CE
:10058000C9C0BEF03CEC15F0FF0E0001C025BC6FE9
:10059000FF0EC121BD6FC4C0BEF03CEC15F01200CF
:1005A000FF0EC025BC6FFF0EC121BD6F09EC19F015
:1005B0000001C419D8B41200FF0EC025BC6FFF0E95
:1005C000C121BD6FC4C0BEF03CEC15F01200C1519A
:1005D00004E1210EC05DD8A012005B0EC419D8A49E
:1005E0001200010EC025BC6F000EC121BD6F09ECC9
:1005F00019F00001C56F080EC527C0C0BCF0C1C00E
:10060000BDF009EC19F00001C66FC76BC52B03D014
:10061000D890C637C737C52FFBD70001C251C619BE
:1006200004E1C351C719D8B41FD0C0C0BCF0C1C0C9
:10063000BDF0C8C0BEF03CEC15F0010E0001C025B5
:10064000BC6F000EC121BD6FC9C0BEF03CEC15F0FF
:10065000FF0E0001C025BC6FFF0EC121BD6FC4C0DD
:10066000BEF03CEC15F01200FF0EC025BC6FFF0E73
:10067000C121BD6F09EC19F09BD7000E0001D06FAE
:10068000000ECF6F0301E751FC0B0001D06F030197
:10069000E751030B0001CF6F79D04E04D8A41200AC
:1006A000D0C0C9F0230E3BECFAF0010EB06F000E83
:1006B0000101BC6F010EBD6F000E6B6F000E696F04
:1006C0001200D0513F18D8A406D0010E3E6E000E85
:1006D0000101696F02D0000E3E6E4D04D8A40AD00D
:1006E0003E50D8A407D0D0C03FF0010E3E6E010EA0
:1006F00001016A6F4E50D8A41200420E0001B619D3
:10070000D8A412003E04D8A409D0420EB36512004A
:10071000470EB3611200CAEC17F012000101692BF9
:10072000040E69651200000E696F000E3E6E000E29
:100730000201996F000E0001B06F010E0101AE6F52
:10074000000E6B6F470E0001B66FB651B6253D0126
:100750006F6FFE0E706F010E0101B36F1200D0A516
:1007600012004D04D8A412003E04D8A41200D0C038
:10077000CDF0700ECD17D8B41200D0390F0B070B87
:10078000400F0101B26FB2C1B3F0C5D7CF51000A1B
:10079000D8B483D7010AD8B494D7030AD8B4DFD722
:1007A000010A1200000ED06FC9C0C2F0CAC0C3F067
:1007B000030EC56FE80EC46F0EEC14F0C251D26F79
:1007C000D2C0BCF0BD6BFC0EBF6F180EBE6FDFEC6D
:1007D00017F0C951BC25C26FCA51BD21C36F000EAD
:1007E000C56F640EC46F0EEC14F0C251D16FD2C04D
:1007F000BCF0BD6BFC0EBF6F180EBE6FDFEC17F0C8
:10080000BCC0CCF0BDC0CDF0D1C0BCF0BD6BFF0E04
:10081000BF6F9C0EBE6FDFEC17F0BC51CC27BD51F3
:10082000CD23C951CC25C26FCA51CD21C36F000E53
:10083000C56F0A0EC46F0EEC14F0C251CF6FD251C7
:10084000180D6F00CCFFCCF0D1519C0D6F00CCFF88
:10085000CDF0CF51F60DF350CD25CC25C925CE6F67
:10086000540ECB19D8B404D0740ECB19D8A403D02D
:10087000D2C0D0F01FD0480ECB19D8B404D0680E27
:10088000CB19D8A403D0D1C0D0F014D05A0ECB19B4
:10089000D8B404D07A0ECB19D8A403D0CFC0D0F0EE
:1008A00009D0450ECB19D8B403D0650ECB19D8B4F6
:1008B000CEC0D0F0D0511200D76F020E0101EB6F05
:1008C000D7C0ECF15AD0CCC0EDF1030E2DD0CC51F5
:1008D000CD25D56FD5290101ED6FCEC0EEF1040E07
:1008E0000001D86FCD05D8A404D0D0C0EFF1050E1B
:1008F000D86F020ECD19D8A406D0CFC0EFF1D0C06A
:10090000F0F1060ED86F030ECD19D8A44AD0CFC08F
:10091000EFF1D0C0F0F1D1C0F1F1070E05D0000E1B
:100920000101ED6F030E27D0D86F3BD0010E0101FE
:10093000ED6FD0C0EEF1040E0001D86FD105D8A044
:1009400030D00101ED2BD1C0EFF1050E14D0010E16
:10095000E7D7020E0101ED6FD2C0EEF1D3C0EFF187
:10096000050E0001D86FD405D8A01BD00101ED2BD6
:10097000D4C0F0F1060E0001D7D70001D751000A0C
:10098000D8B4A1D7010AD8B4A2D7040AD8B4C7D71B
:100990000D0AD8B4CBD7010AD8B4DBD7180AD8B41B
:1009A000D6D7CAC0C1F0CBC0C2F0EDC1C3F0D8C029
:1009B000C4F0F4EC0AF0D66FD6C0BCF00101EB51E4
:1009C00044EC18F01200216E71D04D04D8A412002E
:1009D0005504D8A414D0000E0201B56F000EB66FF6
:1009E0003E0EB76F000EB86F000EB96FB50E1E6EDB
:1009F000020E1F6E050E206E8FEC16F013D0000E47
:100A00000201CA6F000ECB6F3E0ECC6F000ECD6F91
:100A1000000ECE6FCA0E1E6E020E1F6E050E206EE9
:100A20008FEC16F0050E0201886F100E876F120012
:100A30004D04D8A4120018C237F119C236F136C1DC
:100A40005AF037C15BF0010E0101B56F010E4E6E19
:100A50005504D8A414D05BC0B5F25AC0B6F23F0E0C
:100A60000201B76F5AC0B8F2000EB96FB50E1E6E14
:100A7000020E1F6E050E206E8FEC16F013D05BC0B9
:100A8000CAF25AC0CBF23F0E0201CC6F5AC0CDF26F
:100A9000000ECE6FCA0E1E6E020E1F6E050E206E69
:100AA0008FEC16F0050E0201886F12002150220A09
:100AB000D8B41200010AD8B412000D0AD8B485D7F0
:100AC000010AD8A41200B4D70101E905D8A44ED078
:100AD00079C2EDF07AC2EEF03BEC13F0EDC00CF110
:100AE000EEC00DF1010E0101626F6151D8A40CD06E
:100AF000000EC06F000EBF6F0CC1BCF00DC1BDF089
:100B000066EC13F0010113D0010EC06F270EBF6514
:100B100023D0000EBF6F0DD0000E09D0640E07D099
:100B2000500E05D03C0E03D0280E01D0140E636F7A
:100B300013D06451000AD8B4F9D7140AD8B4F4D742
:100B40003C0AD8B4EFD7140AD8B4EAD76C0AD8B4A0
:100B5000E5D7340AD8B4E0D764516319D8B404D0C7
:100B600063C164F1010E7B6F000EE96F0001B505F2
:100B7000D8B403D0AE05D8A406D0010E0101616F30
:100B8000000E606F1200800E01010C5D0C0E0D59FD
:100B9000D8B014D06151D8A412005050D8A412007B
:100BA0000201465104E1650E455DD8A004D0010E56
:100BB0000101606F1200454B462B1200000E616F61
:100BC000000E606F12000101EA05D8A412007DC278
:100BD000EDF07EC2EEF010EC13F0EDC01AF1EEC0B5
:100BE0001BF1010E0101826F1AC1EFF01BC1F0F081
:100BF0001AC151F21BC152F2A10E0001EF5D0F0E9E
:100C0000F059D8A002D0000E4FD0B90EEF5D0B0EF8
:100C1000F059D8B0F8D7D10EEF5D070EF059D8A033
:100C200002D0640E41D0E90EEF5D030EF059D8A05A
:100C300002D05A0E39D0590EEF5D020EF059D8A0ED
:100C400002D0500E31D0C30EEF5D010EF059D8A086
:100C500002D04B0E29D02D0EEF5D010EF059D8A019
:100C600002D0400E21D0F05104E1A10EEF5DD8A0DA
:100C700002D0320E19D0F05104E16F0EEF5DD8A012
:100C800002D0300E11D0F05104E15B0EEF5DD8A020
:100C900002D0200E09D0F05104E1470EEF5DD8A03C
:100CA00002D0190E01D0100E486E0101A705D8A47C
:100CB00005D02F0E486402D0000E486E000EEA6F79
:100CC0001200000EE76F000EE86F5CD0480EC26F96
:100CD000E50EC36F070EC46F020EC56FE851D6252F
:100CE000E06F000ED721E16F600083F3F6FF600034
:100CF00087F3F7FF000EF86E0800F550E00FC66F9F
:100D0000E751FC0D6F00CCFFE2F0E851080DF35005
:100D1000E225D925C76FDAC0C8F0DBC0C9F0DCC056
:100D2000CAF0DDC0CBF0DEC0CCF0DFC0CDF0F6C045
:100D3000CEF0BAEC00F0E851D625E06F000ED721D6
:100D4000E16F600083F3F6FF600087F3F7FF000EAA
:100D5000F86E0800F550490AD8B412D0E851D625EB
:100D6000E06F000ED721E16F600083F3F6FF6000B3
:100D700087F3F7FF000EF86E0800F550690AD8B443
:100D8000E72BE82BFF0EE06FFF0EE16FD851E26F0B
:100D9000E36BE051E227E151E323E851E46FE56BB7
:100DA000E251E45DE551800AE66FE351800AE659BD
:100DB000D8B012008BD71C6E020E0101EB6F1CC065
:100DC000ECF14ED011C0EDF1030E48D011501224B9
:100DD0001A6E1A28ED6F13C0EEF1040E1D6E120488
:100DE000D8A404D015C0EFF1050E1D6E020E121826
:100DF000D8A406D014C0EFF115C0F0F1060E1D6E98
:100E0000030E1218D8A43FD014C0EFF115C0F0F1B2
:100E100016C0F1F1070E22D0000EED6FD5D7010EEE
:100E2000ED6F15C0EEF1040E1D6E1604D8A02BD088
:100E3000ED2B16C0EFF1050E11D0010EEED7020E0C
:100E4000ED6F17C0EEF118C0EFF1050E1D6E19041D
:100E5000D8A019D0ED2B19C0F0F1060E1D6E13D0DD
:100E60001C50000AD8B4AED7010AD8B4AFD7040AD0
:100E7000D8B4D2D70D0AD8B4D2D7010AD8B4DFD7A4
:100E8000180AD8B4DAD70FC006F010C007F0EDC1C9
:100E900008F01DC009F045EC0BF01B6E1BC001F003
:100EA0000101EB51C7EC18F01200216E050E020192
:100EB000176506D00C0E1C6103D01CC200F202D0D4
:100EC000000E006F0051D8B45ED0010E226E10D01B
:100ED0001C0E2224D96EDA6A020EDA22000E2224B7
:100EE000E16EE26A020EE2226F007FFFE7FF222A34
:100EF0002250005DD8B0ECD7010E0101656F43D0E0
:100F00004B50D8A44B065504D8A413D05BC0B5F2FF
:100F10005AC0B6F2310E0201B76F34C1B8F2B50E45
:100F20001E6E020E1F6EB951050F206E8FEC16F06B
:100F300012D05BC0CAF25AC0CBF2310E0201CC6FA4
:100F400034C1CDF2CA0E1E6E020E1F6ECE51050FB9
:100F5000206E8FEC16F05450D8B411D00F0E020151
:100F6000D317D3C2BEF23F0ECF171C0ED0171C0EE4
:100F7000D1173F0EBA171C0EBB171C0EBC170B0E59
:100F80000201886F12002150210AD8B4B9D7030A90
:100F9000D8B41200010A1200000E0001C06F000E4A
:100FA000C16F010EC26FC251020D2A0EF324D96E19
:100FB000020EF420DA6EBC51DE1807E1BD51DE18D6
:100FC000D8A403D0010EC06F11D0C251020D2A0E59
:100FD000F324D96E020EF420DA6EDE50DE10D8B49F
:100FE000C2C0C1F0C22B050EC265DDD7C051D8A466
:100FF0001200C151D8B434D0C151020D2A0EF324CD
:10100000D96E020EF420DA6E6000F3F2DEFF6000AB
:10101000F7F2DDFFC1C058F11200BCC02EF2BDC016
:101020002FF2020E586F1200BCC030F2BDC031F278
:10103000030E586F1200BCC032F2BDC033F2040E72
:10104000586F1200BCC034F2BDC035F2050E586FA7
:101050001200BCC02CF2BDC02DF2010E586F120060
:1010600001015851010AD8B4D8D7030AD8B4DCD743
:10107000010AD8B4E0D7070AD8B4E4D7010AD8A443
:101080001200E7D70001BD6F0101E705D8B433D0E6
:10109000000ED56F000E0001BE6F0ED0BE51600F66
:1010A000D96EDA6ADB0EBE25E16EE26A030EE22239
:1010B0006F007FFFE7FFBE2BBD51BE5DD8A0EED70E
:1010C00056C0BCF0030EBC17D8A45688040E5418A2
:1010D000D8A402D0010E546E040E5318D8A402D026
:1010E000010E536E040E5218D8A402D0010E526E97
:1010F000010E0101D56F020EE719D8B41200000EDF
:10110000556E000E0001BF6F10D0DA0EBF25D96EEC
:10111000DA6A030EDA22CE0EBF25E16EE26A030E12
:10112000E2226F007FFFE7FFBF2BBF51BD5DD8B04C
:10113000ECD756C0BCF0030EBC17D8A4568A540492
:10114000D8A402D0020E546E5304D8A402D0020ECA
:10115000536E5204D8A402D0020E526E010E556E88
:101160001200BC6F05D0000E01D0010EBD6F66D01D
:101170000001BC51000AD8B4F6D70A0AD8B4F3D794
:10118000010AD8B4F0D7070AD8B4EDD7010AD8B409
:10119000EAD7030AD8B4E7D7010AD8B4E4D71F0ABC
:1011A000D8B4E1D7010AD8B4DED70F0AD8B4DBD758
:1011B000010AD8B4D8D73F0AD8B4D5D7010AD8B4D1
:1011C000D2D7030AD8B4CFD7010AD8B4CCD70B0AE8
:1011D000D8B4C9D7010AD8B4C6D7030AD8B4C3D77C
:1011E000010AD8B4C0D7070AD8B4BDD7010AD8B409
:1011F000BAD7030AD8B4B7D7010AD8B4B4D71C0AEF
:10120000D8B4B1D7070AD8B4AED7010AD8B4ABD78F
:101210000C0AD8B4A8D7780AD8B4A5D7030AD8B48A
:10122000A2D7010AD8B49FD7080AD8B49CD7070A16
:10123000D8B499D7010AD8B496D797D7BD51120020
:10124000C76F0001C005D8A402D01E0EBE27010E34
:10125000CA6F5CD0BB98BB9ACA51BF25AF0F34ECA4
:1012600019F0BB8A0001C005D8A40FD0BB98BB9A67
:10127000BE510F0B34EC19F0BB8ABB9A0001BE398A
:101280000F0B100F34EC19F00ED0BB98BB9ABE397F
:101290000F0B100F34EC19F0BB8ABB9A0001BE5142
:1012A0000F0B34EC19F0BB8ABB88000E0001C96F2C
:1012B00028D0000EC86FCA05D8B4C881BD51CA195C
:1012C000D8B4C88FC951D8B414D0C951C16FC26B3A
:1012D000FF0EC36FFF0EC46FC751C56FC66BC351FE
:1012E000C527C451C623C151C51904E1C251C6194D
:1012F000D8B4C869BB9AC85134EC19F0BB8A000154
:10130000C92BC751C95DD8A0D4D7CA2BCA51BD5D5E
:10131000D8B0A0D7BB881200256E16C224F0000EEC
:10132000266E4DD02550D8B40ED02350D8B40BD053
:10133000255002011819D8A408D023501919D8A48F
:1013400004D0010E01D0000E266E02011A51BF0B0F
:101350000101356F335102011B19D8B407D01BC2EC
:1013600033F133C1A4F1010E0101A36F2604D8A407
:1013700014D0010E0101E36F010EBE6F000E0201D9
:10138000666F000E656F010E0001AF6F010E4E6EAD
:101390000101355155EC07F004D001013551E3EC62
:1013A00004F0130E0101DE25D96EDA6A020EDA228C
:1013B000DF50346F11D0010E0001926F0DD0245018
:1013C000400AD8B409D0110AD8B406D0D00AD8B48B
:1013D000A9D7040AD8B4EFD726501200040EBE6E67
:1013E000000EBD6E010EBA6E500EBB6E980EBC6E36
:1013F000030EC66EFE0EC26E030EC36E270EC46EC3
:10140000FC0EC56E0C0E3A01706F000E606F040E7C
:10141000506F010E806F020E406FF00E716F040E60
:10142000816F000E516FFC0E416F070E616F040E4D
:10143000826F000E426F000E526F180E626F030E25
:10144000726F4369536963697369070E836F180E7E
:10145000E36F210E136F220E146F090EE56F130E4A
:10146000E16F190EE46F0B0EDE6F140EE26F040EC7
:10147000D96F1F0E0A6F1E0E0B6F230E186F240EEE
:10148000196F050EDA6F130E166F160EDF6F12004E
:101490004E04D8A413D05450D8A410D05350D8A47C
:1014A0000DD05250D8A40AD0020EC96F230EC4EC3E
:1014B000E4F00301DA6FDA5142EC08F00101D105E2
:1014C000D8A405D03DEC03F0000E0101D16F4D040E
:1014D000D8A415D06B51D8A412D0D005D8A40FD061
:1014E000410E0001B619D8B40AD0010EC06F410EEA
:1014F00026EC11F0030E3F6E000E0001B36F0101E8
:10150000AF05D8A41200470E0001B66FB651B6253C
:101510003D016F6FFE0E706F010E0101B36F000E83
:101520000201996F000E0001B06F010E0101AE6F54
:10153000000EAF6F000E4D6E000E6B6F1200BD6F90
:10154000000E0001BF6FBB98BB9ABF51B00F34ECC7
:1015500019F0BB8A0001BD05D8A40AD0BB9A0E0EB3
:1015600034EC19F0BB8ABB9A110E34EC19F009D097
:10157000BB9A000E34EC19F0BB8ABB9A100E34EC07
:1015800019F0BB8ABB88000E0001BE6FBB9A000E2B
:1015900034EC19F0BB8A0001BE2B650EBE65F6D790
:1015A000BF2B070EBF65CFD7BB98BB9AB00E34ECEC
:1015B00019F0BB8A0001BD05D8A40AD0BB9A0E0E53
:1015C00034EC19F0BB8ABB9A110E34EC19F009D037
:1015D000BB9A000E34EC19F0BB8ABB9A100E34ECA7
:1015E00019F0BB8ABB881200000EC96F2CD0C951FC
:1015F000C125C56F000EC221C66F600017F3F6FF4C
:1016000060001BF3F7FF000EF86EEB0EC76F010EC4
:10161000C86FC951C727000EC823C451C725D96E4A
:10162000000EC821DA6E1F0EF76403D00800F550D3
:1016300007D06F00DBFFE1FF6F00DFFFE2FFE75045
:10164000DF6E0001C92BC351C95DD8A0D0D7EB0E06
:10165000BC6F010EBD6FC951C425BE6FF4EC17F00D
:10166000C56FEB0EC66F010EC76FC951C627000EBE
:10167000C723C451C625D96E000EC721DA6E60009B
:1016800017F3DFFFC951C4251200000E0E6E2BD0D8
:101690000E5006240A6E000E07200B6E60002BF021
:1016A000F6FF60002FF0F7FF000EF86EEB0E0C6EE9
:1016B000010E0D6E0E500C26000E0D2209500C244A
:1016C000D96E000E0D20DA6E1F0EF76403D00800ED
:1016D000F55007D06F00DBFFE1FF6F00DFFFE2FF97
:1016E000E750DF6E0E2A08500E5CD8A0D1D7EB0E63
:1016F000016E010E026E0E500924036E30EC18F0DC
:101700000A6EEB0E0B6E010E0C6E0E500B26000EC9
:101710000C2209500B24D96E000E0C20DA6E6000EA
:101720002BF0DFFF0E5009241200BE6F45C0BDF044
:10173000180E0001BD17D8B41DD045380F0B010B92
:10174000471A4704D8A40CD04650FF0ABD6FBE51BB
:10175000BD5DD8A02BD04650BE2729D01F0E05D086
:101760004650BE5DD8B003D0000EBE6F24D04650A8
:10177000BE5F21D045A41FD04704D8A40FD0BC51D0
:10178000D8B4E2D7BE51D8A403D0000E01015D6FDA
:1017900046500001BE5DD8A0E7D7E9D7BC51D8A418
:1017A000D3D7BE51D8A4F4D7010EF0D7BE691F0E0F
:1017B000BE6501D0D3D7000E466EBE511200BE6F7B
:1017C0004704D8A436D04650FF0A0001BD6FBE5171
:1017D000BD5DD8B002D0BE6912D04650BE270FD032
:1017E000050EBE6530D0050E2AD0030EBE652BD087
:1017F000030E25D0020EBE6526D0020E20D0BC51AD
:10180000640AD8B4EDD70A0AD8B4EFD7010AD8B41D
:10181000ECD7150AD8B4E9D7060AD8B4EBD7FE0A34
:10182000D8B4E8D7010AD8B4E0D7070AD8B4DDD7CE
:10183000D7D70001BE51465CD8A003D0010EBE6FC1
:1018400002D04650BE5F000E466EBE511200300EF2
:10185000F66E320EF76E000EF86E00EEE1F210EE4C
:101860001CF009006F00D7FFEEFFE550E150F9E1F1
:10187000500EF66E330EF76E000EF86E09006F0014
:10188000D4FFF6F000EE00F3F20EEE6AE806FDE19A
:1018900000EE00F2E10EEE6AE806FDE100EE00F176
:1018A00010EE00F1EE6AE550E150FCE1E250FAE1A1
:1018B00000EE60F0590EEE6AE806FDE100EE2FF052
:1018C0002D0EEE6AE806FDE1080ED56E000ED66E0E
:1018D000000ED76E000180EFA9F09397660E00010D
:1018E000BC6F210EBD6F000EBE6F81EC19F0390187
:1018F00093996E0E0001BC6F2C0EBD6F000EBE6F73
:101900007AEC19F0000E3D01EC6F000EED6F000E49
:10191000EE6F000EEF6F000EF06F000EF16FB00E65
:10192000F26F800EF36F000EF46F8A0EF56F000EEB
:10193000F66F000EF76F000EF86F000EF96F000ED5
:10194000FA6F000E586E000E0101DB6F150E0201DA
:10195000FF6F000E596E000E0101DA6F000EDD6F91
:10196000390193871200D96F0A0E0001D76502D0A2
:101970000A0ED76FD90EC26FF80EC36F570EC46F21
:10198000020EC56F010EC66FD9C0C7F0D6C0C8F031
:10199000000EC96F000ECA6F000ECB6F000ECC6F29
:1019A000000ECD6FF6C0CEF0BAEC00F0B20EC26FF2
:1019B000FD0EC36F050EC46F020EC56F000EC66F1D
:1019C000D751080DF350D925D86FD829C76FD6C085
:1019D000C8F0000EC96F000ECA6F000ECB6F000E6C
:1019E000CC6F000ECD6FF6C0CEF0BAEC00F0D75140
:1019F00012000201745104E13D0E735DD8A00DD0B8
:101A0000000E0001B56F000E01016B6F000ED66F66
:101A1000000E0201746F000E736F3C0E0101BC6575
:101A20001ED0000EBD6F000EBC6F000E0001B06F27
:101A3000010E0101AE6F000E6B6F000E3E6E420E86
:101A40000001B66FB651B6253D016F6FFE0E706F87
:101A5000010E0101B36F000E4E6E010EAB6F02015D
:101A60005B51571904E15C515819D8B412005BC29C
:101A700057F25CC258F2010EB26F12004704D8A4AC
:101A80001FD04650BE6FBF6BBE1DC06FBF1DC16F64
:101A9000BC51C05DBD51C159D8B003D0BC69BD694E
:101AA00004D04650BC27000EBD23BC51335CBD5151
:101AB0003458D8B020D033C0BCF034C0BDF01BD0F7
:101AC000FF0EBE6FFF0EBF6FBCC0C0F0BDC0C1F047
:101AD000BE51C027BF51C1234650C05D000EC15941
:101AE000D8B005D0000EBD6F010EBC6F04D04650BB
:101AF000BC5F000EBD5B000E466EBCC0BCF0BDC03E
:101B0000BDF01200C06F000E0001C16FC005D8A467
:101B10002FD0010E0101C46F0001BC51BE6FBF6B1D
:101B2000BE510101245D0001BF5101012559D8A01A
:101B300006D000019905D8A402D0000E12D00001F1
:101B4000BD51BE6FBF6BBE510101245D0001BF518D
:101B500001012559D8A016D000019951D8A412D05E
:101B6000010E996F000E0101256F000E246F07D042
:101B7000000E0101256F000E246F000EC46F010ED0
:101B80000001C16F0001C15112006F00D8FF2BF09E
:101B90006F00DCFF2CF06F00E0FF2DF06F00D4FF32
:101BA0002EF0390193B1A3A103D036ECFEF023D07F
:101BB00093A302D0A3B3F9D793B7A3A703D0B3ECF1
:101BC00010F019D093B9A3A903D037EC16F013D0B5
:101BD0009AB3AAA303D088EC0FF00DD093A502D03E
:101BE000A3B5E3D792AF02D0A2BFDFD79AB3AAA31F
:101BF00002D0A6EC19F06000BBF0F5FF6000B7F072
:101C0000F8FF6000B3F0F7FF6000AFF0F6FF1100DF
:101C10000001D66F710E0001C26FF70EC36F0F0E79
:101C2000C46F020EC56FD651020DF350060FC66F7A
:101C30004A0EC76F040EC86F000EC96F000ECA6F40
:101C4000000ECB6F000ECC6F000ECD6FF6C0CEF045
:101C5000BAEC00F0710EC26FF70EC36F0F0EC46FB7
:101C6000020EC56FD651020DF350070FC66F590E05
:101C7000C76F040EC86F000EC96F000ECA6F000E4A
:101C8000CB6F000ECC6F000ECD6FF6C0CEF0BAEC6D
:101C900000F012005AEC19F0D9EC18F0EEEC09F053
:101CA0004EEC19F09BEC19F08DEC12F05EEC17F095
:101CB000FAEC18F026EC19F047EC17F074EC17F07A
:101CC0002FEC17F09EEC15F07EEC15F06DEC0CF09F
:101CD00042EC19F0B5EC17F05EEC11F0A00E00012B
:101CE000BD6FC80EBE6FA40EBF6FA60EC06FA20E52
:101CF000C16F2F0EC26F270EC36F810EC46F100EFF
:101D0000C56FFA0EC66F900EC76FAF0EC86F400E4C
:101D1000EEEC10F01200D66F040E0001D66502D072
:101D2000040ED66F3E0EC26FEB0EC36F220EC46F51
:101D3000040EC56FD629C66F220EC76F030EC86F7B
:101D4000000EC96F000ECA6F000ECB6F000ECC6F75
:101D5000000ECD6FF6C0CEF0BAEC00F02A0EC26FC6
:101D6000F10EC36F0A0EC46F030EC56FD6510A0F72
:101D7000C66F480EC76F040EC86F000EC96F000E05
:101D8000CA6F000ECB6F000ECC6F000ECD6FF6C089
:101D9000CEF0BAEC00F01200D66F040E0001D6654A
:101DA00002D0040ED66F710EC26FF70EC36F0F0E06
:101DB000C46F020EC56FD629C66F3A0EC76F060EE6
:101DC000C86F000EC96F000ECA6F000ECB6F000EF9
:101DD000CC6F000ECD6FF6C0CEF0BAEC00F0BF0EA7
:101DE000C26FFC0EC36F050EC46F010EC56FD6C067
:101DF000C6F04D0EC76F070EC86F000EC96F000EFC
:101E0000CA6F000ECB6F000ECC6F000ECD6FF6C008
:101E1000CEF0BAEC00F01200EC51FD0DF350360F8D
:101E2000EE6FECC0EDF0FF0EED27EDB1EE2B510E95
:101E3000C26FFC0EC36F660EC46F010EC56F000E3D
:101E4000C66F000EC76F010EC86F000EC96F000E7F
:101E5000CA6F010ECB6F000ECC6F000ECD6FF6C0B7
:101E6000CEF0BAEC00F0EAC0D6F0EBC0D7F0ECC090
:101E7000D8F0EEC0D9F0010EDA6F000EDB6F000E65
:101E8000DC6F010EDD6F000EDE6F000EDF6FB5EC54
:101E9000E6F01200C66F240E0001C66102D0240EC7
:101EA00004D0F00EC66502D0F00EC66FC6C0C4F0F6
:101EB000C43B0F0EC417C451C65D0101816FC6C07B
:101EC000C4F00001C43B0F0EC417C6C0C5F0D890C3
:101ED000C533C451C55D0101806FD89080317F6FDB
:101EE0000001C6390F0B01017E6F140E0001C06F97
:101EF000C65119EC16F001017D6F160E0001C06F7E
:101F0000C65119EC16F001017C6F0001C651120098
:101F1000AA933C016AAB02D0010E01D0000E471813
:101F2000D8B405D0000E6ABB010E476E2AD056AB5E
:101F300027D09E50D8B424D001017C519E5CD8B0EB
:101F400002D04F0E17D07D519E5CD8B002D0270E24
:101F500011D07E519E5CD8B002D0130E0BD07F51B1
:101F60009E5CD8B002D0090E05D080519E5CD8B0DE
:101F700003D0040E462604D081519E5CD8A0462A88
:101F8000462A010E0101A86F1200C16F05D0000E94
:101F900001D0010EC06F21D00001C1510A0AD8B48E
:101FA000F6D7010AD8B4F3D7070AD8B4F0D7010A94
:101FB000D8B4EDD7030AD8B4EAD7240AD8B4E7D7FF
:101FC000190AD8B4E4D7070AD8B4E1D7010AD8B4BB
:101FD000DED70C0AD8B4DBD7DCD70A0EBC6FC151F0
:101FE0008AEC17F0080AD8B408D00A0EBC6FC151A9
:101FF0008AEC17F0090AD8A402D0000EC06FC051B5
:10200000120001011C511D11D8B402D0010EA86F9D
:102010000001A551D8B403D0010E0101A86F010140
:10202000A805D8A406D0000E216F000E206F000E68
:10203000A86F0001AE51D8A406D0B551D8A403D0E2
:10204000AF51D8B402D0000E01D0010E0101BB6F18
:10205000BB05D8A41200E00E205D2E0E2159D8A099
:102060001200060E0001A419D8B41200A4C0A3F0F7
:10207000060EA46F010EA16F12004704D8A422D04F
:102080004650BE6FBF6BBE1DC06FBF1DC16FBC5140
:10209000C05DBD51C159D8B003D0BC69BD6904D081
:1020A0004650BC27000EBD23BC510101085D000154
:1020B000BD5101010959D8B014D008C1BCF009C103
:1020C000BDF00FD04650BC5D000EBD59D8B005D054
:1020D000000EBD6F000EBC6F04D04650BC5F000EFA
:1020E000BD5B000E466EBCC0BCF0BDC0BDF01200B2
:1020F00001012A510001CA5DC26F01012B5100018B
:10210000CB59C36F000EC56F640EC46F0EEC14F094
:10211000C251956F0101745100019519D8B40DD0C9
:1021200001012A510001CA5D01012B510001CB5967
:10213000D8A003D0010E0101736F0001CA51010143
:102140002A5D0001CB5101012B59D8A0120010ECDF
:1021500000F003D077ECFDF04F6E4F50D8B4FAD7B3
:102160009FEC19F01200000E926E010E0101D96F62
:10217000150E5924D96EDA6A020EDA226F00A3F71F
:10218000DFFF592A140E596402D0000E596E030E57
:102190005918D8B417C2E0F15950276E286AE05197
:1021A000296E2A6A040E2926000E2A222750291891
:1021B00012E128502A18D8A40ED0000ED96F59C0A9
:1021C000DEF1000E596E5AC023F05B508CEC09F022
:1021D0000101DF6F1200000ED86F1200C96FC9C075
:1021E000CAF0BDC0CBF0BEC0CCF0BFC0CDF0C0C007
:1021F000CEF0C1C0CFF0C2C0D0F0C3C0D1F0C4C0D7
:10220000D2F0C5C0D3F0C6C0D4F0C7C0D5F0C8C0A6
:10221000D6F0BA90E40E00D000D0E82EFCD700D063
:1022200000D0BA80BB98000E0001D76FBB9AD7517F
:10223000CA0FD96EDA6ADF5034EC19F0BB8A00019C
:10224000D72B0C0ED765F2D7BB881200C16FC1C067
:10225000B6F00001B651B6253D016F6FFE0E706FEE
:10226000010E0101B36F010E6B6F000E0201996F39
:10227000000E0001B06F010E0101AE6F000E696F1C
:102280003E04D8A40FD0000E0001606FC051D8B436
:1022900002D00C0E01D0000E616F000E626F000EB6
:1022A000636F08D0000E0001606FC051D8B4F3D73F
:1022B0001C0EF2D7040E42EC08F01200420E000190
:1022C000B66FB651B6253D016F6FFE0E706F000EF2
:1022D000716F000E726F000E746F100E756F000E2E
:1022E0007B6F6C69900E736F3901A29FA3933D01C0
:1022F00079953901A391A3953D0176997997390193
:10230000928F93833D017A853901938193853D01B5
:1023100076817A87210E3A01136F000E3D01796FA5
:10232000000E766F73991200C15104E1020EC05D78
:10233000D8A012D0C15110E11F0EC05DD8A0C0B10D
:102340000BD0FF0EC025BC6FFF0EC121BD6F09EC85
:1023500019F05A0AD8B412D00001C15104E1210E7B
:10236000C05DD8A01200FF0EC025BC6FFF0EC121BA
:10237000BD6F09EC19F05B0AD8A41200FF0E000132
:10238000C025BC6FFF0EC121BD6FFF0EBE6F3CECC0
:1023900015F0120001013805D8A41CD0000E386FCA
:1023A000000E3B6F000E3A6F000E0001CC6F37C07D
:1023B000CDF038C0CEF0020ED06F020ECF6F040EFB
:1023C000D26F040ED16F090E2DECDCF0CCC037F0CB
:1023D000CDC038F001013905D8A402D0000E396F04
:1023E0003BC1DCF0395071ECF5F001013A6F3B5123
:1023F0003A19D8B412003AC13BF1120001011C5144
:102400001D11D8B402D0010EA86F0001A551D8B497
:1024100003D0010E0101A86F5050D8A403D0010EC3
:102420000101BA6F0101A805D8A408D0000E02016D
:10243000646F000E636F000E0101A76FA00E020112
:10244000635D0F0E6459D8A012000001AE51D8A4EC
:102450001200B551D8A41200010E0101A76F12009D
:10246000BD6F010E0001BC6FBD05D8A402D0010EE6
:1024700023D0020EBD19D8A402D0020E1DD0040E26
:10248000BD19D8A402D0030E17D0080EBD19D8A4C8
:1024900002D0040E11D0100EBD19D8A402D0050E22
:1024A0000BD0200EBD19D8A402D0060E05D0400EC8
:1024B000BD19D8A402D0070EBC6FBC511200CB6F5F
:1024C0000001C851D8B40DD0C851070BC46F180E05
:1024D000FCEC16F0020E0001C46F150EFCEC16F0B9
:1024E00005D0010EC46F150EFCEC16F00001CB51A7
:1024F000D8B40DD0CB51070BC46F190EFCEC16F0FD
:10250000020E0001C46F160EFCEC16F01200010E54
:10251000C46F160EFCEC16F01200000EDE6F000EFB
:10252000DF6F000EE06F000EE16F000EE46F000E33
:10253000E56F000EEA6F000EEC6F000EF16F000EFB
:10254000F36F000EF46F000EF56F000EF66F000EC5
:10255000F76F000EF96F000EFA6F000EFB6F000EA2
:10256000FC6F030EFD6F000EFE6F1F0EFF6F840EDB
:10257000F86F1200AE0E0001CE6F470ECF6FA10EA6
:10258000D06F3F0ED16FEDC0BCF0EEC0BDF0BE6BA2
:10259000BF6B000E01EC02F0BCC0CAF0BDC0CBF0B6
:1025A000BEC0CCF0BFC0CDF073ECE8F0CAC0E3F021
:1025B000CBC0E4F0CCC0E5F0CDC0E6F09FECFFF07E
:1025C000E3C0EDF0E4C0EEF01200AE0E0001CE6FFD
:1025D000470ECF6FA10ED06F3F0ED16FEDC0BCF094
:1025E000EEC0BDF0BE6BBF6B000E01EC02F0BCC0D4
:1025F000CAF0BDC0CBF0BEC0CCF0BFC0CDF073EC14
:10260000E8F0CAC0E3F0CBC0E4F0CCC0E5F0CDC048
:10261000E6F09FECFFF0E3C0EDF0E4C0EEF0120056
:10262000000E0001CE6F000ECF6F800ED06F3F0EF8
:10263000D16FEDC0BCF0EEC0BDF0BE6BBF6B000E45
:1026400001EC02F0BCC0CAF0BDC0CBF0BEC0CCF003
:10265000BFC0CDF073ECE8F0CAC0E3F0CBC0E4F04B
:10266000CCC0E5F0CDC0E6F09FECFFF0E3C0EDF0AC
:10267000E4C0EEF01200140E0001CE6FAE0ECF6F6C
:10268000C70ED06F3F0ED16FEDC0BCF0EEC0BDF0F5
:10269000BE6BBF6B000E01EC02F0BCC0CAF0BDC047
:1026A000CBF0BEC0CCF0BFC0CDF073ECE8F0CAC038
:1026B000E3F0CBC0E4F0CCC0E5F0CDC0E6F09FEC99
:1026C000FFF0E3C0EDF0E4C0EEF01200050E0001F3
:1026D000BC5D100EBD59D8A002D0640E12001F0EB2
:1026E000BC5D0F0EBD59D8A002D0500E1200610E75
:1026F000BC5D0E0EBD59D8A002D03C0E1200C10E1A
:10270000BC5D0D0EBD59D8A002D0280E1200E50EFA
:10271000BC5D0C0EBD59D8A002D0140E1200000EE4
:1027200012000001C76F000E0001C56F000EC66FDA
:10273000640EC06FC75119EC16F0300FC46F0A0E4B
:10274000C06F640EBC6FC7518AEC17F019EC16F01D
:10275000300FC56F0A0EBC6FC7518AEC17F0300FEF
:10276000C66FC4C0F8F22E0E0201F96FC5C0FAF2AE
:10277000C6C0FBF21200C16FBEC0C2F0BFC0C3F042
:10278000B5EC17F00001C151C1253D01586F6AEC4D
:1027900018F0600003F356FD3D015D8B57EC18F017
:1027A0000CD060000BF3D9FF60000FF3DAFFDF50AD
:1027B00016EC17F00001C24BC32B0001C007C02963
:1027C000D8A4EFD7A3EC18F012000101E805D8A4B3
:1027D000120075C2EDF076C2EEF0BAEC12F0EDC068
:1027E00059F2EEC05AF2A10E0201595D0F0E5A596C
:1027F000D8A006D00001B551D8A402D0010E01D056
:10280000000E0101AC6F0001AE510101AC19D8B44A
:102810001200ACC1AEF0010E7B6F1200000EC86F4B
:10282000000EC76FC451C511D8B41CD0010EC66FBD
:1028300004D0D890C437C537C62BC5AFFAD7D890C7
:10284000C737C837C451C25DC551C359D8A005D0D8
:10285000C451C25FC551C35BC781D890C533C4336F
:10286000C62FEDD7C7C0C2F0C8C0C3F01200000128
:10287000BD6F4704D8A411D04650FF0A0001BC6FB9
:10288000BD51BC5DD8B002D0BD6902D04650BD2755
:10289000110EBD6511D0110E0ED00001BD51465C68
:1028A000D8A003D0010EBD6F02D04650BD5F070E09
:1028B000BD6102D0070EBD6F000E466EBD51120005
:1028C0000001BD6F0001BD05D8A40FD0BB98BB9A15
:1028D000A00E34EC19F0BB8A350EE82EFED700F0BE
:1028E000BB9AC80E34EC19F00ED0BB98BB9AA10E5F
:1028F00034EC19F0BB8A350EE82EFED700F0BB9AF7
:10290000C00E34EC19F0BB8ABB880001BD51120027
:10291000D86FD8C0D9F01DD0510EC26FFC0EC36F56
:10292000660EC46F010EC56F000EC66F000EC76F36
:10293000D9C0C8F0000EC96F000ECA6F000ECB6F71
:10294000000ECC6F000ECD6FD7C0CEF0BAEC00F009
:10295000D92B0001D951D65DD8A01200DDD7BD6FAB
:102960004704D8A413D04650FF0A0001BC6FBD51E4
:10297000BC5DD8B002D0BD6902D04650BD27BD5164
:102980003C5CD8B00DD03CC0BDF00AD04650000130
:10299000BD5DD8B003D0000EBD6F02D04650BD5F04
:1029A000000E466EBD511200BD6F4704D8A411D071
:1029B0004650FF0A0001BC6FBD51BC5DD8B002D0CB
:1029C000BD6902D04650BD27040EBD650CD0040E73
:1029D00006D046500001BD5DD8B003D0000EBD6FDB
:1029E00002D04650BD5F000E466EBD51120001017F
:1029F000D951D8A41AD034C1BCF0A50E0001BC65D1
:102A000002D0640E0BD09B0EBC6502D0420E06D0E5
:102A1000960EBC6502D0210E01D0000EBC6F34C1F1
:102A200068F1010E0101676F02D066C1BCF00001C0
:102A3000BC5112003C0174AB04D00001BC6BBC2B38
:102A400002D00001BC6B3C0174AB02D0010E01D07E
:102A5000000E0101B719D8B402D0010E01D0000E4A
:102A60000001BC15BD6F3C01000E74BB010E0101DD
:102A7000B76F0001BD511200000ED2BE010EBF6F34
:102A8000BD51030B3901E16F6000F3F2E0F9600022
:102A9000FBF2E3F93F0EE517E585D29E550EE66F92
:102AA000AA0EE66FE583E5B3FED7E5950001BFB159
:102AB00002D0D29E01D0D28E1200BE51BF11D8B426
:102AC00018D0010EC06F04D0D890BE37BF37C02BCE
:102AD000BFAFFAD7BE51BC5DBF51BD59D8A004D01D
:102AE000BE51BC5FBF51BD5BD890BF33BE33C02F5A
:102AF000F1D7BCC0BCF0BDC0BDF01200000EB36E7B
:102B0000000EB46E050EB56EEC0EB16E780EB06EA2
:102B1000B0506F00C4FEBCF00001BD6BBCC0BDF086
:102B2000BC6BBC110201FD6F0001BD510201FE6FC3
:102B30003901A4919481010EB26E1200000E9B6EB9
:102B4000000E9C6E020E9D6EE20E996E000E986E47
:102B500098506F0064FEBCF00001BD6BBCC0BDF0BE
:102B6000BC6BBC110301FB6F0001BD510301FC6F85
:102B70003901A89D010E9A6E1200C95101011C1560
:102B80000001C26FCA5101011D150001C36FC9C008
:102B9000C4F0CAC0C5F00EEC14F0C251CB6FCB51DB
:102BA000D8B407D00A0EA419D8A403D0010E01018D
:102BB000836F0001CB511200C9510201531500016E
:102BC000C26FCA51020154150001C36FC9C0C4F0DD
:102BD000CAC0C5F00EEC14F0C251CB6FCB51D8B4C3
:102BE00007D00A0EA419D8A403D0010E0101836FE7
:102BF0000001CB511200000E0001BE6FCABE02D010
:102C0000010E01D0000EBE6FBE51A719BD6FBD51A0
:102C1000BE15A56FBE51D8A403D0BC6BBC2B02D08F
:102C20000001BC6BBD51BE19BC15A66FBEC0A7F09C
:102C30001200C16F000E0001C36FC051D8B415D08F
:102C4000010EC26F03D0D890C037C22BC0AFFBD7E4
:102C5000D890C337C051C15DD8A003D0C051C15F67
:102C6000C381D890C033C22FF3D7C35112000201E1
:102C7000FF51D8B410D0EB0E5824D96EDA6A010E89
:102C8000DA22DF503D01EA6F582A150E58640AD047
:102C9000150E586E07D039019399000E0101D76FB8
:102CA000000E596E0201FF071200350EC26FFA0EB8
:102CB000C36F0B0EC46F010EC56F060EC66F3F0EBD
:102CC000C76F000EC86F010EC96F000ECA6F000EED
:102CD000CB6F000ECC6F000ECD6FF6C0CEF0BAEC0D
:102CE00000F01200350EC26FFA0EC36F0B0EC46FE8
:102CF000010EC56F010EC66F3F0EC76F000EC86F85
:102D0000010EC96F000ECA6F000ECB6F000ECC6FA4
:102D1000000ECD6FF6C0CEF0BAEC00F012000D0E32
:102D2000206012001EC00FF01FC010F020C011F074
:102D3000000E126E000E136E000E146E000E166E54
:102D4000000E156E000E176E000E196E000E186E36
:102D5000000EDBEC06F01200E90E0001CA6FFE0E59
:102D6000CB6F000ECC6F000ECD6F000ECE6F000E3D
:102D7000CF6F000ED16F000ED06F000ED26F000E1D
:102D8000D46F000ED36F050E5CEC04F0120000014E
:102D9000BD6F1F0E0001BD6502D01F0EBD6FBB9839
:102DA000BB9A270E34EC19F0BB8ABB9A810E34EC27
:102DB00019F0BB8ABB9A0001BD5134EC19F0BB8AF3
:102DC000BB881200C56FDF0E0001C66F020EC76F11
:102DD000C5C0DFF2C4C0E0F2080EC4611200C451E5
:102DE000D8B41200C6C0BEF0C7C0BFF0020EC06F9C
:102DF000580EBBEC13F01200C56FDF0E0001C66F5A
:102E0000020EC76FC5C0DFF2C4C0E0F2080EC46195
:102E10001200C451D8B41200C6C0BEF0C7C0BFF083
:102E2000020EC06F580EBBEC13F012000001BC6F15
:102E30000001BD695750D8A412000BD03D0162AB10
:102E400004D06000F3F255FD1200050EE82EFED707
:102E500000F00001BD2FF2D7010E576E1200050ED3
:102E6000576F000E586F070E596F010E5A6F070EFD
:102E70005B6F110E5C6F000E5D6F220E5E6F000EB9
:102E80005F6F9B0E566F3901AA939A831200010E51
:102E9000966E000E956E000E976E9368000E926E01
:102EA000A9919981000E0001BC6F000EBD6F000E4C
:102EB000BE6F88EC19F0D00E946E12000F0E3C011C
:102EC0006B6F000E6C6F010E6D6F270E6E6F070E2D
:102ED0006F6F260E706F190E716F290E726F160EBE
:102EE000736F830E6A6F12000A0E3C01756F0E0E2F
:102EF000766F050E776F050E786F050E796F020EEF
:102F00007A6F000E7B6F000E7C6F000E7D6F860E59
:102F1000746F1200BD6F080E0001BE6F000EBF6F10
:102F2000D890BD35BF35BF6FD890BD37BC51BF5DA0
:102F3000D8A002D0BC51BF5FBE2FF2D7BF51120044
:102F4000BC6F0001BC05D8A40BD0010EBD6F120EE2
:102F50003D6408D0120E916F010E01015F6F02D027
:102F6000000EBD6F0001BD5112003D015DAF03D0E9
:102F70005750D8B41200000E576E800E5E6F200EB0
:102F80005F6F030E656F840E5D6F000E636F000E42
:102F9000606F1200B3C0B6F00001B351B3253D011C
:102FA0006F6FFE0E706F010E0101B36F010E4E6E5A
:102FB000010E0001B06F010E0101AE6F1200BC5195
:102FC000BE036F00CCFFC0F06F00D0FFC1F0BC515A
:102FD000BF03F350C127BD51BE03F350C127C0C08A
:102FE000BCF0C1C0BDF01200000EBF6F000EC06F7C
:102FF00009D0C051BC25D96E000EBD21DA6EDF505C
:10300000BF1BC02BBE51C05DD8A0F3D7BF5112006B
:10301000060E0001946503D0110E946504D00C0EC9
:10302000946F94C06FF1B151D8B403D0030EB16561
:103030001200020EB16F1200C951020155150001B4
:10304000C26FCA51020156150001C36FC9C0C4F056
:10305000CAC0C5F00EEC14F0C251CB6FCB511200B8
:10306000000E046E000E056E09D005500124D96EC5
:10307000000E0220DA6EDF50041A052A0350055CA8
:10308000D8A0F3D7045012000001BD6F010E01015A
:10309000D76FBCC0DCF1BCC0FFF2390193B905D0D9
:1030A0006000F7F2EAFD010E586E938912000001EC
:1030B000BC695750D8A4120007D03D015DAB120087
:1030C000050EE82EFED700F00001BC2FF6D7010E4A
:1030D000576E12000001BC695750D8A4120007D0E7
:1030E0003D0161BF1200050EE82EFED700F0000181
:1030F000BC2FF6D7010E576E12000001BC6F010104
:10310000E6510001BC19D8B408D03E01F89F600018
:10311000F3F2F1FEF88FF89DF8810001BC51120026
:103120006F0060FFBBF0390194B1A4A103D070EC33
:1031300019F005D099B1A9A102D08FEC19F0600067
:10314000EFF2D8FF1100BC695750D8A4120007D085
:103150003D0163B51200050EE82EFED700F0000118
:10316000BC2FF6D7010E576E1200B2A409D0B29050
:103170006000EBF2B1FF6000E7F2B0FFB280120036
:103180006000EBF2B1FF6000E7F2B0FF1200026EE8
:10319000010E0101D76F01C0DCF101C0FFF239015E
:1031A00093B905D060000BF0EAFD010E586E9389CB
:1031B0001200000EC06F000EC16F000EC26F000E35
:1031C000C36F000EC46F000EC56F000EC66F000EF9
:1031D000C76F12003E01F0510001BF6FBE6B3E0190
:1031E000EF510001BE25BC6F3E01000E0001BF2162
:1031F000BD6F1200040EA26E130EA16E140EA36E0C
:10320000F00E9F6E000E9E6E3901A791E00EA06E2B
:103210001200BD51030B3901E16F6000F3F2E0F9D8
:103220003F0EE517E58100F000F03901E35112008F
:10323000AE47A13FAE47A13F6666663F14AEC73FAB
:103240000000803F5E01052020202000060EAE6EAB
:10325000000EAD6E000EAF6E610EAB6E000EAA6E6C
:10326000A495C00EAC6E12000001BC6F010E3D01B2
:10327000126F6000F3F211FD3901A2A9FDD73D01E3
:1032800010511200200E3D01156F030E166F070E30
:10329000196F010E1C6F830E146F1200600E39013E
:1032A000D96F000EDB6F000EDD6F080EDF6F000EB2
:1032B000DE6F1200D28A39018381838383878389F9
:1032C0008385828F8A8384918991120000019251B3
:1032D000D8B403D0ECECFEF0120048EC0AF0120077
:1032E000A491FDC2B9F0FEC2BAF0B5EC18F051ECF1
:1032F000F9F01200BCC0F5F3BDC0F6F3BEC0F7F3A1
:103300001200BCC0F8F3BDC0F9F3BEC0FAF312005E
:10331000BCC0F2F3BDC0F3F3BEC0F4F31200A99138
:10332000010E0101E46F000E596E12000001BC6F26
:103330000001BC511200820E3E01C16F1200BE920C
:10334000C6921200AC8E1200B2801200AA93120034
:1033500001FFFFFFFFFFFFFFFFFFFFFFFFFFFFFF7B
:10336000FFFFFFFFFFFFFFFFFFFFFFFFFFFFFFFF6D
:10337000FFFFFFFFFFFFFFFFFFFFFFFFFFFFFFFF5D
:10338000FFFFFFFFFFFFFFFFFFFFFFFFFFFFFFFF4D
:10339000FFFFFFFFFFFFFFFFFFFFFFFFFFFFFFFF3D
:10AE6000FFFF0000000000000000000000000000E4
:10AE700000FEFE00000000007F7F60606060608078
:10AE8000C0C0C0C0C0803F7F6060607F3FFEFE00EA
:10AE900080C0C0407F7F1F3B716040000060600049
:10AEA000000000000C0C000000F0FC1E061EFCF070
:10AEB0007F7F0303037F7FC0E0F070E0FEFE1F3F53
:10AEC0007870387F7FF0F080C0E070707F7F030182
:10AED00000000000000000000000005A776569745F
:10AEE00065204C6F6B00496E746572666163650026
:10AEF00050726F6772616D005374617475730053A3
:10AF00006574757000A100000000000000000000E2
:10AF10000000000000000000000000000000000031
:10AF20000000000000000000000000000000000021
:10AF30000000000000000000000000000000000011
:10AF40000000000000000000000000000000000001
:10AF500000000000000000000000000000000000F1
:10AF600000000000000000000000000000000000E1
:10AF700000000000000000000000000000000000D1
:10AF800000000000000000000000000000000000C1
:10AF900000000000000000000000000000000000B1
:10AFA00000000000000000000000000000000000A1
:10AFB0000000000000000000000000000000000091
:10AFC0000000000000000000000000000000000081
:10AFD0000000000000000000000000000000000071
:10AFE0000000000000000000000000000000000061
:10AFF0000000000000000000000000000000000051
:10B000000000000000000000000000000000000040
:10B010000000000000000000000000000000000030
:10B020000000000000000000000000000000000020
:10B030000000000000000000000000000000000010
:10B040000000000000000000000000000000000000
:10B050000000000000000000000000FE02020202EA
:10B0600002020202020202020202020202020202C0
:10B0700002020202020202020202020202020202B0
:10B0800002020202020202020202020202020202A0
:10B09000020202020202020202020202FE0000FF9B
:10B0A00000000000000000000000000000000000A0
:10B0B0000000000000000000000000000000000090
:10B0C0000000000000000000000000000000000080
:10B0D0000000000000000000000000000000000070
:10B0E000FF0000FF00000000000000000000000062
:10B0F0000000000000000000000000000000000050
:10B10000000000000000000000000000000000003F
:10B11000000000000000000000000000000000002F
:10B1200000000000FF0000FF000000000000000021
:10B13000000000000000000000000000000000000F
:10B1400000000000000000000000000000000000FF
:10B1500000000000000000000000000000000000EF
:10B160000000000000000000FF00007F4040404061
:10B1700040404040404040404040404040404040CF
:10B1800040404040404040404040404040404040BF
:10B1900040404040404040404040404040404040AF
:10B1A0004040404040404040404040407F0000FE22
:10B1B0000202020202020202020202020202FA3247
:10B1C000C202FA0282424242820242FA420202FA77
:10B1D000824242820282424282C202FA020242FA5F
:10B1E00042020202020202020202020202020202FF
:10B1F000FE0000FF00000000808000800080000052
:10B2000000800780E0931700F30484840300008328
:10B21000840400F700808007000384840207800311
:10B2200084840003040400000000A00080008080EB
:10B2300000000000FF0000FF000000070808050FE5
:10B2400000070808040F00000F0000000F010000B5
:10B250000F00070A0A0B000F0908080700070A0A6F
:10B260000B000F0100000F000000000000000F00A5
:10B270000F0100000F000000FF0000FF00000000B1
:10B2800000000000000000000000000000000000BE
:10B29000000000FF0101010101FF000000FF0101AA
:10B2A000010101FF0000000000000000000000009C
:10B2B000000000000000000000000000FF00007F10
:10B2C000404040404040404040404040404040407E
:10B2D00040404040404040FF8080808080FF4040B0
:10B2E00040FF8080808080FF4040404040404040A0
:10B2F000404040404040404040404040404040404E
:10B300007F0000FE02020202FA02020202E29AE258
:10B310000202FA82422202FA82422202C20202029D
:10B32000C202824242420242FA4202028242428205
:10B33000C202C2824242820282424282FA02020275
:10B34000FA020202FE0000FF00008080058000F08B
:10B35000078080000700878182040087818204F0D3
:10B360000384840207008485058200F0030484F0CE
:10B37000830404028780070080008780030404049C
:10B38000A700800085800000FF0000FF000708087C
:10B39000050F000F0908080700090A0A040007083A
:10B3A0000808000F0100000F00070808050F00073C
:10B3B00008080007080800070A0A0B000F01000030
:10B3C0000F0000000F000F0100000F00FF0000FF42
:10B3D000000000000000000000000000000000006D
:10B3E000000000FF0101010101FF0000FF01010158
:10B3F0000101FF000000FF0101010101FF00000049
:10B40000000000000000000000000000000000003C
:10B41000FF00007F404040404040404040404040AE
:10B4200040404040404040FF8080808080FF40405E
:10B43000FF8080808080FF404040FF80808080804F
:10B44000FF4040404040404040404040404040403D
:10B45000404040407F0000FE02020202020282429F
:10B460004282C202FA824242820282424242028204
:10B4700042424202FA824243820282424282C20233
:10B48000FA020242FA4202028242428202C282422C
:10B490004282020202020202FE0000FF00000000DF
:10B4A0000000030404020700070404040300040569
:10B4B0000502000304040400A70080008780030441
:10B4C0000402070003040400030404000305050547
:10B4D000000700000007000000000000FF0000FF60
:10B4E000000000000000000000000000000000005C
:10B4F0000000000000000000000000000F000F012D
:10B5000000000F000000000000000000000000002C
:10B51000000000000000000000000000000000002B
:10B52000FF0000FF0000000000000000000000001D
:10B530000000000000000000000000FF0101010108
:10B5400001FF000000FF0101010101FF00000000F8
:10B5500000000000000000000000000000000000EB
:10B5600000000000FF00007F40404040404040405D
:10B57000404040404040404040404040404040FF0C
:10B580008080808080FF404040FF8080808080FFFE
:10B5900040404040404040404040404040404040AB
:10B5A00040404040404040407F0000FE0202020216
:10B5B00002020202020202020202F2628202F202AB
:10B5C00002828282020282F2820202F202828202FB
:10B5D00002028282028202F2020282F282020202EB
:10B5E000020202020202020202020202FE0000FF46
:10B5F00000000000000000000000000000000F003C
:10B6000001060F0007080808070000070808000FD8
:10B610000100000F00070808050F000708080007D1
:10B62000080800000000000000000000000000000A
:10B63000FF0000FF00000000000000000000708814
:10B640008850F80078808040F80008FE090100FF6B
:10B65000100808F00070A8A8B000FF90888870005B
:10B6600070A8A8B000F8100808F000000000000062
:10B6700000000000FF0000FF0080008080000090BC
:10B68000000080808000F0008080000080F0800159
:10B6900000000000808000008000008000F00000BA
:10B6A00000008080008000800000008000F00080AA
:10B6B00080000080F0800000FF00007F404F41408C
:10B6C000404F404F4047484848404F4140404F401E
:10B6D00040474848404040474A4A4B404F4241401B
:10B6E0004047484840474848454F40474848444FEE
:10B6F000404F494848474040474848407F0000FE87
:10B700000202C232C2020202828202F202820202F9
:10B710008202028282020202828282020282828289
:10B7200002920202828202028202028202820202E9
:10B730000282028202828202020282820282020269
:10B74000FE0000FF000E0101010E00070808090FAE
:10B75000000F02010000070A0A0B00090A0A040090
:10B76000090A0A04000F00070A0A0B000F02010071
:10B7700000070808040F000F0100000F0007282829
:10B78000251F0000FF0000FF000000000000000077
:10B7900000000000000000000000000000F8100899
:10B7A00008F000F9007088888800FF100808F00091
:10B7B000087F8880000000000000000000000000FA
:10B7C0000000000000000000FF0000FF000000007B
:10B7D0000000000000000000000000E02020C02069
:10B7E00020C000C0242024C000C0202040E000FC75
:10B7F000000000E400C020202000FC402020C00009
:10B80000000000000000000000000000FF00007FBA
:10B810004040404040404040404040404040404325
:10B8200040404340404340414242424140414A4AF5
:10B8300049474041424240434041424242404340E6
:10B8400040404340404040404040404040404040F5
:10B850007F0000FE0202C242424282020202020253
:10B860000202020202020202020202020202420278
:10B8700002020202020202020202028242420202A8
:10B8800002020202C20202020202020202020202D8
:10B89000C2020202FE0000FF00003F060A12210061
:10B8A0001C2222143E003E0402023C001CA2A29470
:10B8B0007E003E001C2A2A2C003E0804020002FFE3
:10B8C00002001C2222143E003F0402023C003E08FB
:10B8D000040200021F222000FF0000FF0000000001
:10B8E0000000000000000000000000000000000058
:10B8F0000000000000000000000000000000000048
:10B900000000000000000000000000000000000037
:10B91000000000000000000000000000FF0000FF29
:10B920000000000000000000000000000000000017
:10B9300000000000E01010A0F000FE40A010001079
:10B94000FE100000F20030C000C030000000000017
:10B9500000000000000000000000000000000000E7
:10B96000FF00007F40404040404040404040404059
:10B9700040404040404040404041414041404140C3
:10B9800040414040404141404140404041404040B2
:10B9900040404040404040404040404040404040A7
:10B9A000404040407F0000FE02020202020202020A
:10B9B0000202020202020282828282020202020267
:10B9C0000202020202020202020202020202020257
:10B9D0000202020202020202020202020202020247
:10B9E0000202020202020202FE0000FF000000004A
:10B9F00000000000000000000000007F4444443BC1
:10BA0000007C1008040038545458007C0404780466
:10BA1000047800485454240038545458000000005E
:10BA2000000000000000000000000000FF0000FF18
:10BA30000000000000000000000000000000000006
:10BA400000000000000000000000000000000000F6
:10BA500000000000000000000000000000000000E6
:10BA600000000000000000000000000000000000D6
:10BA7000FF0000FF000000000000000000000000C8
:10BA80000000000000000000E01010A0F000FE40E8
:10BA9000A0100010FE100000F20030C000C0300006
:10BAA0000000000000000000000000000000000096
:10BAB00000000000FF00007F404040404040404008
:10BAC0004040404040404040404040404041414074
:10BAD0004140414040414040404141404140404060
:10BAE0004140404040404040404040404040404055
:10BAF00040404040404040407F0000FE02020202C1
:10BB000002020202C232C2020282020202820282E5
:10BB1000F282020202828282020282828202828295
:10BB2000020202828202820282F28202029202F205
:10BB3000020282020202020202020202FE0000FF70
:10BB4000000000000000000E0101010E00070808BF
:10BB5000040F000007C82820070808080700EF00A6
:10BB6000000F00000F0007080805EF000007080895
:10BB7000000F000F02050800010101010100000093
:10BB8000FF0000FF000000000000000000000000B7
:10BB90000000000000000000017F01000E11110AEA
:10BBA0001F001F0201011E001F04020100010F11EE
:10BBB0001000000000000000000000000000000075
:10BBC00000000000FF0000FF000000000000000077
:10BBD000000000000000000000000000E01010A0C5
:10BBE000F000FE40A0100010FE100000F20030C077
:10BBF00000C0300000000000000000000000000055
:10BC00000000000000000000FF00007F40404040B6
:10BC10004040404040404040404040404040404024
:10BC2000404141404140414040414040404141400D
:10BC30004140404041404040404040404040404002
:10BC40004040404040404040404040407F0000FE77
:10BC5000020202021AE202E21A0202C2A2A2C20214
:10BC600002E28242220202FA422222C20202EA02D4
:10BC700002E2422222C20202C2222242FA0202C28C
:10BC8000A2A2C20202E2422222C202020202020274
:10BC9000FE0000FFF8F8F8F8F8F8FBF8F8F8F8F903
:10BCA000FAFAFAF8F8FBF8F8F8F8F8FBFAFAFAF901
:10BCB000F8F8FBF8F8FBF8F8F8FBF8F8F9FA1A1AB4
:10BCC0001B1818191A1A1A18181B1818181B1818E4
:10BCD00018181818FF0000FF0303FBFBFBFBFBFB1E
:10BCE000FB0303FFFFFFFFFFFFFFFFFFFFFFFFFF60
:10BCF000FFFFFFFFFFFFFFFFFFFFFFFFFFFFFFFF54
:10BD0000FFFF0080C04040C08000C0C04040C080F5
:10BD10000040404040C0C000FF0000FFFE00E2F0D5
:10BD2000FAF8FAF0E200FEFFFFFFFFFFFFFFFFFF60
:10BD3000FFFFFFFFFFFFFFFFFFFFFFFFFFFFFFFF13
:10BD4000FFFFFFFFFFFF000F1F10101D0D001F1F43
:10BD500010101F0F00181C1613111000FF00007F99
:10BD6000414054414B434B415440417F7F7F7F7F53
:10BD70007F7F7F7F7F7F7F7F7F7F7F7F7F7F7F7FD3
:10BD80007F7F7F7F7F7F7F7F7F7F4040404040403D
:10BD900040404040404040404040404040404040A3
:10BDA0007F0000FE020202020202020202020202FE
:10BDB0000202020202E29AE2020202FA0282420253
:10BDC0000242FA42020202CA020282424242820253
:10BDD00002C2824242820202020202020202020203
:10BDE00002020202FE0000FF00000000000000004E
:10BDF000000000000000000007000000070000072E
:10BE00000102040000000304040000070000030412
:10BE10000404030000070000000700000000000009
:10BE20000000000000000000FF0000FF0000000014
:10BE3000000000000000000000000000000000F80A
:10BE4000100808F00000F90000708888880000FFE2
:10BE5000100808F00000087F888000000000000043
:10BE6000000000000000000000000000FF0000FFD4
:10BE700000804040800000C0008040000040F0484A
:10BE8000000080404040800000F80000000080403A
:10BE90004080C00000C00080400000804040800022
:10BEA00000C80000804040400000F8804040800012
:10BEB000FF00007F404345454540404741404040EA
:10BEC00040405F4040404344444443404043444436
:10BED0004040435454524F4040474140404040430B
:10BEE0004545454040474040434444444040474026
:10BEF000404047407F0000FE0202020202020202AE
:10BF0000020202020202020202826282020202E2D1
:10BF1000020202020202E202020202220202020201
:10BF200002020202020202020202020202020202F1
:10BF30000202020202020202FE0000FF00000000F4
:10BF40000000000000000000000000001C030203CD
:10BF50001C00001F040A110000010F111000001F37
:10BF600000000E1111110E00001F0201011E000041
:10BF7000000000000000000000000000FF0000FFC3
:10BF80000000000000000000000000000000C020D1
:10BF9000000000000000000000E0000000000000C1
:10BFA0000000000000000000000000000000000091
:10BFB00000200000000000000000E0000000000081
:10BFC000FF0000FF000E15151600001F04020100FF
:10BFD00000017F0100000E1111110E00000F101062
:10BFE00000000E51514A3F00001F04020100000EE4
:10BFF00015151600001F00000E11111100001F0280
:10C0000001011E00FF00007F404040404040404092
:10C010004040404040404040404040404040404020
:10C020004040404040404040404040404040404010
:10C030004040404040404040404040404040404000
:10C0400040404040404040407F0000FE020202026B
:10C0500002020202020202E29AE20202C2020202A8
:10C06000C20242FA420202824242428302028282B7
:10C07000820202F20A0A0AF20242F24A0A0242F278
:10C080004A0A02020202020202020202FE0000FF4B
:10C090000000000000000000000007000000070092
:10C0A000030404020700000304040003A40484033F
:10C0B00080800000000000030404040300001F004F
:10C0C0000000001F00000000000000000000000051
:10C0D000FF0000FF00000000000000000000000062
:10C0E0000000000000000000000000000000000050
:10C0F0000F000F0100000F00000000000000000012
:10C10000000000000000000000000000000000002F
:10C1100000000000FF0000FF000000000000000021
:10C12000000000000000000000000000000000FF10
:10C130000101010101FF000000FF0101010101FFF8
:10C1400000000000000000000000000000000000EF
:10C150000000000000000000FF00007F4040404061
:10C1600040404040404040404040404040404040CF
:10C17000404040FF8080808080FF404040FF8080C2
:10C18000808080FF40404040404040404040404030
:10C190004040404040404040404040407F0000FE22
:10C1A000020202020202FA020202028242424282B7
:10C1B00002FA8242220282424282C20282424282C7
:10C1C000FA02C282424202824242820282424242D7
:10C1D000028242424202824242820202020202027F
:10C1E000FE0000FF000000000000070404840003BC
:10C1F000040404830007818204000384848207F01E
:10C20000038484040700878080000083850505F08F
:10C2100004050582008485050200038505050000EC
:10C2200000000000FF0000FF000000000000000010
:10C230000001060C070C060100070A0A0B0007089C
:10C240000808000F0100000F00090A0A0400070A8D
:10C250000A0B00070808000F0100000F000000048F
:10C260000000000000000000FF0000FF00000000D0
:10C27000000000000000FF0101010101FF0000FFBC
:10C280000101010101FF0000FF0101010101FF00A7
:10C2900000FF0101010101FF00000000000000009B
:10C2A000000000000000000000000000FF00007F10
:10C2B00040404040404040404040FF80808080807F
:10C2C000FF4040FF8080808080FF4040FF80808072
:10C2D0008080FF4040FF8080808080FF4040404061
:10C2E000404040404040404040404040404040404E
:10C2F0007F000000000000000000000000000000BF
:10C30000000000000000000000000000000000002D
:10C31000000000000000000000000000000000001D
:10C32000000000000000000000000000000000000D
:10C3300000000000000000000000000000000000FD
:10C3400000000000000000000000000000000000ED
:10C3500000000000000000000000000000000000DD
:10C3600000000000000000000000000000000000CD
:10C370000000000000000000000000FCFA060606B5
:10C380000606060606060646A626262646060606CD
:10C39000868686060606860686860606060686863D
:10C3A00006E606060686868606060686068686064D
:10C3B0000606060606060606060606FAFC00003F06
:10C3C0005F60606060606060606060646869696A46
:10C3D000646060676A6A6A6360606F6160606F6012
:10C3E00060676868656F6060676A6A6A6360606FEB
:10C3F0006160606F60606060606060606060605F2E
:10C400003F0000FCFA0606E6C68606060606064655
:10C41000A62626264606060686868606060686067C
:10C42000868606060606868606E60606068686864C
:10C43000060606860686860606060606060686C6DC
:10C44000E60606FAFCFE003F5FE0E0EFE7E3E1E02E
:10C45000E0E0E0E4E8E9E9EAE4E0E0E7EAEAEAE388
:10C46000E0E0EFE1E0E0EFE0E0E7E8E8E5EFE0E082
:10C47000E7EAEAEAE3E0E0EFE1E0E0EFE0E0E0E075
:10C48000E0E1E3E7EFE0E0DFBF7FFF0305F9F9F963
:10C49000F9F9F9F9F9F9F9B959D9D9D9B9F9F9F98C
:10C4A000797979F9F9F979F97979F9F9F9F97979FC
:10C4B000F919F9F9F9797979F9F9F979F97979F9CC
:10C4C000F9F9F9F9F9F9F9F9F9F9F90503FFFFC0F3
:10C4D000A09F9F9F9F9F9F9F9F9F9F9B9796969593
:10C4E0009B9F9F989595959C9F9F909E9F9F909FA7
:10C4F0009F9897979A909F9F989595959C9F9F90AE
:10C500009E9F9F909F9F9F9F9F9F9F9F9F9F9FA04A
:10C51000C0FF00FCFA060606060606060606060624
:10C52000060606060606060606060606E6F636367B
:10C53000F6E6060606F6F6C6E676360606060606AB
:10C54000060606060606060606060606060606068B
:10C55000060606FAFC00003F5F6060606060606095
:10C5600060606060606060606060606060606060CB
:10C57000676F6C6C6F676060606F6F63676E6C6035
:10C5800060606060606060606060606060606060AB
:10C59000606060606060605F3F0000FCFA0606E675
:10C5A000C6860606060606060606060606060606EB
:10C5B00006060606E6F63636F6E6060606F6F6C67B
:10C5C000E67636060606060606060606060606068B
:10C5D00006060606060686C6E60606FAFCFE003FC6
:10C5E0005FE0E0EFE7E3E1E0E0E0E0E0E0E0E0E0B2
:10C5F000E0E0E0E0E0E0E0E0E7EFECECEFE7E0E0F7
:10C60000E0EFEFE3E7EEECE0E0E0E0E0E0E0E0E0E8
:10C61000E0E0E0E0E0E0E0E0E0E1E3E7EFE0E0DF01
:10C62000BF7FFF0305F9F9F9F9F9F9F9F9F9F9F912
:10C63000F9F9F9F9F9F9F9F9F9F9F9F91909C9C99A
:10C640000919F9F9F90909391989C9F9F9F9F9F94A
:10C65000F9F9F9F9F9F9F9F9F9F9F9F9F9F9F9F94A
:10C66000F9F9F90503FFFFC0A09F9F9F9F9F9F9F20
:10C670009F9F9F9F9F9F9F9F9F9F9F9F9F9F9F9FCA
:10C680009890939390989F9F9F90909C9891939F40
:10C690009F9F9F9F9F9F9F9F9F9F9F9F9F9F9F9FAA
:10C6A0009F9F9F9F9F9F9FA0C0FF00FCFA060606CA
:10C6B00006060606C6261626C60606F686464686DA
:10C6C0000606F6864646860606C6068646460606DA
:10C6D000C6060606C6060686464646860606F6864A
:10C6E0004646860606060606060606FAFC00003FD3
:10C6F0005F606060606060606F6161616F60606F0B
:10C700006468686760606F6468686760606F6160D4
:10C7100060606060676868646F60606768686864CC
:10C7200060606F6060606F60606060606060605FEC
:10C730003F0000FCFA0606E6C6860606C626162652
:10C74000C60606F6864646860606F68646468606E9
:10C7500006C6068646460606C6060606C6060686B9
:10C76000464646860606F68646468606060686C679
:10C77000E60606FAFCFE003F5FE0E0EFE7E3E1E0FB
:10C78000EFE1E1E1EFE0E0EFE4E8E8E7E0E0EFE44B
:10C79000E8E8E7E0E0EFE1E0E0E0E0E0E7E8E8E457
:10C7A000EFE0E0E7E8E8E8E4E0E0EFE0E0E0EFE039
:10C7B000E0E1E3E7EFE0E0DFBF7FFF0305F9F9F930
:10C7C000F9F9F9F939D9E9D939F9F90979B9B97919
:10C7D000F9F90979B9B979F9F939F979B9B9F9F9F9
:10C7E00039F9F9F939F9F979B9B9B979F9F9097969
:10C7F000B9B979F9F9F9F9F9F9F9F90503FFFFC0C0
:10C80000A09F9F9F9F9F9F9F909E9E9E909F9F9067
:10C810009B9797989F9F909B9797989F9F909E9F7D
:10C820009F9F9F9F9897979B909F9F989797979B65
:10C830009F9F909F9F9F909F9F9F9F9F9F9F9FA025
:10C84000C0FF00FE0202D20202C282424282020203
:10C85000C2020202C2020282424242820202C202B8
:10C8600082424202028242424282020202020202E8
:10C870000202020206FE0602826212120A0A121264
:10C8800062820206FE00007F40404F40404F404021
:10C89000404F404040434C4340404047494949494C
:10C8A00040404F41404040404044494B4A44404052
:10C8B0004040404040404040607F604041464848E2
:10C8C00050504848464140607F0000FE0202D202BC
:10C8D00002C2824242820202C2020202C2020282F8
:10C8E000424242820202C202824242020282424228
:10C8F00042820202020202020202020206FE060254
:10C90000826212120A0A121262820206FEFE003FC0
:10C9100040C0CFC0C0CFC0C0C0CFC0C0C0C3CCC358
:10C92000C0C0C0C7C9C9C9C9C0C0CFC1C0C0C0C0CC
:10C93000C0C4C9CBCAC4C0C0C0C0C0C0C0C0C0C0D1
:10C94000E0FFE0C0C1C6C8C8D0D0C8C8C6C1C0C01A
:10C95000BF7F00FE06FA2AFAFA3A7ABABA7AFAFAE7
:10C960003AFAFAFA3AFAFA7ABABABA7AFAFA3AFA27
:10C970007ABABAFAFA7ABABABA7AFAFAFAFAFAFAD7
:10C98000FAFAFAFA06FE060282E2F2F2FAFAF2F293
:10C99000E2820206FE00007F605F505F5F505F5FD3
:10C9A0005F505F5F5F5C535C5F5F5F5856565656E3
:10C9B0005F5F505E5F5F5F5F5F5B5654555B5F5FBD
:10C9C0005F5F5F5F5F5F5F5F607F604041474F4FCA
:10C9D0005F5F4F4F474140607F0000FE06FA2AFA32
:10C9E000FA3A7ABABA7AFAFA3AFAFAFA3AFAFA7AE7
:10C9F000BABABA7AFAFA3AFA7ABABAFAFA7ABABA97
:10CA0000BA7AFAFAFAFAFAFAFAFAFAFA06FE060222
:10CA100082E2F2F2FAFAF2F2E2820206FEFE003F4F
:10CA200060DFD0DFDFD0DFDFDFD0DFDFDFDCD3DCD4
:10CA3000DFDFDFD8D6D6D6D6DFDFD0DEDFDFDFDF41
:10CA4000DFDBD6D4D5DBDFDFDFDFDFDFDFDFDFDF1C
:10CA5000E0FFE0C0C1C7CFCFDFDFCFCFC7C1C0C0CD
:10CA6000BF7F00FE0202F2828282F20202F2929202
:10CA70009262020232428242320202020202020246
:10CA80000202020202020202020202020202020286
:10CA90000202020206FE0602826212120A0A121242
:10CAA00062820206FE00007F40404F4040404F40FF
:10CAB000404F4142444840404C4241424C4040403B
:10CAC0004040404040404040404040404040404066
:10CAD0004040404040404040607F604041464848C0
:10CAE00050504848464140607F0000FE0202F282FA
:10CAF0008282F20202F292929262020232428242F6
:10CB000032020202020202020202020202020202D5
:10CB100002020202020202020202020206FE0602F1
:10CB2000826212120A0A121262820206FEFE003F9E
:10CB300040C0CFC0C0C0CFC0C0CFC1C2C4C8C0C039
:10CB4000CCC2C1C2CCC0C0C0C0C0C0C0C0C0C0C0C8
:10CB5000C0C0C0C0C0C0C0C0C0C0C0C0C0C0C0C0D5
:10CB6000E0FFE0C0C1C6C8C8D0D0C8C8C6C1C0C0F8
:10CB7000BF7F00FE06FA0A7A7A7A0AFAFA0A6A6A25
:10CB80006A9AFAFACABA7ABACAFAFAFAFAFAFAFA55
:10CB9000FAFAFAFAFAFAFAFAFAFAFAFAFAFAFAFAF5
:10CBA000FAFAFAFA06FE060282E2F2F2FAFAF2F271
:10CBB000E2820206FE00007F605F505F5F5F505FB1
:10CBC0005F505E5D5B575F5F535D5E5D535F5F5FB0
:10CBD0005F5F5F5F5F5F5F5F5F5F5F5F5F5F5F5F65
:10CBE0005F5F5F5F5F5F5F5F607F604041474F4FA8
:10CBF0005F5F4F4F474140607F0000FE06FA0A7AB0
:10CC00007A7A0AFAFA0A6A6A6A9AFAFACABA7ABAA4
:10CC1000CAFAFAFAFAFAFAFAFAFAFAFAFAFAFAFAA4
:10CC2000FAFAFAFAFAFAFAFAFAFAFAFA06FE060240
:10CC300082E2F2F2FAFAF2F2E2820206FEFE003F2D
:10CC400060DFD0DFDFDFD0DFDFD0DEDDDBD7DFDFAF
:10CC5000D3DDDEDDD3DFDFDFDFDFDFDFDFDFDFDF01
:10CC6000DFDFDFDFDFDFDFDFDFDFDFDFDFDFDFDFD4
:10CC7000E0FFE0C0C1C7CFCFDFDFCFCFC7C1C0C0AB
:10CC8000BF7F00FE0202F2828282F20202F29292E0
:10CC90009262020202020202028202028202028204
:10CCA00082020282F28202028202028202028282F4
:10CCB0008202020206FE0602826212120A0A1212A0
:10CCC00062820206FE00007F40404F4040404F40DD
:10CCD000404F41424448404141414141404F42411F
:10CCE0004040474A4A4B4040474848404F424140F5
:10CCF0004047484848474040607F60404146484878
:10CD000050504848464140607F0000FE0202F282D7
:10CD10008282F20202F29292926202020202020203
:10CD2000028202028202028282020282F2820202F3
:10CD300082020282020282828202020206FE06024F
:10CD4000826212120A0A121262820206FEFE003F7C
:10CD500040C0CFC0C0C0CFC0C0CFC1C2C4C8C0C116
:10CD6000C1C1C1C1C0CFC2C1C0C0C7CACACBC0C087
:10CD7000C7C8C8C0CFC2C1C0C0C7C8C8C8C7C0C064
:10CD8000E0FFE0C0C1C6C8C8D0D0C8C8C6C1C0C0D6
:10CD9000BF7F00FE06FA0A7A7A7A0AFAFA0A6A6A03
:10CDA0006A9AFAFAFAFAFAFAFA7AFAFA7AFAFA7A53
:10CDB0007AFAFA7A0A7AFAFA7AFAFA7AFAFA7A7A43
:10CDC0007AFAFAFA06FE060282E2F2F2FAFAF2F2CF
:10CDD000E2820206FE00007F605F505F5F5F505F8F
:10CDE0005F505E5D5B575F5E5E5E5E5E5F505D5E88
:10CDF0005F5F585555545F5F5857575F505D5E5F92
:10CE00005F58575757585F5F607F604041474F4FAB
:10CE10005F5F4F4F474140607F0000FE06FA0A7A8D
:10CE20007A7A0AFAFA0A6A6A6A9AFAFAFAFAFAFA52
:10CE3000FA7AFAFA7AFAFA7A7AFAFA7A0A7AFAFA42
:10CE40007AFAFA7AFAFA7A7A7AFAFAFA06FE06029E
:10CE500082E2F2F2FAFAF2F2E2820206FEFE003F0B
:10CE600060DFD0DFDFDFD0DFDFD0DEDDDBD7DFDE8E
:10CE7000DEDEDEDEDFD0DDDEDFDFD8D5D5D4DFDFFE
:10CE8000D8D7D7DFD0DDDEDFDFD8D7D7D7D8DFDF01
:10CE9000E0FFE0C0C1C7CFCFDFDFCFCFC7C1C0C089
:10CEA000BF7F00FE0202F2828282F20202F29292BE
:10CEB0009262020202020202020202121212927232
:10CEC0000202221212926202028202020282020212
:10CED0000202020206FE0602826212120A0A1212FE
:10CEE00062820206FE00007F40404F4040404F40BB
:10CEF000404F41424448404041414141414040400F
:10CF00004E41404040404C4A4948484040484542D4
:10CF10004548404040404040607F6040414648486E
:10CF200050504848464140607F0000FE0202F282B5
:10CF30008282F20202F292929262020202020202E1
:10CF40000202021212129272020222121292620261
:10CF500002820202028202020202020206FE0602AD
:10CF6000826212120A0A121262820206FEFE003F5A
:10CF700040C0CFC0C0C0CFC0C0CFC1C2C4C8C0C0F5
:10CF8000C1C1C1C1C1C0C0C0CEC1C0C0C0C0CCCA77
:10CF9000C9C8C8C0C0C8C5C2C5C8C0C0C0C0C0C05C
:10CFA000E0FFE0C0C1C6C8C8D0D0C8C8C6C1C0C0B4
:10CFB000BF7F00FE06FA0A7A7A7A0AFAFA0A6A6AE1
:10CFC0006A9AFAFAFAFAFAFAFAFAFAEAEAEA6A8AE1
:10CFD000FAFADAEAEA6A9AFAFA7AFAFAFA7AFAFAE1
:10CFE000FAFAFAFA06FE060282E2F2F2FAFAF2F22D
:10CFF000E2820206FE00007F605F505F5F5F505F6D
:10D000005F505E5D5B575F5F5E5E5E5E5E5F5F5F53
:10D01000515E5F5F5F5F53555657575F5F575A5D6D
:10D020005A575F5F5F5F5F5F607F604041474F4F70
:10D030005F5F4F4F474140607F0000FE06FA0A7A6B
:10D040007A7A0AFAFA0A6A6A6A9AFAFAFAFAFAFA30
:10D05000FAFAFAEAEAEA6A8AFAFADAEAEA6A9AFA90
:10D06000FA7AFAFAFA7AFAFAFAFAFAFA06FE0602FC
:10D0700082E2F2F2FAFAF2F2E2820206FEFE003FE9
:10D0800060DFD0DFDFDFD0DFDFD0DEDDDBD7DFDF6B
:10D09000DEDEDEDEDEDFDFDFD1DEDFDFDFDFD3D5CA
:10D0A000D6D7D7DFDFD7DADDDAD7DFDFDFDFDFDFC5
:10D0B000E0FFE0C0C1C7CFCFDFDFCFCFC7C1C0C067
:10D0C000BF7F00FCFA0606060606060606060606EA
:10D0D00006060606060686E6763676E68606060620
:10D0E000F6F6060606F6F60606E6F6B6B6B6B63660
:10D0F00006060606060606060606060606060606D0
:10D10000060606FAFC00003F5F60606060606060D9
:10D110006060606060606060606E6F6363636363E3
:10D120006F6E6060676F6C6C6C6F6F60606C6D6D64
:10D130006D6D6F67606060606060606060606060BF
:10D14000606060606060605F3F0000FCFA0606E6B9
:10D15000C68606060606060606060606060686E6CF
:10D16000763676E686060606F6F6060606F6F6062F
:10D1700006E6F6B6B6B6B63606060606060606068F
:10D1800006060606060686C6E60606FAFCFE003F0A
:10D190005FE0E0EFE7E3E1E0E0E0E0E0E0E0E0E0F6
:10D1A000E0EEEFE3E3E3E3E3EFEEE0E0E7EFECEC08
:10D1B000ECEFEFE0E0ECEDEDEDEDEFE7E0E0E0E0EF
:10D1C000E0E0E0E0E0E0E0E0E0E1E3E7EFE0E0DF46
:10D1D000BF7FFF0305F9F9F9F9F9F9F9F9F9F9F957
:10D1E000F9F9F9F9F9F9791989E9891979F9F9F95F
:10D1F0000909F9F9F90909F9F91909494949C9F96F
:10D20000F9F9F9F9F9F9F9F9F9F9F9F9F9F9F9F98E
:10D21000F9F9F90503FFFFC0A09F9F9F9F9F9F9F64
:10D220009F9F9F9F9F9F9F9F9F91909C9C9C9C9C3A
:10D2300090919F9F989093939390909F9F93929299
:10D240009290989F9F9F9F9F9F9F9F9F9F9F9F9F11
:10D250009F9F9F9F9F9F9FA0C0FF00FCFA0606060E
:10D2600006060606060606060606060666969616CE
:10D2700026060686F68606060686464686C60606FE
:10D28000C606864646060686F6860606060606068E
:10D290000606060606060606060606FAFC00003F17
:10D2A0005F6060606060606060606060606060607F
:10D2B000646869696660606067686860606768681C
:10D2C000646F60606F616060606060606768686024
:10D2D0006060606060606060606060606060605F4F
:10D2E0003F0000FCFA0606E6C686060606060606A7
:10D2F000060606066696961626060686F68606062E
:10D300000686464686C60606C6068646460606863D
:10D31000F68606060606060606060606060686C6FD
:10D32000E60606FAFCFE003F5FE0E0EFE7E3E1E03F
:10D33000E0E0E0E0E0E0E0E0E4E8E9E9E6E0E0E0C9
:10D34000E7E8E8E0E0E7E8E8E4EFE0E0EFE1E0E08C
:10D35000E0E0E0E0E7E8E8E0E0E0E0E0E0E0E0E0B6
:10D36000E0E1E3E7EFE0E0DFBF7FFF0305F9F9F974
:10D37000F9F9F9F9F9F9F9F9F9F9F9F9996969E9AD
:10D38000D9F9F9790979F9F9F979B9B97939F9F95D
:10D3900039F979B9B9F9F9790979F9F9F9F9F9F9AD
:10D3A000F9F9F9F9F9F9F9F9F9F9F90503FFFFC004
:10D3B000A09F9F9F9F9F9F9F9F9F9F9F9F9F9F9F7C
:10D3C0009B979696999F9F9F9897979F9F989797BF
:10D3D0009B909F9F909E9F9F9F9F9F9F9897979F97
:10D3E0009F9F9F9F9F9F9F9F9F9F9F9F9F9F9FA04C
:10D3F000C0FF2A3E003E00F8080808080808080890
:10D4000008C8380000000000FF0000000000000015
:10D4100000F807000000000000FF0000000000000E
:10D42000C03F0000000000000000FF0000000000FE
:10D43000F80700000000001C221C000F0808080864
:10D440000F0000000000002A3E003E00F808080817
:10D45000080808080808C8380000000000FF00009D
:10D46000000000000000F807000000000000FF00BE
:10D470000000000000C03F0000000000000000FFAE
:10D480000000000000F80700000000001C221C0043
:10D490000F0C0C0C0C0F0000000000002A3E003E98
:10D4A00000F8080808080808080808C8380000003C
:10D4B0000000FF0000000000000000F8070000006E
:10D4C000000000FF000000000000C03F000000005E
:10D4D00000000000FF0000000000F807000000004E
:10D4E000001C221C000F0E0E0E0E0F00000000008C
:10D4F000002A3E003E00F808080808080808080846
:10D50000C8380000000000FF00000000000000001C
:10D51000F807000000000000FF000000000000C04D
:10D520003F0000000000000000FF0000000000F8C5
:10D530000700000000001C221C000F0F0F0F0F0F30
:10D540000000000000002A3E003E00F8080808081D
:10D550000808080808C8380000000000FF000000A4
:10D560000000000000F807000000000000FF0000BD
:10D5700000000000C03F0000000000000000FF802D
:10D5800080808080F80700000000001C221C000F33
:10D590000F0F0F0F0F0000000000002A3E003E009A
:10D5A000F8080808080808080808C838000000003B
:10D5B00000FF0000000000000000F807000000006D
:10D5C0000000FF000000000000C03F00000000005D
:10D5D000000000FFC0C0C0C0C0F80700000000008D
:10D5E0001C221C000F0F0F0F0F0F00000000000087
:10D5F0002A3E003E00F8080808080808080808C87D
:10D60000380000000000FF0000000000000000F8EB
:10D6100007000000000000FF000000000000C03F05
:10D620000000000000000000FFE0E0E0E0E0F8079C
:10D6300000000000001C221C000F0F0F0F0F0F0036
:10D6400000000000002A3E003E00F8080808080814
:10D6500008080808C8380000000000FF00000000AB
:10D6600000000000F807000000000000FF000000BC
:10D67000000000C03F0000000000000000FFF0F0CC
:10D68000F0F0F0F80700000000001C221C000F0F53
:10D690000F0F0F0F0000000000002A3E003E00F8B0
:10D6A000080808080808080808C838000000000032
:10D6B000FF0000000000000000F80700000000006C
:10D6C00000FF000000000000C03F0000000000005C
:10D6D0000000FFF8F8F8F8F8F80700000000001C58
:10D6E000221C000F0F0F0F0F0F0000000000002A78
:10D6F0003E003E00F8080808080808080808C8386E
:10D700000000000000FF0000000000000000F8071B
:10D71000000000000000FF000000000000C03F000B
:10D7200000000000000000FFFCFCFCFCFCFC07000B
:10D73000000000001C221C000F0F0F0F0F0F000035
:10D74000000000002A3E003E00F80808080808080B
:10D75000080808C8380000000000FF0000000000B2
:10D76000000000F807000000000000FF00000000BB
:10D770000000C03F0000000000000000FFFEFEFEB1
:10D78000FEFEFE0700000000001C221C000F0F0F11
:10D790000F0F0F0000000000002A3E003E00F808B6
:10D7A0000808080808080808C8380000000000FF3A
:10D7B0000000000000000000F8070000000000006A
:10D7C000FF000000000000C03F000000000000005B
:10D7D00000FFFFFFFFFFFFFF0700000000001C220B
:10D7E0001C000F0F0F0F0F0F0000000000002A3E5B
:10D7F000003E00F8080808080808080808C83800AB
:10D8000000000000FF0000000000000000F807001A
:10D810000000000000FF808080808080C03F00000A
:10D82000000000000000FFFFFFFFFFFFFF070000F8
:10D830000000001C221C000F0F0F0F0F0F00000034
:10D840000000002A3E003E00F80808080808080802
:10D850000808C8380000000000FF000000000000B9
:10D860000000F807000000000000FFC0C0C0C0C0FA
:10D87000C0C03F0000000000000000FFFFFFFFFFEE
:10D88000FFFF0700000000001C221C000F0F0F0FFD
:10D890000F0F0000000000002A3E003E00F80808BC
:10D8A00008080808080808C8380000000000FF0041
:10D8B00000000000000000F807000000000000FF6A
:10D8C000E0E0E0E0E0E0E03F0000000000000000F9
:10D8D000FFFFFFFFFFFFFF0700000000001C221CEE
:10D8E000000F0F0F0F0F0F0000000000002A3E0076
:10D8F0003E00F8080808080808080808C8380000AA
:10D90000000000FF0000000000000000F807000019
:10D9100000000000FFF0F0F0F0F0F0F03F00000039
:10D920000000000000FFFFFFFFFFFFFF07000000F7
:10D9300000001C221C000F0F0F0F0F0F0000000033
:10D9400000002A3E003E00F80808080808080808F9
:10D9500008C8380000000000FF00000000000000C0
:10D9600000F807000000000000FFF8F8F8F8F8F8E9
:10D97000F83F0000000000000000FFFFFFFFFFFF76
:10D98000FF0700000000001C221C000F0F0F0F0FEC
:10D990000F0000000000002A3E003E00F8080808C2
:10D9A000080808080808C8380000000000FF000048
:10D9B000000000000000F807000000000000FFFC6D
:10D9C000FCFCFCFCFCFC3F0000000000000000FF31
:10D9D000FFFFFFFFFFFF0700000000001C221C00EC
:10D9E0000F0F0F0F0F0F0000000000002A3E003E37
:10D9F00000F8080808080808080808C838000000E7
:10DA00000000FF0000000000000000F80700000018
:10DA1000000000FFFEFEFEFEFEFEFE3F00000000D6
:10DA200000000000FFFFFFFFFFFFFF0700000000F6
:10DA3000001C221C000F0F0F0F0F0F000000000032
:10DA4000002A3E003E00F8080808080808080808F0
:10DA5000C8380000000000FF0000000000000000C7
:10DA6000F807000000000000FFFFFFFFFFFFFFFFBF
:10DA70003F0000000000000000FFFFFFFFFFFFFF6E
:10DA80000700000000001C221C000F0F0F0F0F0FDB
:10DA90000000000000002A3E003E00F808080808C8
:10DAA0000808080808C8380000000000FF808080CF
:10DAB0008080808080F807000000000000FFFFFFEA
:10DAC000FFFFFFFFFF3F0000000000000000FFFF1E
:10DAD000FFFFFFFFFF0700000000001C221C000FDB
:10DAE0000F0F0F0F0F0000000000002A3E003E0045
:10DAF000F8080808080808080808C83800000000E6
:10DB000000FFC0C0C0C0C0C0C0C0F8070000000017
:10DB10000000FFFFFFFFFFFFFFFF3F0000000000CE
:10DB2000000000FFFFFFFFFFFFFF070000000000F5
:10DB30001C221C000F0F0F0F0F0F00000000000031
:10DB40002A3E003E00F8080808080808080808C827
:10DB5000380000000000FFE0E0E0E0E0E0E0E0F896
:10DB600007000000000000FFFFFFFFFFFFFFFF3F77
:10DB70000000000000000000FFFFFFFFFFFFFF07A5
:10DB800000000000001C221C000F0F0F0F0F0F00E1
:10DB900000000000002A3E003E00F80808080808BF
:10DBA00008080808C8380000000000FFF0F0F0F096
:10DBB000F0F0F0F0F807000000000000FFFFFFFFAA
:10DBC000FFFFFFFF3F0000000000000000FFFFFF1D
:10DBD000FFFFFFFF0700000000001C221C000F0FCA
:10DBE0000F0F0F0F0000000000002A3E003E00F85B
:10DBF000080808080808080808C8380000000000DD
:10DC0000FFF8F8F8F8F8F8F8F8F807000000000056
:10DC100000FFFFFFFFFFFFFFFF3F000000000000CD
:10DC20000000FFFFFFFFFFFFFF0700000000001CD8
:10DC3000221C000F0F0F0F0F0F0000000000002A22
:10DC40003E003E00F8080808080808080808C83818
:10DC50000000000000FFFCFCFCFCFCFCFCFCFC07E2
:10DC6000000000000000FFFFFFFFFFFFFFFF3F007D
:10DC700000000000000000FFFFFFFFFFFFFF0700A4
:10DC8000000000001C221C000F0F0F0F0F0F0000E0
:10DC9000000000002A3E003E00F8080808080808B6
:10DCA000080808C8380000000000FFFEFEFEFEFE67
:10DCB000FEFEFEFE07000000000000FFFFFFFFFF6A
:10DCC000FFFFFF3F0000000000000000FFFFFFFF1C
:10DCD000FFFFFF0700000000001C221C000F0F0FB9
:10DCE0000F0F0F0000000000002A3E003E00F80861
:10DCF0000808080808080808C8380000000000FFE5
:10DD0000FFFFFFFFFFFFFFFFFF0700000000000015
:10DD1000FFFFFFFFFFFFFFFF3F00000000000000CC
:10DD200000FFFFFFFFFFFFFF0700000000001C22B5
:10DD30001C000F0F0F0F0F0F0000000000002A3E05
:10DD4000003E00F8888888888888888888C83800D5
:10DD500000000000FFFFFFFFFFFFFFFFFFFF0700C6
:10DD60000000000000FFFFFFFFFFFFFFFF3F00007C
:10DD7000000000000000FFFFFFFFFFFFFF070000A3
:10DD80000000001C221C000F0F0F0F0F0F000000DF
:10DD90000000002A3E003E00F8C8C8C8C8C8C8C86D
:10DDA000C8C8C8380000000000FFFFFFFFFFFFFFEA
:10DDB000FFFFFF07000000000000FFFFFFFFFFFF65
:10DDC000FFFF3F0000000000000000FFFFFFFFFF1B
:10DDD000FFFF0700000000001C221C000F0F0F0FA8
:10DDE0000F0F0000000000002A3E003E00F8E8E8A7
:10DDF000E8E8E8E8E8E8E8E8380000000000FFFFAD
:10DE0000FFFFFFFFFFFFFFFF07000000000000FF14
:10DE1000FFFFFFFFFFFFFF3F0000000000000000CA
:10DE2000FFFFFFFFFFFFFF0700000000001C221C98
:10DE3000000F0F0F0F0F0F0000000000002A3E0020
:10DE40003E00F8F8F8F8F8F8F8F8F8F8F8380000B4
:10DE5000000000FFFFFFFFFFFFFFFFFFFF070000C5
:10DE600000000000FFFFFFFFFFFFFFFF3F0000007B
:10DE70000000000000FFFFFFFFFFFFFF07000000A2
:10DE800000001C221C000F0F0F0F0F0F00000000DE
:10DE90000000000000000000000000000000000082
:10DEA0000000000000000000000000000000000072
:10DEB0000000000000000000000000000000000062
:10DEC0000000000000000000000000000000000052
:10DED0000000000000000000000000000000000042
:10DEE0000000000000000000000000000000000032
:10DEF0000000000000000000000000000000000022
:10DF00000000000000000000000000000000000011
:10DF10000000000000000000000000000000000001
:10DF200000000000000000000000000000000000F1
:10DF300000000000000000000000000000000000E1
:10DF400000000000000000000000000000000000D1
:10DF500000000000000000000000000000000000C1
:10DF600000000000000000000000000000000000B1
:10DF700000000000000000000000000000000000A1
:10DF80000000000000000000000000000000000091
:10DF90000000000000000000000000000000000081
:10DFA0000000000000000000000000000000000071
:10DFB0000000000000000000000000000000000061
:10DFC0000000000000000000000000000000000051
:10DFD0000000000000000000000000000000000041
:10DFE0000000000000000000000000000000000031
:10DFF0000000000000000000000000000000000021
:10E000000000000000000000000000000000000010
:10E010000000000000000000000000000000000000
:10E0200000000000000000000000000000000000F0
:10E0300000000000000000000000000000000000E0
:10E0400000000000000000000000000000000000D0
:10E0500000000000000000000000000000000000C0
:10E0600000000000000000000000000000000000B0
:10E0700000000000000000000000000000000000A0
:10E080000000000000000080B0B4B6B63636363668
:10E09000363636363636363636360600000000F06E
:10E0A000F0F0F0F0F0F0F0F0F0E0C00000F0F0F090
:10E0B0000000C0E0F0F0F0F0F0F0F0E0C00000F0A0
:10E0C000F0F00000F0F0F00000000000000000F0B0
:10E0D000F0F0F0F0F0F0F0F0E0C00000F0F0F00050
:10E0E0000000000000000000000000606C6D6D6D1D
:10E0F0000D0100000000000000000000C0C0C0C012
:10E10000C0C0C0C000FFFFFF000000000000FFFF14
:10E11000FF0000F8F8F80000FFFFFFC0C0C0C0C05B
:10E12000FFFFFF0000F8F8F80000FFFFFF1E1E1EB3
:10E130001E1E1E0000F0F8FC3C3C3C3C3CFCFFFF7B
:10E140000000FFFFFF000000000000000000C0D83A
:10E15000DBDBDBDBC3C0C0C0C0C0C0C0C0C0C0C050
:10E160000000010101010101010100FFFFFFF0F0CA
:10E17000F0F0F0F0FF7F3F0000FFFFFF0000F0F144
:10E18000F3F3F3F3F3F3FF7F3F0000FFFFFF000023
:10E190003F7FFFF0F0F0F0F0F000003F7FFFF0F085
:10E1A000F0F0F0FF7F3F00003F7FFFF0F0F0F0F075
:10E1B000F000000206060606060606060606060625
:10E1C0000606060606000000000000000000000031
:10E1D000000000000000000000000000000000003F
:10E1E000000000000000000000000000000000002F
:10E1F000000000000000000000000000000000001F
:10E20000000000000000000000000000000000000E
:10E21000000000000000000000000000000000807E
:10E22000F8FE7E0600000000000080F8FE7E06007A
:10E2300080F8FE7E0E0E0E0E0E0E0E0ECEFEFC387A
:10E240000000000E7EFEF080000000000080E0F084
:10E250007C1E0F0301000000000000000000000011
:10E2600000000000000000000000000000000000AE
:10E27000000000000000000000000000000000009E
:10E28000000000C0F8FFFFC7C0C0C0C0C0C0C0F8D9
:10E29000FF3F0700C0F8FFFFC7C0C0C0C0C0C0C07C
:10E2A000F0FE7F0F01000000000000037FFFFCF084
:10E2B000783E0F0701000000000000000000000091
:10E2C000000000000000000000000000000000004E
:10E2D000000000000000000000000000000000003E
:10E2E00000000000000000E0FCFF1F030303030325
:10E2F0000303E3FFFF1F0300E0FCFF1F070F3FFDC9
:10E30000F1C101010101010000000000000080E0F6
:10E31000F07C1E0F0F3FFFF0C00000000000000067
:10E3200000000000000000000000000000000000ED
:10E3300000000000000000000000000000000000DD
:10E340000000000000000000000000607E7F1F0150
:10E35000000000000000607E7F1F0100607E7F1FC4
:10E36000010000000000030F3F7C7040000080C0EF
:10E37000F0783E0F0701000000000000010F7F7ED3
:10E38000700000000000000000000000000000001D
:10E39000000000000000000000000000000000007D
:10E3A000000000000000000000000000000000006D
:10E3B000000000000000000000000000000000005D
:10E3C000000000000000000000000000000000004D
:10E3D000000000000000000000000000000000003D
:10E3E000000000000000000000000000000000002D
:10E3F000000000000000000000000000000000001D
:10E40000000000000000000000000000000000000C
:10E4100000000000000000000000000000000000FC
:10E4200000000000000000000000000000000000EC
:10E4300000000000000000000000000000000000DC
:10E4400000000000000000000000000000000000CC
:10E4500000000000000000000000000000000000BC
:10E4600000000000000000000000000000000000AC
:10E47000000000000000000000000000000000009C
:10E48000808080808080808080808080808080808C
:10E49000808080808080808080808080808080807C
:10E4A000808080808080808080808080808080806C
:10E4B000808080808080808080808080808080805C
:10E4C000808080808080808080808080808080804C
:10E4D000808080808080808080808080808080803C
:10E4E00080000030F0F0F1793D3F3733F1F1F17900
:10E4F0003D3F3733F1F1F1793D3F3733F1F1F179B8
:10E500003D3F3733F1F1F1793D3F3733F1F1F179A7
:10E510003D3F3733F1F1F1793D3F3733F1F1F17997
:10E520003D3F3733F1F1F1793D3F3733F1F1F17987
:10E530003D3F3733F1F1F1793D3F3733F1F1F17977
:10E540003D3F3733010101000000000000000000E2
:10E550000000000000000000FCFC00000000000DB6
:10E560000D000000001C3C00001C3C0000000000EE
:10E5700000002020F02C20F02C120F02120F0202BB
:10E58000F0F898FE9898100819197F191F0F182491
:10E590002498E0380C301C07192424181834C4843B
:10E5A0000404000609101009061B00003C1C0000B2
:10E5B000000000000000000000E0F81C0C0000005B
:10E5C000071F3830000000000C1CF8E0000000308D
:10E5D000381F0700000080800000000000010100DB
:10E5E00000008080E0E08080000101070701010059
:10E5F0000000000000000000301E0E0000008080BF
:10E600008080808080010101010101010000000083
:10E610000000000000181800000000000000C030DA
:10E620000C00300C03000000F0F87C840CF8F00FB4
:10E630001F30213E1F0F30381CFCFC000000303022
:10E640003F3F303030381C0C9CF8F0383C3E3733BC
:10E650003130181C0C8C8CFCF818383031313F1FCD
:10E66000FCFC808080FCFC00010101013F3FFCFCC0
:10E67000CCCCCC8C0C18383030391F0FC0E0F0B83F
:10E680009C8C041F3F3131313F1F0C0C0C8CCCFC97
:10E6900078003E3F03010000F8FC8C8C8CFCF81FD6
:10E6A0003F3131313F1FF8FC8C8C8CFCF81839312C
:10E6B00031313F1F000060600000000000060600CE
:10E6C0000000000000606000000020301E0E00000E
:10E6D00080C06030180C040103060C183020606004
:10E6E000606060606006060606060606040C1830C8
:10E6F00060C0802030180C060301181C0C8CCCFC68
:10E700007800003737010000E0108848C810E007A3
:10E71000081112131209F0F89C8C9CF8F01F1F01CD
:10E7200001011F1FFCFCCCCCCCFC381F1F18181893
:10E730001F0FF8FC0C0C0C3C380F1F1818181E0E7D
:10E74000FCFC0C0C1CF8F01F1F18181C0F07FCFC1D
:10E75000CCCCCC0C0C1F1F1818181818FCFC8C8C77
:10E760008C0C0C1F1F0101010000F8FC0C8C8C9C10
:10E77000980F1F1819191F0FFCFCC0C0C0FCFC1F0C
:10E780001F0000001F1F00FCFC00000000001F1FF6
:10E79000000000000C0C0C0C0CFCFC0E1E38303879
:10E7A0001F0FFCFCC0E070381C1F1F0103070E1C6C
:10E7B000FCFC00000000001F1F1818181818FCFCB3
:10E7C00070E070FCFC1F1F0000001F1FFCFC3CF0F1
:10E7D00000FCFC1F1F00031E1F1FF0F81C0C1CF880
:10E7E000F0070F1C181C0F07FCFC8C8C8CFCF81F0E
:10E7F0001F0101010100F0F80C0C0CF8F0070F18D4
:10E800001A1C0F13FCFCCCCCCCFC781F1F01030797
:10E810001E1C70F8DCCC9C9830060C1C191D0F07D0
:10E820000C0C0CFC0C0C0C0000001F000000FCFC8D
:10E83000000000FCFC0F1F18180C1F1FFCFC8000C0
:10E8400080FCFC00030F1E0F0300FCFC00F800FC22
:10E85000FC0F1F1C0F1C1F0F0C3CF0C0F03C0C18D1
:10E860001E0701071E187CFCC0C0FC7C0000001FB6
:10E870001F0000000C0C8CCCEC7C3C1E1F1B1918DC
:10E880001818FCFC0C0C0C0C003F3F3030303000F2
:10E890000C30C000000000000000030C3000000C31
:10E8A0000C0C0CFCFC00303030303F3F6030180C5A
:10E8B00018306000000000000000000000000000B0
:10E8C000003030303030303000000C3C00000000B0
:10E8D0000000000000000060606060E0C00E1F1BD0
:10E8E0001B0F1F1FFCFC80C0C0C0801F1F0D18180D
:10E8F0001F0F80C0E06060E0C0070F1C18181C0CE0
:10E9000080C0C0C080FCFC0F1F18180D1F1FC0E086
:10E91000606060E0C00F1F1B1B1B1B0BC0C0F8FC1E
:10E92000CCCC0C00003F3F000000C0E0606060E025
:10E93000C001333636363F1FFCFCC0C0C0C0801F4C
:10E940001F0000001F1F00CCCC00000000001F1F94
:10E950000000000000000000ECEC001C3C30303FE8
:10E960003F00FCFC0080C0E0601F1F03070F1C1865
:10E97000FCFC0000000000070F1C181C0C00E0E06D
:10E9800060C060E0C01F1F001F001F1FE0E0C0E06C
:10E99000E0E0C01F1F0100001F1F80C0E060E0C05A
:10E9A00080070F1C181C0F07E0E0606060E0C03FAC
:10E9B0003F0606060703C0E0606060E0E00307066C
:10E9C00006063F3FE0E080C0C060601F1F010100FD
:10E9D0000000C0E0606060604008191B1B1B1E0C3B
:10E9E000C0C0FCFCC0C0C000000F1F181818E0E039
:10E9F000000000E0E0070F18180C1F1FE0E0000007
:10EA000000E0E000030F1C0F0300E0E0000000E066
:10EA1000E0070F1C0F1C0F0760E0800080E060180B
:10EA20001C0703071C18E0E0000000E0E00133339E
:10EA300033333F1F606060E0E0E0601C1E1F1B1965
:10EA4000181880C070080C0C0001030E1030300044
:10EA50000000FCFC00000000003F3F000000000C34
:10EA60000C0870C080003030100E0301C0E0E0C020
:10EA70000080C003010003070703FCF8F0E0C0803A
:10EA8000007F3F1F0F070301FCFE1F6183FEFC4355
:10EA9000474C484F47430C0E07FFFF0000404C4CCB
:10EAA0004F4F4C4C0C0E87C3E77E3C4E4F4F4D4CA6
:10EAB0004C4C0607036363FFFE464E4C4C4C4F47DD
:10EAC0003F7F606060FFFF40404040404F4F3F3F0E
:10EAD000333373E3C3464E4C4C4E4743F0F87C6EE1
:10EAE00067E3C1474F4C4C4C4F470383C3E3733F2D
:10EAF0001E404F4F40404040FEFF636363FFFE47B0
:10EB00004F4C4C4C4F473E7F636363FFFE464E4C79
:10EB10004C4C4F4760F0B0B0B03020444C4D4D4DA0
:10EB20004F460080C0E0F0F8FC0103070F1F3F7F55
:10EB30000000000000000040404040404040000015
:10EB400000000000000000000000000000000000C5
:10EB500000000000000000000000000000000000B5
:10EB600000000000000000000000000000000000A5
:10EB70000000000000000000000000000000000095
:10EB80000000000000000000000000000000000085
:10EB90000000000000000000000000000000000075
:10EBA0000000000000000000000000000000000065
:10EBB0000000000000000000000000000000000055
:10EBC0000000000000000000000000000000000045
:10EBD00010284444C4040404C44444281000000021
:10EBE000000000000000000000F008040404F4F439
:10EBF00004040484C4E467000000078484848484DB
:10EC00008484040404040408F00000FF00000000F1
:10EC1000FFFF1C3E77E3C1800000003E7FE3C1C1DF
:10EC2000C1C1C163FFFE00000000FF00003F2020C3
:10EC30002020232320202020212323202020282CB3
:10EC40002C2C2C2C2C2C2F27202020203F000000A7
:10EC5000000000000000000010284444C404040424
:10EC6000C444442810000000000000000000000020
:10EC700000F008040404F4F404040484C4E4670009
:10EC800000000784848484848484040404040408C5
:10EC9000F00000FF00000000FFFF1C3E77E3C18092
:10ECA0000000003E7FE3C1C1C1C1C163FFFE00009F
:10ECB0000000FF00003F3F3F3F3F3C3C3F3F3F3FA6
:10ECC0003E3C3C3F3F3F37333333333333333038CD
:10ECD0003F3F3F3F3F0000000000000000000000F9
:10ECE00010284444C4040404C44444281000000010
:10ECF000000000000000000000F008040404F4F428
:10ED000004040484C4E467000000078484848484C9
:10ED10008484040404040408F00000FFF8F8F8F800
:10ED20000707E4C68F1B3978F8F8F8C6873B3939EE
:10ED30003939399B0706F8F8F8F8FF00003F3F3FE4
:10ED40003F3F3C3C3F3F3F3F3E3C3C3F3F3F3733F4
:10ED500033333333333330383F3F3F3F3F000000DE
:10ED6000000000000000000010284444C404040413
:10ED7000C44444281000000000000000000000000F
:10ED800000F0C8C4C4C43434C4C4C4440424A7C0F8
:10ED9000C0C0C744444444444444C4C4C4C4C4C8B4
:10EDA000F00000FFFFFFFFFF0000E3C1881C3E7F73
:10EDB000FFFFFFC1803C3E3E3E3E3E9C0001FFFF08
:10EDC000FFFFFF00003F3F3F3F3F3C3C3F3F3F3F97
:10EDD0003E3C3C3F3F3F37333333333333333038BC
:10EDE0003F3F3F3F3F0000000000000000000000E8
:10EDF00010387C7CFCFCFCFCFC7C7C3810000000A7
:10EE0000000000000000000000F0F8FCFCFC0C0C0E
:10EE1000FCFCFC7C3C1C9FFFFFFFFF7C7C7C7C7C23
:10EE20007C7CFCFCFCFCFCF8F00000FFFFFFFFFF1B
:10EE30000000E3C1881C3E7FFFFFFFC1803C3E3ED7
:10EE40003E3E3E9C0001FFFFFFFFFF00003F3F3FB3
:10EE50003F3F3C3C3F3F3F3F3E3C3C3F3F3F3733E3
:10EE600033333333333330383F3F3F3F3F000000CD
:10EE70000000000000000000000000000000000092
:10EE80000000000000000000000000000000000082
:10EE90000000000000000000000000000000000072
:10EEA0000000000000000000000000000000000062
:10EEB0000000000000000000000000000000000052
:10EEC0000000000000000000000000000000000042
:10EED0000000FCFA06060606060606669696162644
:10EEE000060686F68606060686464686C60606C6D2
:10EEF00006864646060686F68606060606060606C2
:10EF000006FAFC003F5F6060606060606064686992
:10EF100069666060606768686060676868646F60A1
:10EF2000606F6160606060606067686860606060BA
:10EF30006060605F3F00FCFA06E6C686060606666D
:10EF400096961626060686F68606060686464686A1
:10EF5000C60606C606864646060686F686060606E1
:10EF60000686C6E606FAFCFE3F5FE0EFE7E3E1E077
:10EF7000E0E4E8E9E9E6E0E0E0E7E8E8E0E0E7E847
:10EF8000E8E4EFE0E0EFE1E0E0E0E0E0E0E7E8E83F
:10EF9000E0E0E1E3E7EFE0DFBF7FFF0305F9F9F928
:10EFA000F9F9F9996969E9D9F9F9790979F9F9F971
:10EFB00079B9B97939F9F939F979B9B9F9F9790931
:10EFC00079F9F9F9F9F9F9F9F90503FFFFC0A09FFB
:10EFD0009F9F9F9F9F9B979696999F9F9F9897977C
:10EFE0009F9F9897979B909F9F909E9F9F9F9F9F6B
:10EFF0009F9897979F9F9F9F9F9F9FA0C0FFFCFAFE
:10F0000006060606060606060606669696162606F0
:10F010000686F686060606068686860606068606A0
:10F0200086860606060606060606060606FAFC009C
:10F030003F5F6060606060606060606064686969D4
:10F04000666060606768686060676868686760607D
:10F050007F65646463606060606060606060605F82
:10F060003F00FCFA06E6C686060606060606669613
:10F07000961626060686F686060606068686860600
:10F080000606860686860606060606060686C6E680
:10F0900006FAFCFE3F5FE0EFE7E3E1E0E0E0E0E0FE
:10F0A000E4E8E9E9E6E0E0E0E7E8E8E0E0E7E8E80E
:10F0B000E8E7E0E0FFE5E4E4E3E0E0E0E0E0E1E30E
:10F0C000E7EFE0DFBF7FFF0305F9F9F9F9F9F9F997
:10F0D000F9F9996969E9D9F9F9790979F9F9F9F940
:10F0E000797979F9F9F979F97979F9F9F9F9F9F990
:10F0F000F9F9F9F9F90503FFFFC0A09F9F9F9F9FB2
:10F100009F9F9F9F9B979696999F9F9F9897979F4A
:10F110009F98979797989F9F809A9B9B9C9F9F9F54
:10F120009F9F9F9F9F9F9FA0C0FFF0F8FC1E0E0E09
:10F130001EFCF8F0FFFFFF00000000FFFFFF070FBD
:10F140001F3C38383C1F0F0780C0E0F0783C1EFEA3
:10F15000FEFE03030100000000FFFFFF00000000AF
:10F160000000003F3F3FF8FCFE1E0E0E9EFEFCF826
:10F17000000080E0F8FE3F0F03003C3E3F3F3B387D
:10F18000383838381C1E1E0E0E0E1EFEFCF800000D
:10F19000001C1C1C3EFFF7E31C3C3C3838383C3F4D
:10F1A0001F0FFEFEFE00000000FEFEFE070F1F1CEC
:10F1B0001C1C1CFFFFFF000000000000003F3F3F41
:10F1C000FEFEFE0E0E0E0E0E0E0E0F0F0F0E0E0E8C
:10F1D0001EFEFCF83838383838383C3F1F0FFCFE2C
:10F1E000FE0E0E0E0E1E1E1CFFFFFF1C1C1C1CFC28
:10F1F000FCF81F3F3F383838383F3F1F0E0E0E0EC9
:10F200000E0E0EFEFEFC000000C0F0FC3F0F0301DE
:10F2100000003F3F3F0000000000F8FCFE1E0E0E05
:10F220001EFEFCF8E3F7FF3E1C1C3EFFF7E30F1F3A
:10F230003F3C38383C3F1F0FFCFEFE0E0E0E0EFE0C
:10F24000FEFC0F1F1F1C1C1C1CFFFFFF183838384A
:10F250003838383F3F1FF8FCFE1E0E0E1EFEFCF82D
:10F26000FFFFFF80000080FFFFFF01030707070784
:10F270000707030180C0E0F0783C1EFEFEFE03039A
:10F280000100000000FFFFFF000000000000000779
:10F290000707F8FCFE1E0E0E1EFEFCF8C0E0F0781C
:10F2A0003C1E0F07030107070707070707070707A4
:10F2B0001C1E1E0E0E0E1EFEFEFC8080800006062A
:10F2C0008FFFFFF903070707070707070703FEFE7E
:10F2D000FE00000000FEFEFE03070F0E0E0E0EFFE6
:10F2E000FFFF00000000000000070707FEFEFE0E03
:10F2F0000E0E0E0E0E0E07070707070707FFFFFE8D
:10F3000007070707070707070703FCFEFE0E0E0E99
:10F310000E1E1E1CFFFFFF07070707FFFFFE030768
:10F3200007070707070707030E0E0E0E0E0ECEFE89
:10F33000FE3C0000C0F0FC3F0F0300000000070788
:10F34000070000000000F8FCFE1E0E0E1EFEFCF87A
:10F35000F9FFFF8F06068FFFFFF901030707070775
:10F3600007070301FCFEFE0E0E0E0EFEFEFC030759
:10F370000707070707FFFFFF030707070707070739
:10F380000703000000000000000000000000000073
:10F39000000000000000000000000000000000006D
:10F3A00000808080808080808080808080808080DD
:10F3B000808080808080808080808080808080804D
:10F3C000808080808080808080808080808080803D
:10F3D000808080FF808080808482BE80808080FFEB
:10F3E00080808080B2AAAAA4808080FF80808080F4
:10F3F000A2A2AA94808080FF80808080868888BEB8
:10F40000808080FF80FF808080AEAAAA928080806A
:10F4100080FF808080BCAAAABA80808080FF808024
:10F420008082B28A8680808080FF808080BEAAAA87
:10F43000BE80808080FF80FF808080AEAAAA9E80F0
:10F44000808080FF808084BE809CA2A29C8080FF00
:10F4500080808084BE8084BE808080FF808084BE67
:10F4600080A4B2AAA48080FF80FF808084BE80A296
:10F47000A2AA948080FF808084BE80868888BE8017
:10F4800080FF808084BE80AEAAAA928080FF8080A8
:10F4900084BE80BCAAAABA8080FF80FF808084BE20
:10F4A0008082B28A868080FF808084BE80BEAAAAC5
:10F4B000BE8080FF808084BE80AEAAAA9E8080FF2E
:10F4C00080A2B2AAA4809CA2A29C80FF80FF80B2EE
:10F4D000AAAAA480808482BE80FF80B2AAAAA48047
:10F4E000B2AAAAA480FF80B2AAAAA480A2A2AA94C7
:10F4F00080FF80B2AAAAA480868888BE80FF80FF91
:10F5000080B2AAAAA480AEAAAA9280FF80B2AAAAB8
:10F51000A480BCAAAABA80FF80B2AAAAA48082B2A0
:10F520008A8680FF80B2AAAAA480BEAAAABE80FF53
:10F5300080FF80B2AAAAA480AEAAAA9E80FF80A261
:10F54000A2AA94809CA2A29C80FF80A2A2AA9480DE
:10F550008084BE8080FF80A2A2AA9480B2AAAAA4BE
:10F5600080FF80FF80A2A2AA9480A2A2AA9480FF1A
:10F5700080A2A2AA9480868888BE80FF80A2A2AAC8
:10F580009480AEAAAA9280FF80A2A2AA9480BCAA6C
:10F59000AABA80FF80000000000000002F000000D9
:10F5A00003000300543F147E152E2A7F2A3A2215A9
:10F5B0002A5422122D2911280003000000001C22C9
:10F5C00041000041221C00000C0C000008083E080D
:10F5D000080040300000080808080800400000004B
:10F5E00040300806013E4749713E0402017F006237
:10F5F000514946002241493E000708087F004F4913
:10F600004931003C4A493000016119070036494937
:10F6100036002649497E00000012000000403400F8
:10F620000008142241001414141414004122140878
:10F6300002290502000E152B2D123E0909093E3F35
:10F640002525251A1E212121123F2121211E3F257A
:10F650002525213F090909011E2121293A3F0404DA
:10F66000043F3F00000000214141413F3F0C122177
:10F67000003F202020003F060C063F3F030E183FAE
:10F680001E2121211E3F090909061E2129112E3F95
:10F6900009091926122529120001013F01011F2025
:10F6A00020203F030C300C031F301C301F22140895
:10F6B000142203043804033129252321007F41410A
:10F6C0000001060830400041417F000402010204AD
:10F6D00040404040400001020000102A2A2A3C3FDE
:10F6E000242424181C22222222182424243F1C2AE9
:10F6F0002A2A2C087E0901004C5252523C3F040435
:10F7000004383D000000002040403D003F08142226
:10F71000001F202020003C023C023C3E0402023C30
:10F720001C2222221C7E1212120C0C1212127E3E7D
:10F730000404020214262A3214041F2424001E206A
:10F7400020203E06182018061E201C201E241818F3
:10F7500024004E5050503E22322A26220836414183
:10F760000000007F000041413E0800180408100C12
:10F770000000000000000000000000000000000089
:10F78000000000000000000000000000000000C0B9
:10F790002010D012151D111D1512101020C0FF8051
:10F7A000809F848A918086A9A9BE8080FFC0201096
:10F7B000D012151D111D1512101020C0FFF0F0EF12
:10F7C000F4FAE1F0F6D9D9CEF0F0FFC02010D01253
:10F7D000151D111D1512101020C0FFFEFEE1FAF4D8
:10F7E000EFFEF8D7D7C0FEFEFFC0E0D010D2D5DDC7
:10F7F000D1DDD5D2D0D0E0C0FFFFFFE0FBF5EEFFBA
:10F80000F9D6D6C1FFFFFFC0E0F030F2F7FFFFFFEF
:10F81000F7F2F0F0E0C0FFFFFFE0FBF5EEFFF9D6F6
:10F82000D6C1FFFFFF0F3FFFFCF0C00000C0F0FC9F
:10F83000FF3F0F00000000030F3F7E7E3F0F0300DD
:10F840000000005500810081008100412214000069
:10F8500000006A00000000000001020468000000CF
:10F860000003165040000000000000405016030046
:10F87000000000010514404014050100000000FFD5
:10F88000FFFFC7C7C7C7C7EFFFFE7C0000007F7F31
:10F890007F01010103071F7F7C780000000080408A
:10F8A0004020202040408000000000000E31404EEB
:10F8B0009191914040310E000000008060100808D6
:10F8C000E42424C408081060800007182040409FEA
:10F8D00083859840402018070000000000000000C9
:10F8E0000000000000000000000000000000000018
:10F8F0000000000000000000000000000000000008
:10F9000000000000000000000000000000000000F7
:10F9100000000000000000000000000000000000E7
:10F9200000000000000000000000000000000000D7
:10F9300000000000000000000000000000000000C7
:10F9400000000000000000000000000000000000B7
:10F9500000000000000000000000000000000000A7
:10F960000000000000000000000000000000000097
:10F970000000000000000000000000000000000087
:10F9800000000000000000FE02FA0A0A0A0A0A0A41
:10F990000A0A0A0A0A0A0A0A0A0A0A0A0A0A0A0AC7
:10F9A0000A0A0A0A0A0A0A0A0A0A0A0A0A0A0A0AB7
:10F9B0000A0A8A8A8A8A8A8A8A8A8A8A8A8ACACA27
:10F9C000CACACACACACACACACAEAEAEAEAEAEAEAB7
:10F9D000EAEAEAEAEAFAFAFAFAFAFAFA02FE7F4000
:10F9E0005F5858585858585C5C5C5C5C5C5C5C5C6C
:10F9F0005C5C5C5E5E5E5E5E5E5E5E5E5E5E5F5F2B
:10FA00005F5F5F5F5F5F5F5F5F5F5F5F5F5F5F5F06
:10FA10005F5F5F5F5F5F5F5F5F5F5F5F5F5F5F5FF6
:10FA20005F5F5F5F5F5F5F5F5F5F5F5F5F5F5F5FE6
:10FA30005F5F5F407F80808080808080808080806A
:10FA40008C8C8C9EBFBFBFBF929292848289859519
:10FA5000B595858982848080888494B494848880D4
:10FA6000808080808090B090808080808080808046
:10FA700080A080808080809F909F80969589809FC5
:10FA8000958A8080BFA1A1A1A1A18780808080BF2D
:10FA9000A1A1A181819F80808080BFA1818181A15E
:10FAA000BF808080809F8181A1A1A1BF8080808054
:10FAB00087A1A1A1A1A1BF80808080B1A1A1A1A1A6
:10FAC000A1BF80808080BCA0A1A1A1A1BF808080B7
:10FAD00080BFA0A0A0A1A1BF80808080BFA1A1A065
:10FAE000A0A0BF80808080BFA1A1A1A1A0BC808078
:10FAF0008080BFA1A1A1A1A1B18080808C92A1A191
:10FB0000A181828C8080808C92A18181A1928C8045
:10FB100080808C8281A1A1A1928C8080808092A122
:10FB2000A1A1A1928C8080808C90A0A1A1A1928C97
:10FB30008080808C92A1A0A0A1928C8080808C92E9
:10FB4000A1A1A1A0908C8080808C92A1A1A1A19262
:10FB5000808080BE8989BE80B8A8BF80B888406098
:10FB600070787C7E7C7870604002060E1E3E7E3E81
:10FB70001E0E0602000000000000000000000080D1
:10FB80008080808080808080808080808080808075
:10FB9000808080809E9EBFBFAFB7BBBDAFB7BBBDEF
:10FBA000AFB7BBBDAFB7BBBDBF9E92A1A1A1B1B95D
:10FBB000BDAFB7BBBDAFB7BBBDAFB7BBBDBF9E92FF
:10FBC000A1A1A1A1A1A1A1B1B9BDAFB7BBBDAFB763
:10FBD000BBBDBF9E92A1A1A1A1A1A1A1A1A1A1A1D3
:10FBE000B1B9BDAFB7BBBDBF9E92A1A1A1A1A1A15B
:10FBF000A1A1A1A1A1A1A1A1A1B1B9BDBF9E92A1A5
:10FC0000A1A1A1A1A1A1A1A1A1A1A1A1A1A1A1A1E4
:10FC1000A1BF9E92A1A1B1A9A5A3B1A9A5A3B1A974
:10FC2000A5A3B1A9A5A3BFFCFE9393FEFC8098BC3D
:10FC3000E6E6BCFFFF8080FEFE988C8698BEB7B3D8
:10FC4000B3B383B0BCBFB7B3BB9F86B0BBBBBFB7BA
:10FC5000870000000000000000000000000000001D
:10FC60000000000000000000000000000000000094
:10FC70000000000000000000000000000000000084
:10FC80000000000000000000000000000000000074
:10FC90000000000000000000000000000000000064
:10FCA0000000000000000000000000000000000054
:10FCB0000000000000000000000000000000007EC6
:10FCC000FFC3FF7E000607FFFFE7F3FBDFCEC3DBCA
:10FCD000DBFF7E0F1F18FFFFDFDFDBFB737EFFDB29
:10FCE000FB7103F3FB1F0F66FFDBFF660EDFDBFF1D
:10FCF000FE00000000000000000000000000000006
:10FD00000000000406FF060400E3F3FBDFCFC70496
:10FD100006FF060400FFFF1818FFFF0406FF060495
:10FD2000000303FFFF030300000000000000111B9D
:10FD30001511110A04111B1F1F1F0E0446756E6B4F
:10FD40002D5369676E616C3A0050726F66692F457A
:10FD5000636F2F4E5A004465636F64657235362FAA
:10FD600035370048656C6C69676B6569743A0041AA
:10FD70006B6B756C6164756E673A00525353492D15
:10FD80004261636B3A0048616E647265676C6572CC
:10FD9000005A7765697465204C6F6B004C6F6B611E
:10FDA0006472657373650046756E6B74696F6E651A
:10FDB0006E00FEFF01FFFE7FFF80FF7F536F6674C2
:10FDC000776172653A004164722D46756E6B3A0038
:10FDD00056657262696E64656E004C6F6B2D53756B
:10FDE000636865002D2D2D2D2D2D2D2D004B6F6E53
:10FDF00074726173740056657273696F6E0050722D
:10FE00006F6772616D004C6F6B7761686C00537443
:10FE10006174757300526573657400536574757011
:10FE200000413A00200020002000200020005665FC
:10FE30007262696E64756E67206D69742043445AFE
:10FE4000002020206E657520617566626175656EA3
:10FE50002E00204C6173742065696E7374656C6C40
:10FE6000656E00447265686B6E6F706620647275B3
:10FE7000652D0064757263687A756675656872656C
:10FE80006E2E004C6F6B61647265737365205072E7
:10FE90006F67004465636F6465722050726F6772AC
:10FEA000616D00636B656E2C20756D2065696E65F4
:10FEB0006E0048616E647265676C65722D5479706E
:10FEC0000049324320616B7475656C6C3A200050B8
:10FED000726F6772616D6D696572656E00202020BA
:10FEE000202020202020202020004932432D416462
:10FEF00072657373653A0041647265737365206E51
:10FF000065753A004C6F6B616472657373653A0096
:10FF100048617570746D656E7565005A77656974B2
:10FF200065204C6F6B004C6F6B7765636873656C15
:10FF3000004C6F6B2073756368656E0046756E6B61
:10FF400074696F6E656E004932432D537461747528
:10FF500073004272656D73652020200056657262E1
:10FF6000696E64656E0052616E67696572656E00E8
:10FF700073706569636865726E004175746F666160
:10FF80006872740043445A2D49443A20005A656E01
:10FF90007472616C65004B6F6E74726173740042B1
:10FFA0006567696E6E3A004C6F6B7761686C002014
:10FFB0004F4B2020004164723A2000585858582076
:10FFC00000456E64653A00436F64653A0057657298
:10FFD000743A00524553455400536574757000459A
:10FFE00072726F72005265736574004164723A00F8
:10FFF0003F3F3F003200370048005200580000FFEA
:020000040001F9
:100000000401116F0A0E04011119D8A415D20001C0
:10001000A105D8A4A3D0000EA16F070ED66FF6C01D
:10002000D7F0010E88EC14F0B50ED66FFF0ED76F27
:10003000060ED86F000ED96F010EDA6F000EDB6F5F
:10004000000EDC6F000EDD6F000EDE6F000EDF6F46
:1000500061EC06F0010E0101596F00019C05D8A466
:1000600004D0010E0101576F70D0480EC26FE50E2B
:10007000C36F070EC46F020EC56F000EC66F000E71
:10008000C76F050EC86F000EC96F000ECA6F000E55
:10009000CB6F000ECC6F000ECD6FF6C0CEF0BAEC79
:1000A00000F0480EC26FE50EC36F070EC46F020E5C
:1000B000C56F000EC66F090EC76F050EC86F000E24
:1000C000C96F000ECA6F000ECB6F000ECC6F000E12
:1000D000CD6FF6C0CEF0BAEC00F0480EC26FE50E60
:1000E000C36F070EC46F020EC56F000EC66F120EEF
:1000F000C76F050EC86F000EC96F000ECA6F000EE5
:10010000CB6F000ECC6F000ECD6FF6C0CEF0BAEC08
:1001100000F0480EC26FE50EC36F070EC46F020EEB
:10012000C56F000EC66F1A0EC76F050EC86F000EA2
:10013000C96F000ECA6F000ECB6F000ECC6F000EA1
:10014000CD6FF6C0CEF0BAEC00F0010E01015F6F8A
:10015000010E5C6F010E5B6F47ECF2F00101790557
:10016000D8A431D0010EC66F295104E1320E285DAA
:10017000D8A013D04304D8A410D0000E436E000EB4
:10018000296F000E286F010E596F00019C05D8A43D
:1001900021D0010E0101576F1DD0295104E11E0E1F
:1001A000285DD8A017D04350D8A414D0010E436EB8
:1001B000000E296F000E286F010E596F00019C057B
:1001C000D8B4E7D707D0000E296F000E286F000EB5
:1001D000C66FF2D701017805D8A41DD0010EC56FF6
:1001E000275104E1460E265DD8A005D07705D8A496
:1001F00002D0000E0AD0275104E1140E265DD8A0CB
:1002000012D07751D8A40FD0010E776F000E276F50
:10021000000E266F06D0000E276F000E266F000E10
:10022000C56F010E5F6F00018951D8B404D0010180
:100230004C05D8A463D000018851D8B404D0010182
:100240004705D8A45BD000018751D8B404D0010180
:100250004505D8A453D001015905D8A41ED00001EA
:100260009C05D8A407D078C0D6F079C0D7F016EC9A
:10027000C8F006D078C0D6F079C0D7F001ECD4F041
:1002800078C07AF079C07BF07AC0BCF07BC0BDF05A
:10029000CCEC07F0000E0101596F5705D8A40DD022
:1002A00070C0D6F071C0D7F016ECC8F070C072F014
:1002B00071C073F0000E0101576F5F05D8A409D01B
:1002C0000001915114ECFBF091C03DF0000E0101D2
:1002D0005F6F5C05D8A406D05D5108EC0EF0000EEF
:1002E00001015C6F5B05D8A409D000018F51CCECF3
:1002F0000EF08FC090F0000E01015B6F4D05D8A489
:100300002BD04E5100018919D8B423D001014E05DC
:10031000D8A410D0000E0001D76F000ED66F100EBB
:10032000D86F020ED96F080E22ECD1F0010E010138
:10033000C76F08D0010E0001A16F000E0101C76F49
:10034000000E4C6F000E02016A6F000E696F4EC105
:1003500089F0000E01014D6F4605D8A428D03B500E
:1003600000018719D8B420D03B04D8A40FD0000EC8
:10037000D76F000ED66F100ED86F020ED96F070E12
:1003800022ECD1F0010E0101C76F07D0010EA16F61
:10039000000E0101C76F000E456F000E02016A6F6B
:1003A000000E696F3BC087F0000E0101466F4805E3
:1003B000D8A42BD0495100018819D8B423D0010109
:1003C0004905D8A410D0000E0001D76F000ED66FDB
:1003D000100ED86F020ED96F090E22ECD1F0010E6B
:1003E0000101C76F08D0010E0001A16F000E0101CD
:1003F000C76F000E476F000E02016A6F000E696F33
:1004000049C188F0000E0101486F4205D8A41200CE
:1004100043514419D8B40DD04305D8A402D0010EDD
:1004200005D0010E0001A16F000E0101416F43C113
:1004300044F1000E426F12000B0E1119D8A42BD0FC
:100440000001A105D8A413D0070ED66FF6C0D7F0CF
:10045000010E88EC14F0520EEA6FFE0EEB6F110ED7
:10046000EC6F0CEC0FF0000EA16F010EA06F0101FC
:100470005B05D8B404D00001A005D8A41200000187
:100480008F518BEC0EF08FC090F0000EA06F000E1D
:1004900001015B6F12000C0E1119D8A4EBD1100EE4
:1004A0000F6F030E106F6C0E006F6C0E016F6C0EF1
:1004B000026F6C0E036F0001A105D8A4CED0060E0A
:1004C000C26FAF0EC36F440EC46F050EC56F000E32
:1004D000C66F0FC4C7F010C4C8F0000EC96F000E7D
:1004E000CA6F010ECB6F000ECC6F000ECD6FF6C041
:1004F000CEF0BAEC00F0060EC26FAF0EC36F440E22
:10050000C46F050EC56F0E0EC66F0FC4C7F010C4C2
:10051000C8F0000EC96F000ECA6F010ECB6F000E3F
:10052000CC6F000ECD6FF6C0CEF0BAEC00F0480EE6
:10053000C26FE50EC36F070EC46F020EC56F6C0E5F
:10054000C66F04010F510C0F0001C76F0401105159
:10055000030F0001C86F000EC96F000ECA6F010EB5
:10056000CB6F000ECC6F000ECD6FF6C0CEF0BAECA4
:1005700000F0480EC26FE50EC36F070EC46F020E87
:10058000C56F6C0EC66F04010F51150F0001C76FC8
:1005900004011051030F0001C86F000EC96F000E57
:1005A000CA6F010ECB6F000ECC6F000ECD6FF6C080
:1005B000CEF0BAEC00F0480EC26FE50EC36F070E26
:1005C000C46F020EC56F6C0EC66F04010F511E0F73
:1005D0000001C76F04011051030F0001C86F000E26
:1005E000C96F000ECA6F010ECB6F000ECC6F000EEC
:1005F000CD6FF6C0CEF0BAEC00F0480EC26FE50E3B
:10060000C36F070EC46F020EC56F6C0EC66F040178
:100610000F51270F0001C76F04011051030F000194
:10062000C86F000EC96F000ECA6F010ECB6F000EAF
:10063000CC6F000ECD6FF6C0CEF0BAEC00F0260EF7
:10064000EA6FFF0EEB6F0B0EEC6F0CEC0FF0000E71
:10065000A16F010EA06F010E9A6F01015905D8B468
:1006600004D00001A005D8A4FAD0E80E0001785DFE
:10067000030E7959D8A018D0270EBF6F100EBE6F89
:1006800078C0BCF079C0BDF05DEC15F0BCC0C2F024
:10069000BDC0C3F0030EC56FE80EC46F0EEC14F0BE
:1006A000C251600F0401006F0001795104E1640E32
:1006B000785DD8A018D0030EBF6FE80EBE6F78C06B
:1006C000BCF079C0BDF05DEC15F0BCC0C2F0BDC09F
:1006D000C3F0000EC56F640EC46F0EEC14F0C2516F
:1006E000600F0401016F0001795104E10A0E785D89
:1006F000D8A018D0000EBF6F640EBE6F78C0BCF0DB
:1007000079C0BDF05DEC15F0BCC0C2F0BDC0C3F057
:10071000000EC56F0A0EC46F0EEC14F0C251600FCC
:100720000401026F78C0BCF079C0BDF0000E00017A
:10073000BF6F0A0EBE6F5DEC15F0BC51600F040177
:10074000036F480E0001C26FE50EC36F070EC46F42
:10075000020EC56F00C4C6F004010F510C0F00015A
:10076000C76F04011051030F0001C86F000EC96F5D
:10077000000ECA6F010ECB6F000ECC6F000ECD6F56
:10078000F6C0CEF0BAEC00F0480EC26FE50EC36FB3
:10079000070EC46F020EC56F01C4C6F004010F51ED
:1007A000150F0001C76F04011051030F0001C86F3E
:1007B000000EC96F000ECA6F010ECB6F000ECC6F1A
:1007C000000ECD6FF6C0CEF0BAEC00F0480EC26F4E
:1007D000E50EC36F070EC46F020EC56F02C4C6F0EC
:1007E00004010F511E0F0001C76F04011051030FC8
:1007F0000001C86F000EC96F000ECA6F010ECB6FEB
:10080000000ECC6F000ECD6FF6C0CEF0BAEC00F04B
:10081000480EC26FE50EC36F070EC46F020EC56FA0
:1008200003C4C6F004010F51270F0001C76F040174
:100830001051030F0001C86F000EC96F000ECA6F80
:10084000010ECB6F000ECC6F000ECD6FF6C0CEF058
:10085000BAEC00F0000EA06F000E0101596F410EBE
:100860000001BC6F140EBD6F9A5182EC0DF00101B6
:10087000596F1200640E1119D8A499D30001A10573
:10088000D8A415D0070ED66FF6C0D7F0010E88ECAD
:1008900014F0100EEA6FFF0EEB6F0B0EEC6F0CEC0A
:1008A0000FF0000EA16F010EA06F010E966F98055C
:1008B000D8B466D3A005D8A4120062D3060EE96F9F
:1008C000FE0EEA6F080EEB6FA7C0ECF0020E5CECB8
:1008D000F3F0510EC26FFC0EC36F5A0EC46F010EBF
:1008E000C56F000EC66F000EC76F040EC86F000EF6
:1008F000C96F000ECA6F000ECB6F000ECC6F000EDA
:10090000CD6FF6C0CEF0BAEC00F0FE0ED66FFD0E45
:10091000D76F080ED86F030ED96F040EDA6F000E72
:10092000DB6F000EDC6F000EDD6F000EDE6F010E60
:10093000DF6FB5ECE6F0510EC26FFC0EC36F660EB2
:10094000C46F010EC56F000EC66F000EC76F050E97
:10095000C86F000EC96F000ECA6F000ECB6F000E7D
:10096000CC6F000ECD6FF6C0CEF0BAEC00F0A70E43
:10097000D66FFD0ED76F0B0ED86F030ED96F050E15
:10098000DA6F000EDB6F000EDC6F000EDD6F000E05
:10099000DE6F010EDF6FB5ECE6F0510EC26FFC0E9C
:1009A000C36F660EC46F010EC56F000EC66F000EDA
:1009B000C76F060EC86F000EC96F000ECA6F000E1B
:1009C000CB6F000ECC6F000ECD6FF6C0CEF0BAEC40
:1009D00000F01B0ED66FFE0ED76F060ED86F030EFB
:1009E000D96F060EDA6F000EDB6F000EDC6F000EA3
:1009F000DD6F000EDE6F010EDF6FB5ECE6F0510E1D
:100A0000C26FFC0EC36F660EC46F010EC56F000E81
:100A1000C66F000EC76F070EC86F000EC96F000EBD
:100A2000CA6F000ECB6F000ECC6F000ECD6FF6C0FC
:100A3000CEF0BAEC00F00E0ED66FFE0ED76F070E9A
:100A4000D86F030ED96F070EDA6F000EDB6F000E42
:100A5000DC6F000EDD6F000EDE6F010EDF6FB5EC98
:100A6000E6F09ED2FE0EE96FFD0EEA6F080EEB6F08
:100A7000A7C0ECF0030E5CECF3F0510EC26FFC0E5D
:100A8000C36F5A0EC46F010EC56F000EC66F000E05
:100A9000C76F020EC86F000EC96F000ECA6F000E3E
:100AA000CB6F000ECC6F000ECD6FF6C0CEF0BAEC5F
:100AB00000F0060ED66FFE0ED76F080ED86F030E2D
:100AC000D96F020EDA6F000EDB6F000EDC6F000EC6
:100AD000DD6F000EDE6F010EDF6FB5ECE6F0510E3C
:100AE000C26FFC0EC36F5A0EC46F010EC56F000EAD
:100AF000C66F000EC76F050EC86F000EC96F000EDF
:100B0000CA6F000ECB6F000ECC6F000ECD6FF6C01B
:100B1000CEF0BAEC00F0A70ED66FFD0ED76F0B0E1D
:100B2000D86F030ED96F050EDA6F000EDB6F000E63
:100B3000DC6F000EDD6F000EDE6F010EDF6FB5ECB7
:100B4000E6F02BD7A70EE96FFD0EEA6F0B0EEB6FE9
:100B5000A7C0ECF0040E5CECF3F0510EC26FFC0E7B
:100B6000C36F5A0EC46F010EC56F000EC66F000E24
:100B7000C76F020EC86F000EC96F000ECA6F000E5D
:100B8000CB6F000ECC6F000ECD6FF6C0CEF0BAEC7E
:100B900000F0060ED66FFE0ED76F080ED86F030E4C
:100BA000D96F020EDA6F000EDB6F000EDC6F000EE5
:100BB000DD6F000EDE6F010EDF6FB5ECE6F0510E5B
:100BC000C26FFC0EC36F5A0EC46F010EC56F000ECC
:100BD000C66F000EC76F030EC86F000EC96F000E00
:100BE000CA6F000ECB6F000ECC6F000ECD6FF6C03B
:100BF000CEF0BAEC00F0FE0ED66FFD0ED76F080EE9
:100C0000D86F030ED96F030EDA6F000EDB6F000E84
:100C1000DC6F000EDD6F000EDE6F010EDF6FB5ECD6
:100C2000E6F0510EC26FFC0EC36F5A0EC46F010E78
:100C3000C56F000EC66F000EC76F060EC86F000EA0
:100C4000C96F000ECA6F000ECB6F000ECC6F000E86
:100C5000CD6FF6C0CEF0BAEC00F0BBD61B0EE96F3C
:100C6000FE0EEA6F060EEB6FA7C0ECF0050E5CEC13
:100C7000F3F0510EC26FFC0EC36F5A0EC46F010E1B
:100C8000C56F000EC66F000EC76F020EC86F000E54
:100C9000C96F000ECA6F000ECB6F000ECC6F000E36
:100CA000CD6FF6C0CEF0BAEC00F0060ED66FFE0E99
:100CB000D76F080ED86F030ED96F020EDA6F000ED1
:100CC000DB6F000EDC6F000EDD6F000EDE6F010EBD
:100CD000DF6FB5ECE6F0510EC26FFC0EC36F5A0E1B
:100CE000C46F010EC56F000EC66F000EC76F030EF6
:100CF000C86F000EC96F000ECA6F000ECB6F000EDA
:100D0000CC6F000ECD6FF6C0CEF0BAEC00F0FE0E48
:100D1000D66FFD0ED76F080ED86F030ED96F030E76
:100D2000DA6F000EDB6F000EDC6F000EDD6F000E61
:100D3000DE6F010EDF6FB5ECE6F0510EC26FFC0EF8
:100D4000C36F5A0EC46F010EC56F000EC66F000E42
:100D5000C76F040EC86F000EC96F000ECA6F000E79
:100D6000CB6F000ECC6F000ECD6FF6C0CEF0BAEC9C
:100D700000F0A70ED66FFD0ED76F0B0ED86F030EC7
:100D8000D96F040EDA6F000EDB6F000EDC6F000E01
:100D9000DD6F000EDE6F010EDF6FB5ECE6F0510E79
:100DA000C26FFC0EC36F5A0EC46F010EC56F000EEA
:100DB000C66F000EC76F070EC86F000EC96F000E1A
:100DC000CA6F000ECB6F000ECC6F000ECD6FF6C059
:100DD000CEF0BAEC00F02FD60E0EE96FFE0EEA6FE1
:100DE000070EEB6FA7C0ECF0060E5CECF3F0510EB3
:100DF000C26FFC0EC36F5A0EC46F010EC56F000E9A
:100E0000C66F000EC76F020EC86F000EC96F000ECE
:100E1000CA6F000ECB6F000ECC6F000ECD6FF6C008
:100E2000CEF0BAEC00F0060ED66FFE0ED76F080EAD
:100E3000D86F030ED96F020EDA6F000EDB6F000E53
:100E4000DC6F000EDD6F000EDE6F010EDF6FB5ECA4
:100E5000E6F0510EC26FFC0EC36F5A0EC46F010E46
:100E6000C56F000EC66F000EC76F030EC86F000E71
:100E7000C96F000ECA6F000ECB6F000ECC6F000E54
:100E8000CD6FF6C0CEF0BAEC00F0FE0ED66FFD0EC0
:100E9000D76F080ED86F030ED96F030EDA6F000EEE
:100EA000DB6F000EDC6F000EDD6F000EDE6F010EDB
:100EB000DF6FB5ECE6F0510EC26FFC0EC36F5A0E39
:100EC000C46F010EC56F000EC66F000EC76F040E13
:100ED000C86F000EC96F000ECA6F000ECB6F000EF8
:100EE000CC6F000ECD6FF6C0CEF0BAEC00F0A70EBE
:100EF000D66FFD0ED76F0B0ED86F030ED96F040E91
:100F0000DA6F000EDB6F000EDC6F000EDD6F000E7F
:100F1000DE6F010EDF6FB5ECE6F0510EC26FFC0E16
:100F2000C36F5A0EC46F010EC56F000EC66F000E60
:100F3000C76F050EC86F000EC96F000ECA6F000E96
:100F4000CB6F000ECC6F000ECD6FF6C0CEF0BAECBA
:100F500000F01B0ED66FFE0ED76F060ED86F030E75
:100F6000D96F050EDA6F000EDB6F000EDC6F000E1E
:100F7000DD6F000EDE6F010EDF6FB5ECE6F010D016
:100F80009651010AD8B49AD4030AD8B46BD5010A91
:100F9000D8B4D8D5070AD8B461D6010AD8B41CD7BA
:100FA00096C097F0000E986F000EA06F1200650EAD
:100FB0001119D8A470D00001A105D8A447D0070EFC
:100FC000D66FF6C0D7F0010E88EC14F0A70EEA6FCA
:100FD000FF0EEB6F080EEC6F0CEC0FF0040ED66FEB
:100FE000FF0ED76F0C0ED86F000ED96F020EDA6F9E
:100FF000000EDB6F000EDC6F000EDD6F000EDE6F8B
:10100000000EDF6F61EC06F0B205D8A406D05A0ED0
:10101000D66F480EB0ECFCF013D0020EB219D8A473
:1010200006D05A0ED66F200EB0ECFCF009D0030E9D
:10103000B219D8A405D05A0ED66F200EB0ECFCF031
:10104000000EA16F010EA06F010E9A6F01015905EC
:10105000D8B404D00001A005D8A412D078C0D6F02E
:1010600079C0D7F00A0E0001D86F040ED96FA7C05F
:10107000DAF02FECCBF0000EA06F000E0101596FDB
:10108000410E0001BC6F140EBD6F9A5182EC0DF041
:101090000101596F12006D0E1119D8A448D3000137
:1010A000A105D8A494D1070ED66FF6C0D7F0010ED3
:1010B00088EC14F04B0EEA6FFF0EEB6F070EEC6F2F
:1010C0000CEC0FF09251D8B459D06F0ED66FFD0EC4
:1010D000D76F0C0ED86F000ED96F020EDA6F000EAC
:1010E000DB6F000EDC6F000EDD6F000EDE6F010E99
:1010F000DF6FB5ECE6F03C0ED66FFD0ED76F0D0E30
:10110000D86F000ED96F030EDA6F000EDB6F000E82
:10111000DC6F000EDD6F000EDE6F010EDF6FB5ECD1
:10112000E6F0C60ED66FFD0ED76F0A0ED86F000E12
:10113000D96F040EDA6F000EDB6F000EDC6F000E4D
:10114000DD6F000EDE6F010EDF6FB5ECE6F07B0E9B
:10115000D66FFD0ED76F0B0ED86F000ED96F050E30
:10116000DA6F000EDB6F000EDC6F000EDD6F000E1D
:10117000DE6F010EDF6FB5ECE6F058D0840ED66F4F
:10118000FF0ED76F090ED86F000ED96F020EDA6FFF
:10119000000EDB6F000EDC6F000EDD6F000EDE6FE9
:1011A000010EDF6FB5ECE6F0C10ED66FFE0ED76F05
:1011B0000E0ED86F000ED96F030EDA6F000EDB6FC4
:1011C000000EDC6F000EDD6F000EDE6F010EDF6FB4
:1011D000B5ECE6F0EA0ED66FFE0ED76F0D0ED86FA7
:1011E000000ED96F040EDA6F000EDB6F000EDC6F9D
:1011F000000EDD6F000EDE6F010EDF6FB5ECE6F066
:10120000470ED66FFF0ED76F0B0ED86F000ED96F3B
:10121000050EDA6F000EDB6F000EDC6F000EDD6F67
:10122000000EDE6F010EDF6FB5ECE6F0630ED66FD9
:10123000FD0ED76F0C0ED86F000ED96F060EDA6F49
:10124000000EDB6F000EDC6F000EDD6F000EDE6F38
:10125000010EDF6FB5ECE6F0BC0ED66FFD0ED76F5A
:101260000A0ED86F000ED96F070EDA6F000EDB6F13
:10127000000EDC6F000EDD6F000EDE6F010EDF6F03
:10128000B5ECE6F0BC0ED66FFF0ED76F050ED86F2B
:101290004F0ED96F020EDA6F000EDB6F000EDC6F9F
:1012A000000EDD6F000EDE6F010EDF6FB5ECE6F0B5
:1012B000BC0ED66FFF0ED76F050ED86F4F0ED96FCD
:1012C000030EDA6F000EDB6F000EDC6F000EDD6FB9
:1012D000000EDE6F010EDF6FB5ECE6F0BC0ED66FD0
:1012E000FF0ED76F050ED86F4F0ED96F040EDA6F51
:1012F000000EDB6F000EDC6F000EDD6F000EDE6F88
:10130000010EDF6FB5ECE6F0BC0ED66FFF0ED76FA7
:10131000050ED86F4F0ED96F050EDA6F000EDB6F1A
:10132000000EDC6F000EDD6F000EDE6F010EDF6F52
:10133000B5ECE6F0BC0ED66FFF0ED76F050ED86F7A
:101340004F0ED96F060EDA6F000EDB6F000EDC6FEA
:10135000000EDD6F000EDE6F010EDF6FB5ECE6F004
:10136000210ED66FFE0ED76F030ED86F420ED96FC7
:10137000070EDA6F000EDB6F000EDC6F000EDD6F04
:10138000000EDE6F010EDF6FB5ECE6F0F80ED66FE3
:10139000020ED76F050ED86F4F0ED96F070EDA6F9A
:1013A000000EDB6F000EDC6F000EDD6F000EDE6FD7
:1013B000010EDF6FB5ECE6F0000EA16F010E01012A
:1013C0006A6F010EB56F010EB36F010EAE6F0001B3
:1013D0009251D8B4B3D001016205D8A42AD0E40E4A
:1013E0000001D66FFE0ED76F060ED86F430ED96F71
:1013F000020EDA6F000EDB6F000EDC6F000EDD6F89
:10140000000EDE6F000EDF6FB5ECE6F00CC1D6F01B
:101410000DC1D7F04F0ED86F020ED96F000EDA6FE4
:10142000000EDB6F000EDC6FC1ECD6F0000E010188
:10143000626F6705D8A429D0E40E0001D66FFE0EB6
:10144000D76F060ED86F430ED96F030EDA6F000EFA
:10145000DB6F000EDC6F000EDD6F000EDE6F000E26
:10146000DF6FB5ECE6F068C1D6F0D76B4F0ED86FE2
:10147000030ED96F000EDA6F000EDB6F000EDC6F0B
:10148000C1ECD6F0000E0101676FB505D8A429D0D4
:10149000E40E0001D66FFE0ED76F060ED86F430E16
:1014A000D96F040EDA6F000EDB6F000EDC6F000EDA
:1014B000DD6F000EDE6F000EDF6FB5ECE6F05BC097
:1014C000D6F0D76B4F0ED86F040ED96F000EDA6FBF
:1014D000000EDB6F000EDC6FC1ECD6F0000E0101D8
:1014E000B56FA305D8A4F5D0E40E0001D66FFE0EAB
:1014F000D76F060ED86F430ED96F050EDA6F000E48
:10150000DB6F000EDC6F000EDD6F000EDE6F000E75
:10151000DF6FB5ECE6F0A4C1D6F0D76B4F0ED86FF5
:10152000050ED96F000EDA6F000EDB6F000EDC6F58
:10153000C1ECD6F0000E0101A36FCBD001016A050A
:10154000D8A429D0E40E0001D66FFE0ED76F060E88
:10155000D86F430ED96F020EDA6F000EDB6F000EEC
:10156000DC6F000EDD6F000EDE6F000EDF6FB5EC7E
:10157000E6F03FC0D6F0D76B4F0ED86F020ED96F92
:10158000000EDA6F000EDB6F000EDC6FC1ECD6F0E0
:10159000000E01016A6FB305D8A44ED0E40E00011D
:1015A000D66FFE0ED76F060ED86F430ED96F030E9F
:1015B000DA6F000EDB6F000EDC6F000EDD6F000EC9
:1015C000DE6F000EDF6FB5ECE6F0B6C0D6F0D76B7D
:1015D0004F0ED86F030ED96F000EDA6F000EDB6F5F
:1015E000000EDC6FC1ECD6F0E40ED66FFE0ED76FA6
:1015F000060ED86F430ED96F040EDA6F000EDB6F44
:10160000000EDC6F000EDD6F000EDE6F000EDF6F70
:10161000B5ECE6F0B3C0D6F0D76B4F0ED86F040E22
:10162000D96F000EDA6F000EDB6F000EDC6FC1ECBD
:10163000D6F0000E0101B36FAE05D8A44AD0E40E77
:101640000001D66FFE0ED76F060ED86F430ED96F0E
:10165000050EDA6F000EDB6F000EDC6F000EDD6F23
:10166000000EDE6F000EDF6FB5ECE6F0B005D8A41B
:1016700017D0AF0ED66FFF0ED76F060ED86F4A0E7B
:10168000D96F050EDA6F000EDB6F000EDC6F000EF7
:10169000DD6F000EDE6F010EDF6FB5ECE6F016D0E9
:1016A000DF0ED66FFF0ED76F060ED86F490ED96FBB
:1016B000050EDA6F000EDB6F000EDC6F000EDD6FC3
:1016C000000EDE6F010EDF6FB5ECE6F0000E0101DB
:1016D000AE6F8205D8A41200E40E0001D66FFE0E94
:1016E000D76F060ED86F430ED96F060EDA6F000E55
:1016F000DB6F000EDC6F000EDD6F000EDE6F000E84
:10170000DF6FB5ECE6F01AC1D6F01BC1D7F04F0E73
:10171000D86F060ED96F000EDA6F000EDB6F000E69
:10172000DC6FC1ECD6F0000E0101826F12006E0E6C
:101730001119D8A496D30001A105D8A415D0070E7D
:10174000D66FF6C0D7F0010E88EC14F0CF0EEA6F1A
:10175000FE0EEB6F0E0EEC6F0CEC0FF0000EA16F97
:10176000010EA06F010E966F9805D8B468D3A0053E
:10177000D8A4120064D3560EE96FFD0EEA6F0D0E69
:10178000EB6FA7C0ECF0020E5CECF3F0510EC26FF1
:10179000FC0EC36F5A0EC46F010EC56F000EC66FEC
:1017A000000EC76F040EC86F000EC96F000ECA6F1F
:1017B000000ECB6F000ECC6F000ECD6FF6C0CEF0DA
:1017C000BAEC00F0490ED66FFD0ED76F0D0ED86F34
:1017D000030ED96F040EDA6F000EDB6F000EDC6FA4
:1017E000000EDD6F000EDE6F010EDF6FB5ECE6F070
:1017F000510EC26FFC0EC36F660EC46F010EC56F33
:10180000000EC66F000EC76F050EC86F000EC96FC1
:10181000000ECA6F000ECB6F000ECC6F000ECD6FA6
:10182000F6C0CEF0BAEC00F09C0ED66FFD0ED76F6E
:101830000B0ED86F030ED96F050EDA6F000EDB6F3B
:10184000000EDC6F000EDD6F000EDE6F010EDF6F2D
:10185000B5ECE6F0510EC26FFC0EC36F660EC46F9E
:10186000010EC56F000EC66F000EC76F060EC86F63
:10187000000EC96F000ECA6F000ECB6F000ECC6F4A
:10188000000ECD6FF6C0CEF0BAEC00F02C0ED66F85
:10189000FE0ED76F020ED86F030ED96F060EDA6FE9
:1018A000000EDB6F000EDC6F000EDD6F000EDE6FD2
:1018B000010EDF6FB5ECE6F0510EC26FFC0EC36F88
:1018C000660EC46F010EC56F000EC66F000EC76FA7
:1018D000070EC86F000EC96F000ECA6F000ECB6FE7
:1018E000000ECC6F000ECD6FF6C0CEF0BAEC00F05B
:1018F0002A0ED66FFE0ED76F020ED86F030ED96F69
:10190000070EDA6F000EDB6F000EDC6F000EDD6F6E
:10191000000EDE6F010EDF6FB5ECE6F0D0EF87F062
:10192000490EE96FFD0EEA6F0D0EEB6FA7C0ECF0EC
:10193000030E5CECF3F0510EC26FFC0EC36F5A0E37
:10194000C46F010EC56F000EC66F000EC76F020E8A
:10195000C86F000EC96F000ECA6F000ECB6F000E6D
:10196000CC6F000ECD6FF6C0CEF0BAEC00F0560E84
:10197000D66FFD0ED76F0D0ED86F030ED96F020E06
:10198000DA6F000EDB6F000EDC6F000EDD6F000EF5
:10199000DE6F010EDF6FB5ECE6F0510EC26FFC0E8C
:1019A000C36F5A0EC46F010EC56F000EC66F000ED6
:1019B000C76F050EC86F000EC96F000ECA6F000E0C
:1019C000CB6F000ECC6F000ECD6FF6C0CEF0BAEC30
:1019D00000F09C0ED66FFD0ED76F0B0ED86F030E66
:1019E000D96F050EDA6F000EDB6F000EDC6F000E94
:1019F000DD6F000EDE6F010EDF6FB5ECE6F02AD76B
:101A00009C0EE96FFD0EEA6F0B0EEB6FA7C0ECF0BA
:101A1000040E5CECF3F0510EC26FFC0EC36F5A0E55
:101A2000C46F010EC56F000EC66F000EC76F020EA9
:101A3000C86F000EC96F000ECA6F000ECB6F000E8C
:101A4000CC6F000ECD6FF6C0CEF0BAEC00F0560EA3
:101A5000D66FFD0ED76F0D0ED86F030ED96F020E25
:101A6000DA6F000EDB6F000EDC6F000EDD6F000E14
:101A7000DE6F010EDF6FB5ECE6F0510EC26FFC0EAB
:101A8000C36F5A0EC46F010EC56F000EC66F000EF5
:101A9000C76F030EC86F000EC96F000ECA6F000E2D
:101AA000CB6F000ECC6F000ECD6FF6C0CEF0BAEC4F
:101AB00000F0490ED66FFD0ED76F0D0ED86F030ED6
:101AC000D96F030EDA6F000EDB6F000EDC6F000EB5
:101AD000DD6F000EDE6F010EDF6FB5ECE6F0510E2C
:101AE000C26FFC0EC36F5A0EC46F010EC56F000E9D
:101AF000C66F000EC76F060EC86F000EC96F000ECE
:101B0000CA6F000ECB6F000ECC6F000ECD6FF6C00B
:101B1000CEF0BAEC00F0BAD62C0EE96FFE0EEA6FEA
:101B2000020EEB6FA7C0ECF0050E5CECF3F0510E6B
:101B3000C26FFC0EC36F5A0EC46F010EC56F000E4C
:101B4000C66F000EC76F020EC86F000EC96F000E81
:101B5000CA6F000ECB6F000ECC6F000ECD6FF6C0BB
:101B6000CEF0BAEC00F0560ED66FFD0ED76F0D0E0C
:101B7000D86F030ED96F020EDA6F000EDB6F000E06
:101B8000DC6F000EDD6F000EDE6F010EDF6FB5EC57
:101B9000E6F0510EC26FFC0EC36F5A0EC46F010EF9
:101BA000C56F000EC66F000EC76F030EC86F000E24
:101BB000C96F000ECA6F000ECB6F000ECC6F000E07
:101BC000CD6FF6C0CEF0BAEC00F0490ED66FFD0E28
:101BD000D76F0D0ED86F030ED96F030EDA6F000E9C
:101BE000DB6F000EDC6F000EDD6F000EDE6F010E8E
:101BF000DF6FB5ECE6F0510EC26FFC0EC36F5A0EEC
:101C0000C46F010EC56F000EC66F000EC76F040EC5
:101C1000C86F000EC96F000ECA6F000ECB6F000EAA
:101C2000CC6F000ECD6FF6C0CEF0BAEC00F09C0E7B
:101C3000D66FFD0ED76F0B0ED86F030ED96F040E43
:101C4000DA6F000EDB6F000EDC6F000EDD6F000E32
:101C5000DE6F010EDF6FB5ECE6F0510EC26FFC0EC9
:101C6000C36F5A0EC46F010EC56F000EC66F000E13
:101C7000C76F070EC86F000EC96F000ECA6F000E47
:101C8000CB6F000ECC6F000ECD6FF6C0CEF0BAEC6D
:101C900000F02ED62A0EE96FFE0EEA6F020EEB6FF1
:101CA000A7C0ECF0060E5CECF3F0510EC26FFC0E18
:101CB000C36F5A0EC46F010EC56F000EC66F000EC3
:101CC000C76F020EC86F000EC96F000ECA6F000EFC
:101CD000CB6F000ECC6F000ECD6FF6C0CEF0BAEC1D
:101CE00000F0560ED66FFD0ED76F0D0ED86F030E97
:101CF000D96F020EDA6F000EDB6F000EDC6F000E84
:101D0000DD6F000EDE6F010EDF6FB5ECE6F0510EF9
:101D1000C26FFC0EC36F5A0EC46F010EC56F000E6A
:101D2000C66F000EC76F030EC86F000EC96F000E9E
:101D3000CA6F000ECB6F000ECC6F000ECD6FF6C0D9
:101D4000CEF0BAEC00F0490ED66FFD0ED76F0D0E37
:101D5000D86F030ED96F030EDA6F000EDB6F000E23
:101D6000DC6F000EDD6F000EDE6F010EDF6FB5EC75
:101D7000E6F0510EC26FFC0EC36F5A0EC46F010E17
:101D8000C56F000EC66F000EC76F040EC86F000E41
:101D9000C96F000ECA6F000ECB6F000ECC6F000E25
:101DA000CD6FF6C0CEF0BAEC00F09C0ED66FFD0EF3
:101DB000D76F0B0ED86F030ED96F040EDA6F000EBB
:101DC000DB6F000EDC6F000EDD6F000EDE6F010EAC
:101DD000DF6FB5ECE6F0510EC26FFC0EC36F5A0E0A
:101DE000C46F010EC56F000EC66F000EC76F050EE3
:101DF000C86F000EC96F000ECA6F000ECB6F000EC9
:101E0000CC6F000ECD6FF6C0CEF0BAEC00F02C0E09
:101E1000D66FFE0ED76F020ED86F030ED96F050E68
:101E2000DA6F000EDB6F000EDC6F000EDD6F000E50
:101E3000DE6F010EDF6FB5ECE6F0D0EF87F0965164
:101E4000010AD8B498D4030AD8B46AD5010AD8B420
:101E5000D7D5070AD8B460D6010AD8B41BD7D0EFBB
:101E600087F06F0E1119D8A4BCD20001A105D8A427
:101E7000EED0070ED66FF6C0D7F0010E88EC14F046
:101E8000930EEA6FFE0EEB6F100EEC6F0CEC0FF082
:101E9000B3D0C70ED66FFF0ED76F060ED86F000EE9
:101EA000D96F020EDA6F000EDB6F000EDC6F000ED2
:101EB000DD6F000EDE6F000EDF6F61EC06F0CD0E01
:101EC000D66FFF0ED76F060ED86F000ED96F040EB7
:101ED000DA6F000EDB6F000EDC6F000EDD6F000EA0
:101EE000DE6F000EDF6F61EC06F04404D8A40AD068
:101EF000010ED66F020ED76F000ED86F6E51D3EC65
:101F0000E0F016D0BC0ED66FFF0ED76F050ED86F5F
:101F1000460ED96F020EDA6F000EDB6F000EDC6F1B
:101F2000000EDD6F000EDE6F000EDF6F61EC06F05D
:101F300001017A05D8A40ED06AC0D6F06BC0D7F0E4
:101F4000010E0001D86F040ED96F000EDA6F7BEC22
:101F5000D9F059D0BB0E0001D66FFF0ED76F060E19
:101F6000D86F3E0ED96F040EDA6F000EDB6F000ED5
:101F7000DC6F000EDD6F000EDE6F000EDF6F61ECB8
:101F800006F041D0C70ED66FFF0ED76F060ED86F82
:101F9000000ED96F020EDA6F000EDB6F000EDC6FE1
:101FA000000EDD6F000EDE6F000EDF6F61EC06F0DD
:101FB0004404D8A40AD0010ED66F020ED76F000ECB
:101FC000D86F6E51D3ECE0F01ED0BC0ED66FFF0E72
:101FD000D76F050ED86F460ED96F020EDA6F000E5E
:101FE000DB6F000EDC6F000EDD6F000EDE6F000E8B
:101FF000DF6F61EC06F007D09F51010AD8B4C2D759
:10200000020AD8B446D7F20EC26FC20EC36F440E96
:10201000C46F020EC56F010EC66F100EC76F060E9D
:10202000C86F000EC96F000ECA6F000ECB6F000E96
:10203000CC6F000ECD6FF6C0CEF0BAEC00F0000E03
:10204000A16F010EA06F010E966F010E986F98059B
:10205000D8B420D130D1480EC26FE50EC36F070E41
:10206000C46F020EC56F000EC66F250EC76F040E3B
:10207000C86F000EC96F000ECA6F000ECB6F000E46
:10208000CC6F000ECD6FF6C0CEF0BAEC00F0F20EC1
:10209000C26FC20EC36F440EC46F020EC56F010E35
:1020A000C66F100EC76F060EC86F000EC96F000E08
:1020B000CA6F000ECB6F000ECC6F000ECD6FF6C056
:1020C000CEF0BAEC00F0480EC26FE50EC36F070EFB
:1020D000C46F020EC56F5F0EC66F250EC76F020E6E
:1020E000C86F000EC96F000ECA6F000ECB6F000ED6
:1020F000CC6F000ECD6FF6C0CEF0BAEC00F0D4D0AD
:10210000480EC26FE50EC36F070EC46F020EC56F97
:10211000000EC66F250EC76F020EC86F000EC96F86
:10212000000ECA6F000ECB6F000ECC6F000ECD6F8D
:10213000F6C0CEF0BAEC00F09F05D8B439D0F20E5C
:10214000C26FC20EC36F440EC46F020EC56F010E84
:10215000C66F100EC76F060EC86F000EC96F000E57
:10216000CA6F000ECB6F000ECC6F000ECD6FF6C0A5
:10217000CEF0BAEC00F0480EC26FE50EC36F070E4A
:10218000C46F020EC56F5F0EC66F250EC76F040EBB
:10219000C86F000EC96F000ECA6F000ECB6F000E25
:1021A000CC6F000ECD6FF6C0CEF0BAEC00F07CD054
:1021B000F20EC26FC20EC36F440EC46F020EC56F23
:1021C000020EC66F100EC76F060EC86F000EC96FE5
:1021D000000ECA6F000ECB6F000ECC6F000ECD6FDD
:1021E000F6C0CEF0BAEC00F05FD0480EC26FE50E3C
:1021F000C36F070EC46F020EC56F000EC66F250EAB
:10220000C76F020EC86F000EC96F000ECA6F000EB6
:10221000CB6F000ECC6F000ECD6FF6C0CEF0BAECD7
:1022200000F0480EC26FE50EC36F070EC46F020EBA
:10223000C56F000EC66F250EC76F040EC86F000E67
:10224000C96F000ECA6F000ECB6F000ECC6F000E70
:10225000CD6FF6C0CEF0BAEC00F0F20EC26FC20E37
:10226000C36F440EC46F020EC56F020EC66F100E10
:10227000C76F060EC86F000EC96F000ECA6F000E42
:10228000CB6F000ECC6F000ECD6FF6C0CEF0BAEC67
:1022900000F00AD09651010AD8B4DDD6030AD8B4AA
:1022A0002FD7010AD8B4A1D796C097F0000E986F27
:1022B000000EA06F25D001013E05D8A40ED0010E5E
:1022C0000001D66F020ED76FA7C0D8F06C51D3ECC7
:1022D000E0F0000E01013E6F13D03D05D8A410D0F0
:1022E00068C0D6F069C0D7F0010E0001D86F040EA7
:1022F000D96FA7C0DAF07BECD9F0000E01013D6F79
:102300000001A005D8A453D09E05D8A40AD0010E80
:10231000D66F020ED76F010ED86F6C51D3ECE0F080
:1023200043D09D05D8A40DD068C0D6F069C0D7F0C1
:10233000010ED86F040ED96F010EDA6F7BECD9F065
:1023400033D04404D8A430D09F05D8A404D0020EC2
:102350009719D8B40DD001017A05D8A425D0030E61
:1023600000019719D8A420D0030E9F19D8A41CD01F
:10237000F20EC26FC20EC36F440EC46F020EC56F61
:10238000030EC66F100EC76F060EC86F000EC96F22
:10239000000ECA6F000ECB6F000ECC6F000ECD6F1B
:1023A000F6C0CEF0BAEC00F0000E0001A06F9E0562
:1023B000D8A40AD0410EBC6F140EBD6F9A5182ECA6
:1023C0000DF001013E6F12009D05D8A41200410ED0
:1023D000BC6F140EBD6F9A5182EC0DF001013D6F80
:1023E0001200700E1119D8A46ED00001A105D8A456
:1023F00045D0070ED66FF6C0D7F0010E88EC14F06A
:10240000830EEA6FFE0EEB6F100EEC6F0CEC0FF00C
:10241000F70ED66FFE0ED76F0D0ED86F000ED96F68
:10242000020EDA6F000EDB6F000EDC6F000EDD6F48
:10243000000EDE6F000EDF6F61EC06F0B205D8A46F
:1024400006D05A0ED66F480EB0ECFCF013D0020E38
:10245000B219D8A406D05A0ED66F200EB0ECFCF0FC
:1024600009D0030EB219D8A405D05A0ED66F200E8B
:10247000B0ECFCF0000EA16F010EA06F01013C0555
:10248000D8B404D00001A005D8A412D066C0D6F0FC
:1024900067C0D7F00A0E0001D86F040ED96FA7C02D
:1024A000DAF02FECCBF0000EA06F000E01013C6FB4
:1024B000410E0001BC6F140EBD6F9A5182EC0DF0FD
:1024C00001013C6F1200780E1119D8A496D30001B7
:1024D000A105D8A415D0070ED66FF6C0D7F0010E0F
:1024E00088EC14F0D90EEA6FFF0EEB6F060EEC6F5E
:1024F0000CEC0FF0000EA16F010EA06F010E966F95
:102500009805D8B468D3A005D8A4120064D3ED0E02
:10251000E96FFD0EEA6F090EEB6FA7C0ECF0020E3B
:102520005CECF3F0510EC26FFC0EC36F5A0EC46F19
:10253000010EC56F000EC66F000EC76F040EC86F88
:10254000000EC96F000ECA6F000ECB6F000ECC6F6D
:10255000000ECD6FF6C0CEF0BAEC00F0860ED66F4E
:10256000FD0ED76F0B0ED86F030ED96F040EDA6F06
:10257000000EDB6F000EDC6F000EDD6F000EDE6FF5
:10258000010EDF6FB5ECE6F0510EC26FFC0EC36FAB
:10259000660EC46F010EC56F000EC66F000EC76FCA
:1025A000050EC86F000EC96F000ECA6F000ECB6F0C
:1025B000000ECC6F000ECD6FF6C0CEF0BAEC00F07E
:1025C000E40ED66FFD0ED76F090ED86F030ED96FCC
:1025D000050EDA6F000EDB6F000EDC6F000EDD6F94
:1025E000000EDE6F010EDF6FB5ECE6F0510EC26F2C
:1025F000FC0EC36F660EC46F010EC56F000EC66F72
:10260000000EC76F060EC86F000EC96F000ECA6FAE
:10261000000ECB6F000ECC6F000ECD6FF6C0CEF06B
:10262000BAEC00F0D00ED66FFD0ED76F0A0ED86F41
:10263000030ED96F060EDA6F000EDB6F000EDC6F33
:10264000000EDD6F000EDE6F010EDF6FB5ECE6F001
:10265000510EC26FFC0EC36F660EC46F010EC56FC4
:10266000000EC66F000EC76F070EC86F000EC96F51
:10267000000ECA6F000ECB6F000ECC6F000ECD6F38
:10268000F6C0CEF0BAEC00F0150ED66FFE0ED76F86
:10269000060ED86F030ED96F070EDA6F000EDB6FD0
:1026A000000EDC6F000EDD6F000EDE6F010EDF6FBF
:1026B000B5ECE6F0D0EF87F0860EE96FFD0EEA6F1D
:1026C0000B0EEB6FA7C0ECF0030E5CECF3F0510EB9
:1026D000C26FFC0EC36F5A0EC46F010EC56F000EA1
:1026E000C66F000EC76F020EC86F000EC96F000ED6
:1026F000CA6F000ECB6F000ECC6F000ECD6FF6C010
:10270000CEF0BAEC00F0ED0ED66FFD0ED76F090ECD
:10271000D86F030ED96F020EDA6F000EDB6F000E5A
:10272000DC6F000EDD6F000EDE6F010EDF6FB5ECAB
:10273000E6F0510EC26FFC0EC36F5A0EC46F010E4D
:10274000C56F000EC66F000EC76F050EC86F000E76
:10275000C96F000ECA6F000ECB6F000ECC6F000E5B
:10276000CD6FF6C0CEF0BAEC00F0E40ED66FFD0EE1
:10277000D76F090ED86F030ED96F050EDA6F000EF2
:10278000DB6F000EDC6F000EDD6F000EDE6F010EE2
:10279000DF6FB5ECE6F02AD7E40EE96FFD0EEA6FC5
:1027A000090EEB6FA7C0ECF0040E5CECF3F0510ED9
:1027B000C26FFC0EC36F5A0EC46F010EC56F000EC0
:1027C000C66F000EC76F020EC86F000EC96F000EF5
:1027D000CA6F000ECB6F000ECC6F000ECD6FF6C02F
:1027E000CEF0BAEC00F0ED0ED66FFD0ED76F090EED
:1027F000D86F030ED96F020EDA6F000EDB6F000E7A
:10280000DC6F000EDD6F000EDE6F010EDF6FB5ECCA
:10281000E6F0510EC26FFC0EC36F5A0EC46F010E6C
:10282000C56F000EC66F000EC76F030EC86F000E97
:10283000C96F000ECA6F000ECB6F000ECC6F000E7A
:10284000CD6FF6C0CEF0BAEC00F0860ED66FFD0E5E
:10285000D76F0B0ED86F030ED96F030EDA6F000E11
:10286000DB6F000EDC6F000EDD6F000EDE6F010E01
:10287000DF6FB5ECE6F0510EC26FFC0EC36F5A0E5F
:10288000C46F010EC56F000EC66F000EC76F060E37
:10289000C86F000EC96F000ECA6F000ECB6F000E1E
:1028A000CC6F000ECD6FF6C0CEF0BAEC00F0BAD609
:1028B000D00EE96FFD0EEA6F0A0EEB6FA7C0ECF0C9
:1028C000050E5CECF3F0510EC26FFC0EC36F5A0E96
:1028D000C46F010EC56F000EC66F000EC76F020EEB
:1028E000C86F000EC96F000ECA6F000ECB6F000ECE
:1028F000CC6F000ECD6FF6C0CEF0BAEC00F0ED0E4E
:10290000D66FFD0ED76F090ED86F030ED96F020E6A
:10291000DA6F000EDB6F000EDC6F000EDD6F000E55
:10292000DE6F010EDF6FB5ECE6F0510EC26FFC0EEC
:10293000C36F5A0EC46F010EC56F000EC66F000E36
:10294000C76F030EC86F000EC96F000ECA6F000E6E
:10295000CB6F000ECC6F000ECD6FF6C0CEF0BAEC90
:1029600000F0860ED66FFD0ED76F0B0ED86F030EDC
:10297000D96F030EDA6F000EDB6F000EDC6F000EF6
:10298000DD6F000EDE6F010EDF6FB5ECE6F0510E6D
:10299000C26FFC0EC36F5A0EC46F010EC56F000EDE
:1029A000C66F000EC76F040EC86F000EC96F000E11
:1029B000CA6F000ECB6F000ECC6F000ECD6FF6C04D
:1029C000CEF0BAEC00F0E40ED66FFD0ED76F090E14
:1029D000D86F030ED96F040EDA6F000EDB6F000E96
:1029E000DC6F000EDD6F000EDE6F010EDF6FB5ECE9
:1029F000E6F0510EC26FFC0EC36F5A0EC46F010E8B
:102A0000C56F000EC66F000EC76F070EC86F000EB1
:102A1000C96F000ECA6F000ECB6F000ECC6F000E98
:102A2000CD6FF6C0CEF0BAEC00F02ED6150EE96FE1
:102A3000FE0EEA6F060EEB6FA7C0ECF0060E5CEC24
:102A4000F3F0510EC26FFC0EC36F5A0EC46F010E2D
:102A5000C56F000EC66F000EC76F020EC86F000E66
:102A6000C96F000ECA6F000ECB6F000ECC6F000E48
:102A7000CD6FF6C0CEF0BAEC00F0ED0ED66FFD0EC5
:102A8000D76F090ED86F030ED96F020EDA6F000EE2
:102A9000DB6F000EDC6F000EDD6F000EDE6F010ECF
:102AA000DF6FB5ECE6F0510EC26FFC0EC36F5A0E2D
:102AB000C46F010EC56F000EC66F000EC76F030E08
:102AC000C86F000EC96F000ECA6F000ECB6F000EEC
:102AD000CC6F000ECD6FF6C0CEF0BAEC00F0860ED3
:102AE000D66FFD0ED76F0B0ED86F030ED96F030E86
:102AF000DA6F000EDB6F000EDC6F000EDD6F000E74
:102B0000DE6F010EDF6FB5ECE6F0510EC26FFC0E0A
:102B1000C36F5A0EC46F010EC56F000EC66F000E54
:102B2000C76F040EC86F000EC96F000ECA6F000E8B
:102B3000CB6F000ECC6F000ECD6FF6C0CEF0BAECAE
:102B400000F0E40ED66FFD0ED76F090ED86F030E9E
:102B5000D96F040EDA6F000EDB6F000EDC6F000E13
:102B6000DD6F000EDE6F010EDF6FB5ECE6F0510E8B
:102B7000C26FFC0EC36F5A0EC46F010EC56F000EFC
:102B8000C66F000EC76F050EC86F000EC96F000E2E
:102B9000CA6F000ECB6F000ECC6F000ECD6FF6C06B
:102BA000CEF0BAEC00F0D00ED66FFD0ED76F0A0E45
:102BB000D86F030ED96F050EDA6F000EDB6F000EB3
:102BC000DC6F000EDD6F000EDE6F010EDF6FB5EC07
:102BD000E6F0D0EF87F09651010AD8B498D4030AF2
:102BE000D8B46AD5010AD8B4D7D5070AD8B460D604
:102BF000010AD8B41BD7D0EF87F0790E1119D8A4E9
:102C000065D00001A105D8A42FD0070ED66FF6C05D
:102C1000D7F0010E88EC14F0960EEA6FFF0EEB6F02
:102C2000090EEC6F0CEC0FF0000EA16F000E9A6F06
:102C3000F90E9425D66FD76BFF0ED7232E0ED86FC3
:102C4000020ED96F000EDA6F000EDB6F000EDC6F24
:102C500042ECCEF0050ED66F9451F90FD76F070EE8
:102C6000B3EC0CF0070F946F01016E05D8A41200AD
:102C7000F90E6F250001D66FD76BFF0ED7232E0EEE
:102C8000D86F020ED96F000EDA6F000EDB6F000EE8
:102C9000DC6F42ECCEF0050ED66F01016F51F90FDB
:102CA0000001D76F070EB3EC0CF0070F946F000E06
:102CB000C16F080EC06F94C0C2F0C36B5A0EC46FD0
:102CC000A2EC02F0000E01016E6F12007A0E1119D3
:102CD000D8A4C2EF9BF00001A105D8A415D0070E1F
:102CE000D66FF6C0D7F0010E88EC14F0B20EEA6F82
:102CF000FE0EEB6F0F0EEC6F0CEC0FF0000EA16FE1
:102D0000010E966F010E986F9805D8B4A4EF9AF053
:102D1000B3EF9AF0B105D8A455D0F20EC26FC20E2F
:102D2000C36F440EC46F020EC56F110EC66F080E3E
:102D3000C76F020EC86F000EC96F000ECA6F000E7B
:102D4000CB6F000ECC6F000ECD6FF6C0CEF0BAEC9C
:102D500000F0F20EC26FC20EC36F440EC46F020EBB
:102D6000C56F160EC66F080EC76F040EC86F000E33
:102D7000C96F000ECA6F000ECB6F000ECC6F000E35
:102D8000CD6FF6C0CEF0BAEC00F0F20EC26FC20EFC
:102D9000C36F440EC46F020EC56F120EC66F080ECD
:102DA000C76F060EC86F000EC96F000ECA6F000E07
:102DB000CB6F000ECC6F000ECD6FF6C0CEF0BAEC2C
:102DC00000F0B1D0020EB119D8A455D0F20EC26FE6
:102DD000C20EC36F440EC46F020EC56F0F0EC66FD6
:102DE000080EC76F020EC86F000EC96F000ECA6FC3
:102DF000000ECB6F000ECC6F000ECD6FF6C0CEF084
:102E0000BAEC00F0F20EC26FC20EC36F440EC46F74
:102E1000020EC56F180EC66F080EC76F040EC86F7E
:102E2000000EC96F000ECA6F000ECB6F000ECC6F84
:102E3000000ECD6FF6C0CEF0BAEC00F0F20EC26F0D
:102E4000C20EC36F440EC46F020EC56F120EC66F62
:102E5000080EC76F060EC86F000EC96F000ECA6F4E
:102E6000000ECB6F000ECC6F000ECD6FF6C0CEF013
:102E7000BAEC00F058D0030EB119D8A454D0F20E19
:102E8000C26FC20EC36F440EC46F020EC56F0F0E29
:102E9000C66F080EC76F020EC86F000EC96F000E16
:102EA000CA6F000ECB6F000ECC6F000ECD6FF6C058
:102EB000CEF0BAEC00F0F20EC26FC20EC36F440E39
:102EC000C46F020EC56F160EC66F080EC76F040ED4
:102ED000C86F000EC96F000ECA6F000ECB6F000ED8
:102EE000CC6F000ECD6FF6C0CEF0BAEC00F0F20E53
:102EF000C26FC20EC36F440EC46F020EC56F140EB4
:102F0000C66F080EC76F060EC86F000EC96F000EA1
:102F1000CA6F000ECB6F000ECC6F000ECD6FF6C0E7
:102F2000CEF0BAEC00F0480EC26FE50EC36F070E8C
:102F3000C46F020EC56F000EC66F500EC76F040E31
:102F4000C86F000EC96F000ECA6F000ECB6F000E67
:102F5000CC6F000ECD6FF6C0CEF0BAEC00F0480E8C
:102F6000C26FE50EC36F070EC46F020EC56F000E71
:102F7000C66F500EC76F060EC86F000EC96F000EE9
:102F8000CA6F000ECB6F000ECC6F000ECD6FF6C077
:102F9000CEF0BAEC00F0480EC26FE50EC36F070E1C
:102FA000C46F020EC56F6B0EC66F500EC76F020E58
:102FB000C86F000EC96F000ECA6F000ECB6F000EF7
:102FC000CC6F000ECD6FF6C0CEF0BAEC00F0C7D2D9
:102FD000020EB119D8A455D0F20EC26FC20EC36F43
:102FE000440EC46F020EC56F0E0EC66F080EC76F7B
:102FF000020EC86F000EC96F000ECA6F000ECB6FB5
:10300000000ECC6F000ECD6FF6C0CEF0BAEC00F023
:10301000F20EC26FC20EC36F440EC46F020EC56FB4
:10302000190EC66F080EC76F040EC86F000EC96F69
:10303000000ECA6F000ECB6F000ECC6F000ECD6F6E
:10304000F6C0CEF0BAEC00F0F20EC26FC20EC36F43
:10305000440EC46F020EC56F120EC66F080EC76F06
:10306000060EC86F000EC96F000ECA6F000ECB6F40
:10307000000ECC6F000ECD6FF6C0CEF0BAEC00F0B3
:10308000B0D0B105D8A455D0F20EC26FC20EC36F36
:10309000440EC46F020EC56F100EC66F080EC76FC8
:1030A000020EC86F000EC96F000ECA6F000ECB6F04
:1030B000000ECC6F000ECD6FF6C0CEF0BAEC00F073
:1030C000F20EC26FC20EC36F440EC46F020EC56F04
:1030D000170EC66F080EC76F040EC86F000EC96FBB
:1030E000000ECA6F000ECB6F000ECC6F000ECD6FBE
:1030F000F6C0CEF0BAEC00F0F20EC26FC20EC36F93
:10310000440EC46F020EC56F120EC66F080EC76F55
:10311000060EC86F000EC96F000ECA6F000ECB6F8F
:10312000000ECC6F000ECD6FF6C0CEF0BAEC00F002
:1031300058D0030EB119D8A454D0F20EC26FC20EEB
:10314000C36F440EC46F020EC56F0E0EC66F080E1D
:10315000C76F020EC86F000EC96F000ECA6F000E57
:10316000CB6F000ECC6F000ECD6FF6C0CEF0BAEC78
:1031700000F0F20EC26FC20EC36F440EC46F020E97
:10318000C56F170EC66F080EC76F040EC86F000E0E
:10319000C96F000ECA6F000ECB6F000ECC6F000E11
:1031A000CD6FF6C0CEF0BAEC00F0F20EC26FC20ED8
:1031B000C36F440EC46F020EC56F140EC66F080EA7
:1031C000C76F060EC86F000EC96F000ECA6F000EE3
:1031D000CB6F000ECC6F000ECD6FF6C0CEF0BAEC08
:1031E00000F0480EC26FE50EC36F070EC46F020EEB
:1031F000C56F000EC66F500EC76F020EC86F000E6F
:10320000C96F000ECA6F000ECB6F000ECC6F000EA0
:10321000CD6FF6C0CEF0BAEC00F0480EC26FE50EEE
:10322000C36F070EC46F020EC56F000EC66F500E3F
:10323000C76F060EC86F000EC96F000ECA6F000E72
:10324000CB6F000ECC6F000ECD6FF6C0CEF0BAEC97
:1032500000F0480EC26FE50EC36F070EC46F020E7A
:10326000C56F6B0EC66F500EC76F040EC86F000E91
:10327000C96F000ECA6F000ECB6F000ECC6F000E30
:10328000CD6FF6C0CEF0BAEC00F069D1030EB119E3
:10329000D8A455D0F20EC26FC20EC36F440EC46FD5
:1032A000020EC56F0E0EC66F080EC76F020EC86FF6
:1032B000000EC96F000ECA6F000ECB6F000ECC6FF0
:1032C000000ECD6FF6C0CEF0BAEC00F0F20EC26F79
:1032D000C20EC36F440EC46F020EC56F160EC66FCA
:1032E000080EC76F040EC86F000EC96F000ECA6FBC
:1032F000000ECB6F000ECC6F000ECD6FF6C0CEF07F
:10330000BAEC00F0F20EC26FC20EC36F440EC46F6F
:10331000020EC56F150EC66F080EC76F060EC86F7A
:10332000000EC96F000ECA6F000ECB6F000ECC6F7F
:10333000000ECD6FF6C0CEF0BAEC00F0B0D0B10503
:10334000D8A455D0F20EC26FC20EC36F440EC46F24
:10335000020EC56F100EC66F080EC76F020EC86F43
:10336000000EC96F000ECA6F000ECB6F000ECC6F3F
:10337000000ECD6FF6C0CEF0BAEC00F0F20EC26FC8
:10338000C20EC36F440EC46F020EC56F160EC66F19
:10339000080EC76F040EC86F000EC96F000ECA6F0B
:1033A000000ECB6F000ECC6F000ECD6FF6C0CEF0CE
:1033B000BAEC00F0F20EC26FC20EC36F440EC46FBF
:1033C000020EC56F130EC66F080EC76F060EC86FCC
:1033D000000EC96F000ECA6F000ECB6F000ECC6FCF
:1033E000000ECD6FF6C0CEF0BAEC00F058D0020E51
:1033F000B119D8A454D0F20EC26FC20EC36F440EDE
:10340000C46F020EC56F0E0EC66F080EC76F020E98
:10341000C86F000EC96F000ECA6F000ECB6F000E92
:10342000CC6F000ECD6FF6C0CEF0BAEC00F0F20E0D
:10343000C26FC20EC36F440EC46F020EC56F180E6A
:10344000C66F080EC76F040EC86F000EC96F000E5E
:10345000CA6F000ECB6F000ECC6F000ECD6FF6C0A2
:10346000CEF0BAEC00F0F20EC26FC20EC36F440E83
:10347000C46F020EC56F130EC66F080EC76F060E1F
:10348000C86F000EC96F000ECA6F000ECB6F000E22
:10349000CC6F000ECD6FF6C0CEF0BAEC00F0480E47
:1034A000C26FE50EC36F070EC46F020EC56F000E2C
:1034B000C66F500EC76F020EC86F000EC96F000EA8
:1034C000CA6F000ECB6F000ECC6F000ECD6FF6C032
:1034D000CEF0BAEC00F0480EC26FE50EC36F070ED7
:1034E000C46F020EC56F000EC66F500EC76F040E7C
:1034F000C86F000EC96F000ECA6F000ECB6F000EB2
:10350000CC6F000ECD6FF6C0CEF0BAEC00F0480ED6
:10351000C26FE50EC36F070EC46F020EC56F6B0E50
:10352000C66F500EC76F060EC86F000EC96F000E33
:10353000CA6F000ECB6F000ECC6F000ECD6FF6C0C1
:10354000CEF0BAEC00F00BD09651010AD8B48AEF55
:1035500096F0030AD8B43CD5010AD8B497D696C0E1
:1035600097F0000E986FA005D8A412009705D8A474
:1035700055D0F20EC26FC20EC36F440EC46F020E5E
:10358000C56F110EC66F080EC76F020EC86F000E12
:10359000C96F000ECA6F000ECB6F000ECC6F000E0D
:1035A000CD6FF6C0CEF0BAEC00F0F20EC26FC20ED4
:1035B000C36F440EC46F020EC56F160EC66F080EA1
:1035C000C76F040EC86F000EC96F000ECA6F000EE1
:1035D000CB6F000ECC6F000ECD6FF6C0CEF0BAEC04
:1035E00000F0F20EC26FC20EC36F440EC46F020E23
:1035F000C56F120EC66F080EC76F060EC86F000E9D
:10360000C96F000ECA6F000ECB6F000ECC6F000E9C
:10361000CD6FF6C0CEF0BAEC00F0B1D0020E971923
:10362000D8A455D0F20EC26FC20EC36F440EC46F41
:10363000020EC56F0E0EC66F080EC76F020EC86F62
:10364000000EC96F000ECA6F000ECB6F000ECC6F5C
:10365000000ECD6FF6C0CEF0BAEC00F0F20EC26FE5
:10366000C20EC36F440EC46F020EC56F190EC66F33
:10367000080EC76F040EC86F000EC96F000ECA6F28
:10368000000ECB6F000ECC6F000ECD6FF6C0CEF0EB
:10369000BAEC00F0F20EC26FC20EC36F440EC46FDC
:1036A000020EC56F120EC66F080EC76F060EC86FEA
:1036B000000EC96F000ECA6F000ECB6F000ECC6FEC
:1036C000000ECD6FF6C0CEF0BAEC00F058D0030E6D
:1036D0009719D8A454D0F20EC26FC20EC36F440E15
:1036E000C46F020EC56F0E0EC66F080EC76F020EB6
:1036F000C86F000EC96F000ECA6F000ECB6F000EB0
:10370000CC6F000ECD6FF6C0CEF0BAEC00F0F20E2A
:10371000C26FC20EC36F440EC46F020EC56F160E89
:10372000C66F080EC76F040EC86F000EC96F000E7B
:10373000CA6F000ECB6F000ECC6F000ECD6FF6C0BF
:10374000CEF0BAEC00F0F20EC26FC20EC36F440EA0
:10375000C46F020EC56F150EC66F080EC76F060E3A
:10376000C86F000EC96F000ECA6F000ECB6F000E3F
:10377000CC6F000ECD6FF6C0CEF0BAEC00F0000EAC
:10378000A06F12007B0E1119D8A41AD00001A10558
:10379000D8A41200070ED66FF6C0D7F0010E88EC41
:1037A00014F08D0EEA6FFF0EEB6F090EEC6F0CEC50
:1037B0000FF0000EA16F010EA06F010E966F1200A8
:1037C0007C0E1119D8A40AD10001A105D8A441D0BA
:1037D000070ED66FF6C0D7F0010E88EC14F05C0E21
:1037E000EA6FFF0EEB6F0A0EEC6F0CEC0FF02E0E73
:1037F000D66FFE0ED76F130ED86F000ED96F020E64
:10380000DA6F000EDB6F000EDC6F000EDD6F000E56
:10381000DE6F010EDF6FB5ECE6F0410ED66FFE0EE7
:10382000D76F110ED86F000ED96F030EDA6F000E2E
:10383000DB6F000EDC6F000EDD6F000EDE6F010E21
:10384000DF6FB5ECE6F0000EA16F020E966F010E71
:10385000986F9805D8B4B9D0A005D8A41200B5D0F7
:10386000A005D8A41DD0F20EC26FC20EC36F440EC5
:10387000C46F020EC56F090EC66F100EC76F040E1F
:10388000C86F000EC96F000ECA6F000ECB6F000E1E
:10389000CC6F000ECD6FF6C0CEF0BAEC00F01CD0AD
:1038A000F20EC26FC20EC36F440EC46F020EC56F1C
:1038B000080EC66F100EC76F040EC86F000EC96FDA
:1038C000000ECA6F000ECB6F000ECC6F000ECD6FD6
:1038D000F6C0CEF0BAEC00F0F20EC26FC20EC36FAB
:1038E000440EC46F020EC56F1D0EC66F100EC76F5B
:1038F000060EC86F000EC96F000ECA6F000ECB6FA8
:10390000000ECC6F000ECD6FF6C0CEF0BAEC00F01A
:10391000D0EF87F0F20EC26FC20EC36F440EC46FB9
:10392000020EC56F070EC66F100EC76F040EC86F6C
:10393000000EC96F000ECA6F000ECB6F000ECC6F69
:10394000000ECD6FF6C0CEF0BAEC00F0A005D8A402
:103950001ED0F20EC26FC20EC36F440EC46F020EB1
:10396000C56F1F0EC66F100EC76F060EC86F000E14
:10397000C96F000ECA6F000ECB6F000ECC6F000E29
:10398000CD6FF6C0CEF0BAEC00F0D0EF87F0F20EBB
:10399000C26FC20EC36F440EC46F020EC56F1E0EFF
:1039A000C66F100EC76F060EC86F000EC96F000EEF
:1039B000CA6F000ECB6F000ECC6F000ECD6FF6C03D
:1039C000CEF0BAEC00F0D0EF87F09651010AD8B4EF
:1039D00047D7030AD8B49ED7D0EF87F0810E1119CC
:1039E000D8A46CD00001A105D8A41200070ED66F90
:1039F000F6C0D7F0010E88EC14F0E50EEA6FFF0E6A
:103A0000EB6F060EEC6F0CEC0FF0630ED66FFE0E34
:103A1000D76F100ED86F060ED96F030EDA6F000E37
:103A2000DB6F000EDC6F000EDD6F000EDE6F000E30
:103A3000DF6FB5ECE6F0A30ED66FFE0ED76F0F0E5C
:103A4000D86F0A0ED96F040EDA6F000EDB6F000E0E
:103A5000DC6F000EDD6F000EDE6F000EDF6FB5EC69
:103A6000E6F0D30ED66FFF0ED76F060ED86F240E7A
:103A7000D96F050EDA6F000EDB6F000EDC6F000EE3
:103A8000DD6F000EDE6F000EDF6FB5ECE6F0730E3B
:103A9000D66FFE0ED76F100ED86F080ED96F060EB8
:103AA000DA6F000EDB6F000EDC6F000EDD6F000EB4
:103AB000DE6F000EDF6FB5ECE6F07BD6820E1119DB
:103AC000D8A496D30001A105D8A415D0070ED66FAF
:103AD000F6C0D7F0010E88EC14F03C0EEA6FFF0E32
:103AE000EB6F0B0EEC6F0CEC0FF0000EA16F010EE4
:103AF000A06F010E966F9805D8B468D3A005D8A41E
:103B0000120064D3910EE96FFD0EEA6F0B0EEB6F9E
:103B1000A7C0ECF0020E5CECF3F0510EC26FFC0E8D
:103B2000C36F5A0EC46F010EC56F000EC66F000E34
:103B3000C76F040EC86F000EC96F000ECA6F000E6B
:103B4000CB6F000ECC6F000ECD6FF6C0CEF0BAEC8E
:103B500000F0DA0ED66FFD0ED76F0A0ED86F030E87
:103B6000D96F040EDA6F000EDB6F000EDC6F000EF3
:103B7000DD6F000EDE6F010EDF6FB5ECE6F0510E6B
:103B8000C26FFC0EC36F660EC46F010EC56F000ED0
:103B9000C66F000EC76F050EC86F000EC96F000E0E
:103BA000CA6F000ECB6F000ECC6F000ECD6FF6C04B
:103BB000CEF0BAEC00F0280ED66FFE0ED76F020ED4
:103BC000D86F030ED96F050EDA6F000EDB6F000E93
:103BD000DC6F000EDD6F000EDE6F010EDF6FB5ECE7
:103BE000E6F0510EC26FFC0EC36F660EC46F010E7D
:103BF000C56F000EC66F000EC76F060EC86F000EB1
:103C0000C96F000ECA6F000ECB6F000ECC6F000E96
:103C1000CD6FF6C0CEF0BAEC00F0260ED66FFE0ED9
:103C2000D76F020ED86F030ED96F060EDA6F000E33
:103C3000DB6F000EDC6F000EDD6F000EDE6F010E1D
:103C4000DF6FB5ECE6F0510EC26FFC0EC36F660E6F
:103C5000C46F010EC56F000EC66F000EC76F070E52
:103C6000C86F000EC96F000ECA6F000ECB6F000E3A
:103C7000CC6F000ECD6FF6C0CEF0BAEC00F0240E83
:103C8000D66FFE0ED76F020ED86F030ED96F070ED8
:103C9000DA6F000EDB6F000EDC6F000EDD6F000EC2
:103CA000DE6F010EDF6FB5ECE6F0D0EF87F0DA0ED5
:103CB000E96FFD0EEA6F0A0EEB6FA7C0ECF0030E82
:103CC0005CECF3F0510EC26FFC0EC36F5A0EC46F62
:103CD000010EC56F000EC66F000EC76F020EC86FD3
:103CE000000EC96F000ECA6F000ECB6F000ECC6FB6
:103CF000000ECD6FF6C0CEF0BAEC00F0910ED66F8C
:103D0000FD0ED76F0B0ED86F030ED96F020EDA6F50
:103D1000000EDB6F000EDC6F000EDD6F000EDE6F3D
:103D2000010EDF6FB5ECE6F0510EC26FFC0EC36FF3
:103D30005A0EC46F010EC56F000EC66F000EC76F1E
:103D4000050EC86F000EC96F000ECA6F000ECB6F54
:103D5000000ECC6F000ECD6FF6C0CEF0BAEC00F0C6
:103D6000280ED66FFE0ED76F020ED86F030ED96FD6
:103D7000050EDA6F000EDB6F000EDC6F000EDD6FDC
:103D8000000EDE6F010EDF6FB5ECE6F02AD7280ECD
:103D9000E96FFE0EEA6F020EEB6FA7C0ECF0040EA7
:103DA0005CECF3F0510EC26FFC0EC36F5A0EC46F81
:103DB000010EC56F000EC66F000EC76F020EC86FF2
:103DC000000EC96F000ECA6F000ECB6F000ECC6FD5
:103DD000000ECD6FF6C0CEF0BAEC00F0910ED66FAB
:103DE000FD0ED76F0B0ED86F030ED96F020EDA6F70
:103DF000000EDB6F000EDC6F000EDD6F000EDE6F5D
:103E0000010EDF6FB5ECE6F0510EC26FFC0EC36F12
:103E10005A0EC46F010EC56F000EC66F000EC76F3D
:103E2000030EC86F000EC96F000ECA6F000ECB6F75
:103E3000000ECC6F000ECD6FF6C0CEF0BAEC00F0E5
:103E4000DA0ED66FFD0ED76F0A0ED86F030ED96F3C
:103E5000030EDA6F000EDB6F000EDC6F000EDD6FFD
:103E6000000EDE6F010EDF6FB5ECE6F0510EC26F93
:103E7000FC0EC36F5A0EC46F010EC56F000EC66FE5
:103E8000000EC76F060EC86F000EC96F000ECA6F16
:103E9000000ECB6F000ECC6F000ECD6FF6C0CEF0D3
:103EA000BAEC00F0BAD6260EE96FFE0EEA6F020EEB
:103EB000EB6FA7C0ECF0050E5CECF3F0510EC26F97
:103EC000FC0EC36F5A0EC46F010EC56F000EC66F95
:103ED000000EC76F020EC86F000EC96F000ECA6FCA
:103EE000000ECB6F000ECC6F000ECD6FF6C0CEF083
:103EF000BAEC00F0910ED66FFD0ED76F0B0ED86F97
:103F0000030ED96F020EDA6F000EDB6F000EDC6F4E
:103F1000000EDD6F000EDE6F010EDF6FB5ECE6F018
:103F2000510EC26FFC0EC36F5A0EC46F010EC56FE7
:103F3000000EC66F000EC76F030EC86F000EC96F6C
:103F4000000ECA6F000ECB6F000ECC6F000ECD6F4F
:103F5000F6C0CEF0BAEC00F0DA0ED66FFD0ED76FD9
:103F60000A0ED86F030ED96F030EDA6F000EDB6FE7
:103F7000000EDC6F000EDD6F000EDE6F010EDF6FD6
:103F8000B5ECE6F0510EC26FFC0EC36F5A0EC46F53
:103F9000010EC56F000EC66F000EC76F040EC86F0E
:103FA000000EC96F000ECA6F000ECB6F000ECC6FF3
:103FB000000ECD6FF6C0CEF0BAEC00F0280ED66F32
:103FC000FE0ED76F020ED86F030ED96F040EDA6F94
:103FD000000EDB6F000EDC6F000EDD6F000EDE6F7B
:103FE000010EDF6FB5ECE6F0510EC26FFC0EC36F31
:103FF0005A0EC46F010EC56F000EC66F000EC76F5C
:10400000070EC86F000EC96F000ECA6F000ECB6F8F
:10401000000ECC6F000ECD6FF6C0CEF0BAEC00F003
:104020002ED6240EE96FFE0EEA6F020EEB6FA7C0CC
:10403000ECF0060E5CECF3F0510EC26FFC0EC36F99
:104040005A0EC46F010EC56F000EC66F000EC76F0B
:10405000020EC86F000EC96F000ECA6F000ECB6F44
:10406000000ECC6F000ECD6FF6C0CEF0BAEC00F0B3
:10407000910ED66FFD0ED76F0B0ED86F030ED96F52
:10408000020EDA6F000EDB6F000EDC6F000EDD6FCC
:10409000000EDE6F010EDF6FB5ECE6F0510EC26F61
:1040A000FC0EC36F5A0EC46F010EC56F000EC66FB3
:1040B000000EC76F030EC86F000EC96F000ECA6FE7
:1040C000000ECB6F000ECC6F000ECD6FF6C0CEF0A1
:1040D000BAEC00F0DA0ED66FFD0ED76F0A0ED86F6D
:1040E000030ED96F030EDA6F000EDB6F000EDC6F6C
:1040F000000EDD6F000EDE6F010EDF6FB5ECE6F037
:10410000510EC26FFC0EC36F5A0EC46F010EC56F05
:10411000000EC66F000EC76F040EC86F000EC96F89
:10412000000ECA6F000ECB6F000ECC6F000ECD6F6D
:10413000F6C0CEF0BAEC00F0280ED66FFE0ED76FA8
:10414000020ED86F030ED96F040EDA6F000EDB6F0C
:10415000000EDC6F000EDD6F000EDE6F010EDF6FF4
:10416000B5ECE6F0510EC26FFC0EC36F5A0EC46F71
:10417000010EC56F000EC66F000EC76F050EC86F2B
:10418000000EC96F000ECA6F000ECB6F000ECC6F11
:10419000000ECD6FF6C0CEF0BAEC00F0260ED66F52
:1041A000FE0ED76F020ED86F030ED96F050EDA6FB1
:1041B000000EDB6F000EDC6F000EDD6F000EDE6F99
:1041C000010EDF6FB5ECE6F0D0EF87F09651010AF3
:1041D000D8B498D4030AD8B46AD5010AD8B4D7D5CC
:1041E000070AD8B460D6010AD8B41BD7D0EF87F03D
:1041F000830E1119D8A4B1D30001A105D8A43CD0D5
:10420000070ED66FF6C0D7F0010E88EC14F01B0E27
:10421000EA6FFF0EEB6F0B0EEC6F0CEC0FF0EB0E7A
:10422000D66FFF0ED76F050ED86F000ED96F020E36
:10423000DA6F000EDB6F000EDC6F000EDD6F000E1C
:10424000DE6F000EDF6F61EC06F09C05D8A404D091
:10425000000E936F030E03D0010E936F010E966F45
:10426000000EA16F74517511D8A404D0000E756FA3
:10427000010E746F010E986F9805D8B46AD27AD285
:10428000480EC26FE50EC36F070EC46F020EC56FF6
:10429000000EC66F450EC76F040EC86F000EC96FC3
:1042A000000ECA6F000ECB6F000ECC6F000ECD6FEC
:1042B000F6C0CEF0BAEC00F0480EC26FE50EC36F48
:1042C000070EC46F020EC56F6B0EC66F450EC76F2B
:1042D000020EC86F000EC96F000ECA6F000ECB6FC2
:1042E000000ECC6F000ECD6FF6C0CEF0BAEC00F031
:1042F00072C0D6F073C0D7F01E0ED86F020ED96F01
:10430000000EDA6F000EDB6F000EDC6F42ECCEF0B9
:10431000B751D8A41DD0F20EC26FC20EC36F440EA7
:10432000C46F020EC56F0A0EC66F000EC76F040E73
:10433000C86F000EC96F000ECA6F000ECB6F000E63
:10434000CC6F000ECD6FF6C0CEF0BAEC00F01CD0F2
:10435000F20EC26FC20EC36F440EC46F020EC56F61
:104360000C0EC66F000EC76F040EC86F000EC96F2B
:10437000000ECA6F000ECB6F000ECC6F000ECD6F1B
:10438000F6C0CEF0BAEC00F09305D8A41DD0F20E22
:10439000C26FC20EC36F440EC46F020EC56F040E0F
:1043A000C66F000EC76F060EC86F000EC96F000EF5
:1043B000CA6F000ECB6F000ECC6F000ECD6FF6C033
:1043C000CEF0BAEC00F01CD0F20EC26FC20EC36F7A
:1043D000440EC46F020EC56F1A0EC66F000EC76F73
:1043E000060EC86F000EC96F000ECA6F000ECB6FAD
:1043F000000ECC6F000ECD6FF6C0CEF0BAEC00F020
:10440000B205D8A406D05A0ED66F200EB0ECFCF040
:10441000AAD1020EB219D8A406D05A0ED66F200E19
:10442000B0ECFCF0A0D1030EB219D8A49CD15A0E66
:10443000D66F200EB0ECFCF096D1480EC26FE50EA0
:10444000C36F070EC46F020EC56F000EC66F450E18
:10445000C76F020EC86F000EC96F000ECA6F000E44
:10446000CB6F000ECC6F000ECD6FF6C0CEF0BAEC65
:1044700000F0480EC26FE50EC36F070EC46F020E48
:10448000C56F6B0EC66F450EC76F040EC86F000E6A
:10449000C96F000ECA6F000ECB6F000ECC6F000EFE
:1044A000CD6FF6C0CEF0BAEC00F072C0D6F073C09B
:1044B000D7F01E0ED86F020ED96F000EDA6F000E05
:1044C000DB6F000EDC6F42ECCEF0B751D8A41DD0EC
:1044D000F20EC26FC20EC36F440EC46F020EC56FE0
:1044E0000B0EC66F000EC76F040EC86F000EC96FAB
:1044F000000ECA6F000ECB6F000ECC6F000ECD6F9A
:10450000F6C0CEF0BAEC00F01CD0F20EC26FC20EB4
:10451000C36F440EC46F020EC56F0D0EC66F000E42
:10452000C76F040EC86F000EC96F000ECA6F000E71
:10453000CB6F000ECC6F000ECD6FF6C0CEF0BAEC94
:1045400000F09305D8A41DD0F20EC26FC20EC36F47
:10455000440EC46F020EC56F040EC66F000EC76F07
:10456000060EC86F000EC96F000ECA6F000ECB6F2B
:10457000000ECC6F000ECD6FF6C0CEF0BAEC00F09E
:104580001CD0F20EC26FC20EC36F440EC46F020E77
:10459000C56F1A0EC66F000EC76F060EC86F000EED
:1045A000C96F000ECA6F000ECB6F000ECC6F000EED
:1045B000CD6FF6C0CEF0BAEC00F0780ED66F780E64
:1045C000B0ECFCF0D0D0480EC26FE50EC36F070E02
:1045D000C46F020EC56F000EC66F450EC76F020E88
:1045E000C86F000EC96F000ECA6F000ECB6F000EB1
:1045F000CC6F000ECD6FF6C0CEF0BAEC00F0480ED6
:10460000C26FE50EC36F070EC46F020EC56F000EBA
:10461000C66F450EC76F040EC86F000EC96F000E3F
:10462000CA6F000ECB6F000ECC6F000ECD6FF6C0C0
:10463000CEF0BAEC00F072C0D6F073C0D7F01E0E08
:10464000D86F020ED96F000EDA6F000EDB6F000E0E
:10465000DC6F42ECCEF0B751D8A41DD0F20EC26F81
:10466000C20EC36F440EC46F020EC56F0A0EC66F32
:10467000000EC76F040EC86F000EC96F000ECA6F20
:10468000000ECB6F000ECC6F000ECD6FF6C0CEF0DB
:10469000BAEC00F01CD0F20EC26FC20EC36F440E13
:1046A000C46F020EC56F0C0EC66F000EC76F040EEE
:1046B000C86F000EC96F000ECA6F000ECB6F000EE0
:1046C000CC6F000ECD6FF6C0CEF0BAEC00F09305C3
:1046D000D8A41DD0F20EC26FC20EC36F440EC46FB9
:1046E000020EC56F050EC66F000EC76F060EC86FAF
:1046F000000EC96F000ECA6F000ECB6F000ECC6F9C
:10470000000ECD6FF6C0CEF0BAEC00F01CD0F20E69
:10471000C26FC20EC36F440EC46F020EC56F1B0E74
:10472000C66F000EC76F060EC86F000EC96F000E71
:10473000CA6F000ECB6F000ECC6F000ECD6FF6C0AF
:10474000CEF0BAEC00F0780ED66F780EB0ECFCF03C
:104750000AD09651010AD8B493D5030AD8B46DD6BD
:10476000010AD8B430D796C097F0000E986F000EAB
:10477000A06F20D001015705D8A41CD000017051B2
:104780007111D8A404D0000E716F010E706F70C04B
:10479000D6F071C0D7F01E0ED86F020ED96F000E82
:1047A000DA6F000EDB6F000EDC6F42ECCEF0000E15
:1047B0000101576F0001A005D8A4C5D08E05D8A46B
:1047C00036D070C0D6F071C0D7F01E0ED86F020E72
:1047D000D96F000EDA6F000EDB6F000EDC6F42EC5B
:1047E000CEF070C072F071C073F09351D8A4A9D00C
:1047F000F20EC26FC20EC36F440EC46F020EC56FBD
:10480000040EC66F000EC76F060EC86F000EC96F8C
:10481000000ECA6F000ECB6F000ECC6F000ECD6F76
:10482000F6C0CEF0BAEC00F0010E936F8AD0020E03
:104830009719D8A446D001015605D8A41FD0F20E6E
:104840000001C26FC20EC36F440EC46F020EC56F6B
:104850000D0EC66F000EC76F040EC86F000EC96F35
:10486000000ECA6F000ECB6F000ECC6F000ECD6F26
:10487000F6C0CEF0BAEC00F0010E1ED0F20E000130
:10488000C26FC20EC36F440EC46F020EC56F0B0E13
:10489000C66F000EC76F040EC86F000EC96F000E02
:1048A000CA6F000ECB6F000ECC6F000ECD6FF6C03E
:1048B000CEF0BAEC00F0000EB76F9351D8B498D791
:1048C00040D0030E9719D8A43CD09305D8A41DD08E
:1048D000F20EC26FC20EC36F440EC46F020EC56FDC
:1048E000060EC66F000EC76F060EC86F000EC96FAA
:1048F000000ECA6F000ECB6F000ECC6F000ECD6F96
:10490000F6C0CEF0BAEC00F01CD0F20EC26FC20EB0
:10491000C36F440EC46F020EC56F1C0EC66F000E2F
:10492000C76F060EC86F000EC96F000ECA6F000E6B
:10493000CB6F000ECC6F000ECD6FF6C0CEF0BAEC90
:1049400000F0000EA06F410EBC6F140EBD6F9A51A7
:1049500082EC0DF00101576F1200840E1119D8A4DA
:1049600058D2360E0A6F1B0E0E6F5F0E0D6F0001D0
:10497000A105D8A448D0070ED66FF6C0D7F0010E17
:1049800088EC14F0310EEA6FFF0EEB6F0B0EEC6F3C
:104990000CEC0FF09F0ED66FFF0ED76F080ED86F7E
:1049A000000ED96F020EDA6F000EDB6F000EDC6FA7
:1049B000000EDD6F000EDE6F000EDF6F61EC06F0A3
:1049C000C10ED66FFF0ED76F060ED86F000ED96FCF
:1049D000040EDA6F000EDB6F000EDC6F000EDD6F71
:1049E000000EDE6F000EDF6F61EC06F0000EA16FAF
:1049F000010EA06F010E966F010E986F010E01015E
:104A0000406F010E3F6F00019805D8B427D137D110
:104A1000480EC26FE50EC36F070EC46F020EC56F5E
:104A2000000EC66F0DC4C7F0040EC86F000EC96F2C
:104A3000000ECA6F000ECB6F000ECC6F000ECD6F54
:104A4000F6C0CEF0BAEC00F0480EC26FE50EC36FB0
:104A5000070EC46F020EC56F6B0EC66F0DC4C7F094
:104A6000020EC86F000EC96F000ECA6F000ECB6F2A
:104A7000000ECC6F000ECD6FF6C0CEF0BAEC00F099
:104A80008651D8A41DD06E0EC26FEE0EC36F320ECB
:104A9000C46F020EC56F010EC66F0EC4C7F0060EBE
:104AA000C86F000EC96F000ECA6F000ECB6F000EEC
:104AB000CC6F000ECD6FF6C0CEF0BAEC00F0D8D0BF
:104AC0006E0EC26FEE0EC36F320EC46F020EC56F54
:104AD000040EC66F0EC4C7F0060EC86F000EC96F75
:104AE000000ECA6F000ECB6F000ECC6F000ECD6FA4
:104AF000F6C0CEF0BAEC00F0BBD0480EC26FE50EA7
:104B0000C36F070EC46F020EC56F000EC66F0DC4D3
:104B1000C7F0020EC86F000EC96F000ECA6F000EFC
:104B2000CB6F000ECC6F000ECD6FF6C0CEF0BAEC9E
:104B300000F0480EC26FE50EC36F070EC46F020E81
:104B4000C56F6B0EC66F0DC4C7F0040EC86F000EA4
:104B5000C96F000ECA6F000ECB6F000ECC6F000E37
:104B6000CD6FF6C0CEF0BAEC00F08651D8B48BD73A
:104B7000A7D7480EC26FE50EC36F070EC46F020EB3
:104B8000C56F000EC66F0DC4C7F0020EC86F000ED1
:104B9000C96F000ECA6F000ECB6F000ECC6F000EF7
:104BA000CD6FF6C0CEF0BAEC00F0480EC26FE50E45
:104BB000C36F070EC46F020EC56F000EC66F0DC423
:104BC000C7F0040EC86F000EC96F000ECA6F000E4A
:104BD000CB6F000ECC6F000ECD6FF6C0CEF0BAECEE
:104BE00000F08651D8A41DD06E0EC26FEE0EC36FBA
:104BF000320EC46F020EC56F020EC66F0EC4C7F030
:104C0000060EC86F000EC96F000ECA6F000ECB6F84
:104C1000000ECC6F000ECD6FF6C0CEF0BAEC00F0F7
:104C200027D06E0EC26FEE0EC36F320EC46F020E2F
:104C3000C56F050EC66F0EC4C7F0060EC86F000E16
:104C4000C96F000ECA6F000ECB6F000ECC6F000E46
:104C5000CD6FF6C0CEF0BAEC00F00AD09651010A42
:104C6000D8B4D6D6030AD8B448D7010AD8B481D765
:104C700096C097F0000E986F000EA06F40D0010113
:104C80004005D8A41DD031503210D8A404D0000E55
:104C9000326E010E316E31C0D6F032C0D7F00AC488
:104CA000D8F0020E0001D96F000EDA6F000EDB6F34
:104CB000000EDC6F42ECCEF0000E0101406F1FD001
:104CC0003F05D8A41CD02F503010D8A404D0000E1B
:104CD000306E010E2F6E2FC0D6F030C0D7F00AC450
:104CE000D8F0040E0001D96F000EDA6F000EDB6FF2
:104CF000000EDC6F42ECCEF0000E01013F6F0001B0
:104D0000A005D8A46CD08505D8A413D031C0D6F0A6
:104D100032C0D7F00AC4D8F0020ED96F000EDA6F95
:104D2000000EDB6F000EDC6F42ECCEF0000E9A6FCF
:104D300054D08405D8A411D02FC0D6F030C0D7F0FD
:104D40000AC4D8F0040ED96F000EDA6F000EDB6FC4
:104D5000000EDC6F42ECCEF0E9D7030E9719D8A411
:104D60003CD08651D8A41DD06E0EC26FEE0EC36F1C
:104D7000320EC46F020EC56F030EC66F0EC4C7F0AD
:104D8000060EC86F000EC96F000ECA6F000ECB6F03
:104D9000000ECC6F000ECD6FF6C0CEF0BAEC00F076
:104DA0001CD06E0EC26FEE0EC36F320EC46F020EB9
:104DB000C56F060EC66F0EC4C7F0060EC86F000E94
:104DC000C96F000ECA6F000ECB6F000ECC6F000EC5
:104DD000CD6FF6C0CEF0BAEC00F0000EA06F8505E6
:104DE000D8A40AD0410EBC6F140EBD6F9A5182EC4C
:104DF0000DF00101406F12008405D8A41200410E8D
:104E0000BC6F140EBD6F9A5182EC0DF001013F6F23
:104E100012001105D8A4F9D00001A105D8A42DD005
:104E2000E80EC26FDE0EC36F660EC46F040EC56F50
:104E3000010EC66F650EC76F000EC86F000EC96FFA
:104E4000000ECA6F000ECB6F000ECC6F000ECD6F40
:104E5000F6C0CEF0BAEC00F001014E51D8A402D059
:104E6000010E01D0650E416E000E0201A46F010E0D
:104E70000101C36F000E0001A16F060E0101C265A2
:104E80001200650E416002D0412A3ED0E80E0001BA
:104E9000C26FDE0EC36F660EC46F040EC56F020EC6
:104EA000C66F160EC76F040EC86F000EC96F000ED6
:104EB000CA6F000ECB6F000ECC6F000ECD6FF6C028
:104EC000CEF0BAEC00F0710EC26FF70EC36F0F0E8A
:104ED000C46F020EC56F0A0EC66F590EC76F060E5D
:104EE000C86F000EC96F000ECA6F000ECB6F000EA8
:104EF000CC6F000ECD6FF6C0CEF0BAEC00F0000E15
:104F00000101C36F010EC16F3A0E416430D0F80E3B
:104F10000001D66F020ED76F050ED86F415065089D
:104F2000D96F040EDA6F000EDB6F000EDC6F000E1F
:104F3000DD6F000EDE6F010EDF6FB5ECE6F0E80E00
:104F4000D66FFE0ED76F020ED86F41507B08D96F17
:104F5000040EDA6F000EDB6F000EDC6F000EDD6FEB
:104F6000000EDE6F010EDF6FB5ECE6F02DD0F60E11
:104F70000001D66FFD0ED76F080ED86F000ED96FE7
:104F8000040EDA6F000EDB6F000EDC6F000EDD6FBB
:104F9000000EDE6F010EDF6FB5ECE6F0F80ED66F97
:104FA000020ED76F050ED86F2A0ED96F040EDA6F76
:104FB000000EDB6F000EDC6F000EDD6F000EDE6F8B
:104FC000010EDF6FB5ECE6F0E80EC26FDE0EC36FC8
:104FD000660EC46F040EC56F010EC66F41506508A2
:104FE000C76F000EC86F000EC96F000ECA6F000EAB
:104FF000CB6F000ECC6F000ECD6FF6C0CEF0BAECCA
:1050000000F0000E0101C26F1200030E1119D8A4A6
:105010004AD00001A105D8A41BD08305D8A40BD089
:1050200042C0D6F0D76B100ED86F020ED96F020EA9
:1050300022ECD1F00BD0000ED76F000ED66F100E01
:10504000D86F020ED96F050E22ECD1F0000EA16FC1
:1050500001017505D8A4120000018305D8A412002F
:10506000480EC26FE50EC36F070EC46F020EC56F08
:105070004250600FC66F290EC76F050EC86F000E35
:10508000C96F000ECA6F010ECB6F000ECC6F000E01
:10509000CD6FF6C0CEF0BAEC00F042C076F1000E53
:1050A0000101756F1200040E1119D8A442D0100E20
:1050B000056F020E066F0001A105D8A40CD095C0A3
:1050C000D6F0D76B05C4D8F006C4D9F0040E22EC94
:1050D000D1F0000EA16F01017305D8A41200480E93
:1050E0000001C26FE50EC36F070EC46F020EC56FDD
:1050F0009551600FC66F04010551190F0001C76F6C
:1051000004010651030F0001C86F000EC96F000EA5
:10511000CA6F010ECB6F000ECC6F000ECD6FF6C0C4
:10512000CEF0BAEC00F095C074F1000E0101736F7F
:105130001200050E1119D8A49DD0100E0B6F020E8F
:105140000C6F020E096F090E046F0001A105D8A4AF
:105150000DD0000ED76F1E0ED66F0BC4D8F00CC446
:10516000D9F0030E22ECD1F0000EA16F01017305FE
:10517000D8A412000A0E0001C06F955119EC16F068
:10518000600F0401096F0A0E0001BC6F95518AEC93
:1051900017F0600F0401046F600E0919D8B424D011
:1051A000480E0001C26FE50EC36F070EC46F020EFA
:1051B000C56F09C4C6F004010B51150F0001C76F7C
:1051C00004010C51030F0001C86F000EC96F000EDF
:1051D000CA6F010ECB6F000ECC6F000ECD6FF6C004
:1051E000CEF0BAEC00F023D0480E0001C26FE50EFD
:1051F000C36F070EC46F020EC56F6C0EC66F04013D
:105200000B51150F0001C76F04010C51030F000172
:10521000C86F000EC96F000ECA6F010ECB6F000E73
:10522000CC6F000ECD6FF6C0CEF0BAEC00F0480E99
:10523000C26FE50EC36F070EC46F020EC56F04C4C4
:10524000C6F004010B511E0F0001C76F04010C5181
:10525000030F0001C86F000EC96F000ECA6F010E68
:10526000CB6F000ECC6F000ECD6FF6C0CEF0BAEC57
:1052700000F059D7060E1119D8A41200100E076FAE
:10528000020E086F0001A105D8A40CD040C0D6F0D2
:10529000D76B07C4D8F008C4D9F00D0E22ECD1F0BA
:1052A000000EA16F01016C05D8A41200480E000188
:1052B000C26FE50EC36F070EC46F020EC56F40507C
:1052C000600FC66F04010751190F0001C76F040179
:1052D0000851030F0001C86F000EC96F000ECA6F9E
:1052E000010ECB6F000ECC6F000ECD6FF6C0CEF06E
:1052F000BAEC00F040C06DF1000E01016C6F1200BD
:105300004AEC0EF0DCECEFF0000E0001BD6F000E79
:10531000BC6F09EC19F0A10AD8B409D0000E000145
:10532000BD6F000EBC6FA10EBE6F3CEC15F0A10E60
:1053300091EC13F0A4EC19F0210E3A01136F3D012A
:105340007399D28ED28C010E60EC14F0F66FF65188
:105350009FEC0AF0010E0001A46F010E506EC68290
:10536000200E7DEC18F00101E66FA2EC19F08DEC37
:10537000DEF0ACEC16F0000E0001CC6F37C0CDF0C3
:1053800038C0CEF0020ED06F020ECF6F040ED26F77
:10539000040ED16F090E2DECDCF0CCC037F0CDC07F
:1053A00038F0010E0101BB6F0101B005D8A403D094
:1053B0000201614B622B00019251D8A4FEEC11F066
:1053C00000019251D8A401EC10F008EC18F066EC42
:1053D00019F0E2ECFBF000019251D8A464EC05F066
:1053E000E5EC13F0F9EC0CF0E3EC05F06DECF7F004
:1053F000FBEC15F001016005D8A422D0040E0001D9
:10540000A419D8B41DD0030EA419D8B419D0A4057A
:10541000D8B416D0050EA419D8B412D09251D8B46D
:105420000FD0B551D8A40CD0AE51D8A409D0A4C087
:10543000A3F0050EA46F010EA16F010E0101C86F4C
:105440005050D8B4CAEC11F00101AE51D8B40FD00D
:1054500000019251D8A40BD0010E01017B6F6D0E9B
:105460000001A419D8B403D0000E0101AE6F0201EF
:1054700049514A11D8B403D04907D8A04A070101BD
:105480007B05D8A423D00001A405D8B41FD0020105
:1054900049514A11D8A41AD0000E4A6F400E496FE4
:1054A000AEC0EAF0B5C0EBF0AFC0ECF066C1EDF015
:1054B0009BC0EEF043C2EFF044C2F0F085C1F1F0C2
:1054C0000101645170ECF6F001017B6F0A0E0001DE
:1054D000A419D8A48ED39B05D8A40BD0000E9B6F23
:1054E0007CC043F27DC044F2010E01017B6F000ECF
:1054F0004B6F0001AF05D8B403D0B005D8A4E0D0FD
:1055000001015451D8A46DD000017A517C1904E1F5
:105510007B517D19D8B458D0000E0101236F000EC5
:10552000226F010E0001B46F4AD066EC19F0000141
:105530007A517C1910E17B517D19D8A40CD0000E52
:105540000101AB6F000E236F000E226F000E0001F1
:10555000B46F010EA16F0101235104E1C80E225D59
:10556000D8A02DD0000E0001D76F000ED66F100E00
:10557000D86F020ED96F060E22ECD1F07C5174194F
:1055800006E17D517519D8A402D0000E9C6F010E62
:105590000101AB6F000E236F000E226F000E0001A1
:1055A000B46F010EA16F410E0001F46FF00EF36FA6
:1055B000330EE82EFED7F32FFCD7F42FFAD70001D5
:1055C000B405D8A406D0B1D7000E0101AB6F000E10
:1055D000556F00017C517D11D8A403D0010E01014B
:1055E000546F01015351D8A46BD000019C05D8A47D
:1055F00067D07251741904E173517519D8B459D038
:10560000000E0101236F000E226F010E0001B46F26
:105610004CD066EC19F000017251741917E1735106
:105620007519D8A413D07A517C1910E17B517D19DA
:10563000D8A40CD0000E0101AB6F000E236F000E3A
:10564000226F000E0001B46F010EA16F0101235102
:1056500004E1C80E225DD8A028D0000E0001D76F4B
:10566000000ED66F100ED86F020ED96F060E22EC08
:10567000D1F0000E9C6F72C074F073C075F0000E14
:105680000101236F000E226F000E0001B46F010EA6
:10569000A16F410E0001F46FF00EF36F330EE82E90
:1056A000FED7F32FFCD7F42FFAD70001B405D8B4F6
:1056B000B0D774517511D8A403D0010E0101536FF6
:1056C0000101AB05D8B404D000018805D8A402D0EC
:1056D000010E09D00101AB51D8A407D000018851B7
:1056E000D8A403D0000E0101796F5A0E0001A81949
:1056F000D8B404D05A0E4AEC0FF0A86FB151B219C9
:10570000D8B404D0B15163ECF8F0B26F4650D8B4BD
:1057100035D0A751D8A430D0000ECA6F100EC96F73
:105720001CEC18F00009D8A427D0B8C0BCF03D503C
:1057300095EC0BF0916F8705D8A41AD0120E9165E5
:1057400002D0120E07D0030E916105D0010E3D6408
:1057500002D0020E916F050E91610AD0020E906187
:1057600007D0020E8F6F8FC090F0010E01015B6FAA
:10577000010E01015F6F02D0000E466E01015D5106
:105780000001B819D8B411D001015D5196EC19F09F
:10579000B86F010E01015C6F0001B851B71901012A
:1057A0005E6F000E4E6F010E4D6F0001A705D8A46D
:1057B00016D0010E0101CF6F2F5104E13D0E2E5D79
:1057C000D8A00DD00B0E0001A46F000E0101CF6F09
:1057D000000E2F6F000E2E6F010E0001A16F000151
:1057E000A605D8A423D001012F5120E13D0E2E5D46
:1057F000D8B01CD0000ECF6F000E2F6F000E2E6F92
:1058000045A006D0000E0001916F010E01015F6FEF
:1058100045A20CD03D50D8A409D00001B851010ACE
:1058200001015D6F000E4E6F010E4D6F000E000105
:10583000CA6F100EC96FBDEC15F00009D8B406D0C0
:10584000AB51D8A403D0010E0101CA6F000E0001B4
:10585000CA6F100EC96FDCEC15F00009D8B408D07F
:10586000000E0101CA6F000E02016E6F000E6D6F17
:105870000001AA05D8A415D002016E5104E1330E2F
:105880006D5DD8A00ED00C0E0001A46F000E0101BA
:10589000CA6F000E02016E6F000E6D6F010E0001E7
:1058A000A16F02016A5104E1960E695DD8A020D073
:1058B000010E0001A16F000E0101C76F000E020171
:1058C0006A6F000E696F00018905D8A403D0010E2C
:1058D00001014C6F00018705D8A403D0010E01011E
:1058E000456F00018805D8A403D0010E0101476F60
:1058F00098ECEBF001018351D8B402D0000E836F15
:10590000000E0001CA6F100EC96FBDEC15F0E8065D
:10591000D8B409D0000ECA6F100EC96FDCEC15F0B8
:10592000E806D8A41CD0AB51D8A40DD0AAC0CCF0A6
:1059300095C1CDF089C1CEF0000ECF6F0A0ED1EC2B
:10594000E2F0AA6F0CD04AC0CCF093C1CDF087C171
:10595000CEF0000ECF6F0C0ED1ECE2F04A6E000ECE
:10596000CA6F200EC96FBDEC15F0E806D8B409D097
:10597000000ECA6F200EC96FDCEC15F0E806D8A443
:105980003CD0AB51D8A40DD0A9C0CCF094C1CDF07F
:1059900088C1CEF0000ECF6F0B0ED1ECE2F0A96FF4
:1059A0002CD049C0CCF092C1CDF086C1CEF0000E13
:1059B000CF6F0D0ED1ECE2F0496E4904D8A416D099
:1059C000010E0101436F010E426F010E416F010E86
:1059D0000001A16F10EC00F005D066EC19F077EC37
:1059E000FDF04F6E4F50D8A408D0F7D7010E01013B
:1059F000426F000E436F000E416F0001B105D8A445
:105A000004D0A951A0EC17F007D0020EB119D8A408
:105A100005D0A951A0EC17F03B6E18D0030EB119B8
:105A2000D8A414D08A51A0EC17F03B6E8B05D8A4F3
:105A300002D0010E01D0000E0101496F0001885112
:105A400001014919D8B402D0010E486F00018751F5
:105A50003B18D8B411D03B04D8A405D090C05AF15B
:105A6000010E8F6F02D05AC18FF08FC090F0010EDF
:105A700001015B6F010E466F000E0101846F000192
:105A8000A205D8A412D0A2C0CCF0000ECD6F000E9B
:105A9000CE6F000ECF6F140ED1ECE2F0A26FA251C8
:105AA000D8A41AD0A3C0A4F00BD0000ECA6F800EE9
:105AB000C96FDCEC15F0E806D8A406D0640EA46F1C
:105AC000010EA16F010E06D0000ECA6F800EC96FC5
:105AD0001CEC18F00101846F020E0001CA6F000E69
:105AE000C96FDCEC15F0E806D8B409D0020ECA6F15
:105AF000000EC96FBDEC15F0E806D8A414D0ABC0F9
:105B0000CCF0010ECD6F010ECE6F000ECF6F0E0EDA
:105B1000D1ECE2F0AB6F030EB219D8A4ABC085F1A3
:105B2000010E01017B6F01013251D8A477ECFDF029
:105B3000000E0001CA6F400EC96FBDEC15F0E806FB
:105B4000D8A40BD0010E0101CE6F000E0001816FB1
:105B5000000E806F010E01014B6F000E0001CA6F35
:105B6000400EC96F1CEC18F0E806D8A416D081517D
:105B700004E1320E805DD8A010D0000E01014B6F01
:105B800000019251D8B409D010EC00F0A4C0A3F0E9
:105B9000040E0001A46F010EA16F000ECA6F400E2B
:105BA000C96FDCEC15F0E806D8A416D0815114E1D9
:105BB000320E805DD8B010D0000E0101CE6F000E05
:105BC0000001816F000E806F01014B05D8A404D045
:105BD000010E4E1B010E4D6F89C078F10001820548
:105BE000D8A4A3EFC3F0A4C0A3F0030EA46F79EF71
:105BF000C2F00B0EA419D8A434D09B51D8A409D05C
:105C0000010E9B6F7CC043F27DC044F2010E010186
:105C10007B6F1E0E0001A819D8B404D01E0E4AECEA
:105C20000FF0A86F4650D8B407D09051D4EC14F0C0
:105C30008F6F010E01015B6F0001A605D8A40CD087
:105C40000A0EA46F000E0101CF6F000E2F6F000E21
:105C50002E6F010E0001A16F8205D8B4C4D7A3EF47
:105C6000C3F00C0EA419D8A415D19B51D8A417D0F9
:105C7000010E9B6F7CC043F27DC044F2010E010116
:105C80007B6F000E0001CA6F100EC96F1CEC18F07C
:105C90000009D8A404D00A0EA46F010EA16FDC0E77
:105CA000A819D8B404D0DC0E4AEC0FF0A86F465007
:105CB000D8B40DD078C0BCF079C0BDF03EEC0DF08A
:105CC000BCC078F0BDC079F0010E0101596F000130
:105CD0007851335C79513458D8B007D033C078F05C
:105CE00034C079F0010E0101596F0001785179112A
:105CF000D8A407D0000E796F010E786F010E010154
:105D0000596F000E0001CC6F000ECD6F000ECE6FEC
:105D1000000ECF6F120ED1ECE2F0E806D8A407D047
:105D200076C078F077C079F0010E0101596F000E4E
:105D30000001CC6F000ECD6F000ECE6F000ECF6F46
:105D4000130ED1ECE2F0E806D8A407D035C078F005
:105D500036C079F0010E0101596F000E0001CA6FC3
:105D6000100EC96FDCEC15F00009D8B455D0000E48
:105D7000AA6F000E9A6F78517C1904E179517D1950
:105D8000D8B432D076C035F077C036F07CC076F02B
:105D90007DC077F0000E8D6F000E8C6F000E8B6F44
:105DA000000E8A6F000E0101526F000E516F000E3F
:105DB000506F000E4F6F00018905D8A405D0000E6A
:105DC00001014E6F010E4D6F000E0001916F010E2B
:105DD00001015F6F010E00018F6F010E01015B6F0A
:105DE000000E556F000E546F7AC043F27BC044F230
:105DF000000174517C1906E175517D19D8A402D0B7
:105E0000000E9C6F0A0EA46F010EA16F9251D8A4D0
:105E100003D0050E70ECF4F0000E0001CA6F100EF6
:105E2000C96FBDEC15F0E806D8B409D0000ECA6FF2
:105E3000100EC96FDCEC15F0E806D8A40CD0AAC08F
:105E4000CCF095C1CDF089C1CEF0000ECF6F0A0E17
:105E5000D1ECE2F0AA6F000ECA6F200EC96FBDEC44
:105E600015F0E806D8B409D0000ECA6F200EC96F2D
:105E7000DCEC15F0E806D8A4EFD6A9C0CCF094C1AC
:105E8000CDF088C1CEF0000ECF6F0B0ED1ECE2F05A
:105E9000A96FE2D6640EA419D8A488D09B51D8A4C7
:105EA00009D0010E9B6F7CC043F27DC044F2010E0D
:105EB00001017B6F1E0E0001A819D8B404D01E0E7C
:105EC0004AEC0FF0A86F4650D8B408D0A4C0BCF07C
:105ED0009751DFEC0BF0966F010E986FA505D8A4D3
:105EE00002D0010EA06FA605D8B40ED020D0650E4A
:105EF00009D06E0E07D0820E05D0780E03D06D0E3D
:105F000001D0640EA46F11D09751010AD8B4EFD715
:105F1000030AD8B4EED7010AD8B4EDD7070AD8B42B
:105F2000ECD7010AD8B4EBD7ECD7010EA16F000E65
:105F3000CA6F400EC96FBDEC15F0E806D8A408D0B2
:105F4000010E0101CE6F000E0001816F000E806F07
:105F5000000ECA6F400EC96F1CEC18F0E806D8A4FA
:105F600012D0815104E1510E805DD8A00CD00A0EF0
:105F7000A46F010EA16F000E0101CE6F000E000193
:105F8000816F000E806F000ECA6F400EC96FDCEC8F
:105F900015F0E806D8A460D6815107E1510E805D66
:105FA000D8B05AD60A0EB2EFC1F056D6650EA41973
:105FB000D8A4DBD19B51D8A409D0010E9B6F7CC023
:105FC00043F27DC044F2010E01017B6FDC0E000143
:105FD000A819D8B404D0DC0E4AEC0FF0A86F4650D4
:105FE000D8B40DD078C0BCF079C0BDF03EEC0DF057
:105FF000BCC078F0BDC079F0010E0101596F0001FD
:10600000A505D8A404D0010EA06F000E9A6FA605B6
:10601000D8A451D078517C1904E179517D19D8B4B4
:1060200032D076C035F077C036F07CC076F07DC0D7
:1060300077F0000E8D6F000E8C6F000E8B6F000ED0
:106040008A6F000E0101526F000E516F000E506FEB
:10605000000E4F6F00018905D8A405D0000E010184
:106060004E6F010E4D6F000E0001916F010E010188
:106070005F6F010E00018F6F010E01015B6F000E5B
:10608000556F000E546F7AC043F27BC044F200019A
:1060900074517C1906E175517D19D8A402D0000E07
:1060A0009C6F0A0EA46F010EA16F9251D8A403D069
:1060B000050E70ECF4F0000E0001CC6F000ECD6FF9
:1060C000000ECE6F000ECF6F120ED1ECE2F0E8069C
:1060D000D8A407D076C078F077C079F0010E01011E
:1060E000596F000E0001CC6F000ECD6F000ECE6F09
:1060F000000ECF6F130ED1ECE2F0E806D8A407D063
:1061000035C078F036C079F0010E0101596F000EEC
:106110000001CC6F000ECD6F000ECE6F000ECF6F62
:106120000F0ED1ECE2F0E806D8A47BD0030EB21932
:10613000D8A441D0210EF66EFE0EF76E000EF86E5A
:106140000800F550520AD8A413D078C0C9F079C01D
:10615000CAF05A0ECB6FD2EC03F0F36F090EF36165
:1061600005D00A0E7827000E792321D05A0E55D07B
:1061700078C0C9F079C0CAF05A0ECB6FD2EC03F0E8
:10618000F36F060EF36105D00A0E7827000E79230F
:1061900004D03C0E785F000E795B795104E13E0E2D
:1061A000785DD8A004D0000E796F3D0E786F010E97
:1061B0000101596F36D0020EB219D8A409D078C0A7
:1061C000C9F079C0CAF05A0ECB6FD2EC03F0C5D734
:1061D000B205D8A426D078C0C9F079C0CAF0540E50
:1061E000CB6FD2EC03F00009D8A409D078C0C9F075
:1061F00079C0CAF05A0ECB6FD2EC03F0AED778C09C
:10620000C9F079C0CAF05A0ECB6FD2EC03F0F36F2D
:10621000020EF36101D0A5D7140E785F000E795BF2
:10622000C6D7000E0001CC6F000ECD6F000ECE6FF2
:10623000000ECF6F100ED1ECE2F0E806D8A42CD0FF
:10624000020EB219D8B428D0B205D8A425D078C08F
:10625000C9F079C0CAF0540ECB6FD2EC03F000093C
:10626000D8A413D078C0C9F079C0CAF0480ECB6F5B
:10627000D2EC03F0F36F090EF36105D0640E7827BA
:10628000000E792306D0840E01D0E80E785F030E4D
:10629000795B010E0101596F00017851335C79512E
:1062A0003458D8B007D033C078F034C079F0010E3C
:1062B0000101596F000178517911D8A407D0000E5F
:1062C000796F010E786F010E0101596F000E000108
:1062D000CA6F400EC96FBDEC15F0E806D8A40ED009
:1062E000000E9A6F010E0101CE6F000E0001816F4A
:1062F000000E806F7CC078F07DC079F0000ECA6F10
:10630000400EC96F1CEC18F0E806D8A412D08151D9
:1063100004E1510E805DD8A00CD00A0EA46F010ECE
:10632000A16F000E0101CE6F000E0001816F000E03
:10633000806F000ECA6F400EC96FDCEC15F0E806E6
:10634000D8A48AD4815110E1510E805DD8B084D494
:10635000640EA46F000E0101CE6F000E0001816F6C
:10636000000E806F010E77D477D46E0EA419D8A4D6
:1063700088D09B51D8A409D0010E9B6F7CC043F2FA
:106380007DC044F2010E01017B6F1E0E0001A819B1
:10639000D8B404D01E0E4AEC0FF0A86F4650D8B403
:1063A00008D0A4C0BCF09751DFEC0BF0966F010E43
:1063B000986FA505D8A402D0010EA06FA605D8B489
:1063C00012D023D06F0EA46F030EFCECFFF01AD096
:1063D0006F0EA46F010EFCECFFF014D0700E01D014
:1063E000640EA46F0FD09751010AD8B4EBD7030AFB
:1063F000D8B4EED7010AD8B4F1D7070AD8B4F0D789
:10640000010AEED7010E0001A16F000ECA6F400E07
:10641000C96FBDEC15F0E806D8A408D0010E010143
:10642000CE6F000E0001816F000E806F000ECA6FEC
:10643000400EC96F1CEC18F0E806D8A412D08151A8
:1064400004E1510E805DD8A00CD00A0EA46F010E9D
:10645000A16F000E0101CE6F000E0001816F000ED2
:10646000806F000ECA6F400EC96FDCEC15F0E806B5
:10647000D8A42CEFAEF0815102E1ACEFC1F02CEFCB
:10648000AEF06F0EA419D8A4FAD29B51D8A409D0AB
:10649000010E9B6F7CC043F27DC044F2010E0101EE
:1064A0007B6F080E3D6405D0080E0001916F080E49
:1064B0003D6E010E00018F6F010E906F9E51D8A4AA
:1064C0000BD09D51D8A408D01E0EA819D8B404D062
:1064D0001E0E4AEC0FF015D09E05D8A408D0A00ED1
:1064E000A819D8B404D0A00E4AEC0FF00AD09D052C
:1064F000D8A408D0DC0EA819D8B404D0DC0E4AEC1D
:106500000FF0A86F4650D8B435D09E51D8A414D0FF
:106510009D51D8A411D0A4C0BCF09751DFEC0BF072
:10652000966F9F05D8A405D0020E966502D0020E84
:10653000966F010E986F1ED09E05D8A40BD06C519B
:10654000AFEC14F0F36FF3516C6F6D6B010E010142
:106550003E6F10D09D05D8A40DD068C0BCF069C0B6
:10656000BDF03DEC10F0BCC068F0BDC069F0010E9C
:1065700001013D6F0001A505D8A404D0000E9A6F5B
:10658000010EA06FA605D8A46ED09E51D8A461D0EC
:106590009D51D8B43DD05DD0010E9E6F000E446E6B
:1065A000000E9D6F0BD09F05D8B40BD0010E9D6FD0
:1065B000000E01017A6F000E00019E6F010E9A6FAE
:1065C00052D04404D8A44FD0010E0101A16F000E97
:1065D000000114D04404D8A446D001017A05D8A4FF
:1065E00042D000019F05D8B40AD06E51C5EC0FF01F
:1065F0000101A16F00016E51B1EC08F0AD6F000E0A
:106600000101AA6F6F0E0001A46F010EA16F2BD0C4
:106610009751010AD8B4C0D7030AD8B4C4D7010A25
:10662000D8B4D8D720D0000E9E6F010E446E6CC037
:106630006EF06DC06FF014D09F05D8B411D0000E6D
:106640009D6F010E01017A6F68C06AF069C06BF03E
:1066500007D09751010AD8B4E6D7030AD8B4ECD7CB
:10666000010E0001986F0101A105D8B404D000010A
:10667000AD05D8A407D00101AA51D8A403D0010EBA
:106680000001B46F0001B405D8B456D059D066ECFF
:1066900019F000016E5102013B191DE100016F511B
:1066A00002013C19D8A417D000016A51020139191E
:1066B00012E100016B5102013A19D8A40CD0000E6E
:1066C0000101AA6F000E236F000E226F000E000161
:1066D000B46F010EA16F0101235104E1C80E225DC8
:1066E000D8A02AD0000E0001D76F000ED66F100E72
:1066F000D86F020ED96F0B0E22ECD1F0010E010102
:10670000AA6F000EA16F000E0001AD6F000E010117
:10671000236F000E226F000E0001B46F010EA16FF7
:10672000410E0001F46FF00EF36F330EE82EFED72A
:10673000F32FFCD7F42FFAD70001B405D8B4A7D7AC
:10674000A2C0CCF0000ECD6F000ECE6F000ECF6F4A
:10675000140ED1ECE2F0A26FA205D8A406D0A4C01A
:10676000A3F00A0EA46F010EA16F000ECC6F000EF5
:10677000CD6F000ECE6F000ECF6F0F0ED1ECE2F09A
:10678000E806D8A4C6D0030EB219D8A424D09D051B
:10679000D8A405D0000E696F010E686F53D09E51CA
:1067A000D8B4B7D06CC0C9F06DC0CAF05A0ECB6F68
:1067B000D2EC03F0F36F070EF36105D00A0E6C27DD
:1067C000000E6D2304D0460E6C5F000E6D5B010E53
:1067D00001013E6F9ED0020EB219D8A449D09D058A
:1067E000D8A434D068C0C9F069C0CAF0480ECB6FD5
:1067F000D2EC03F0F36F020EF36113D068C0C9F05E
:1068000069C0CAF05A0ECB6FD2EC03F0F36F090ED9
:10681000F36105D00A0E6827000E692313D05A0EC3
:106820000ED068C0C9F069C0CAF05A0ECB6FD2EC66
:1068300003F0F36F030EF36101D0ECD71E0E685F17
:10684000000E695B010E01013D6F63D09E51D8B40B
:1068500060D06CC0C9F06DC0CAF05A0ECB6FD2ECDC
:1068600003F0F36F090EF36101D0A8D75A0EACD72D
:10687000B205D8A44ED09D05D8A424D068C0C9F0D4
:1068800069C0CAF0480ECB6FD2EC03F0F36F020E72
:10689000F36109D068C0C9F069C0CAF05A0ECB6F65
:1068A000D2EC03F0B3D768C0C9F069C0CAF05A0E81
:1068B000CB6FD2EC03F0F36F050EF36101D0AAD7D2
:1068C000320EBDD79E51D8B424D06CC0C9F06DC073
:1068D000CAF0480ECB6FD2EC03F0F36F020EF361F7
:1068E00009D06CC0C9F06DC0CAF05A0ECB6FD2ECA3
:1068F00003F0B7D76CC0C9F06DC0CAF05A0ECB6FA9
:10690000D2EC03F0F36F050EF36101D057D7320ECE
:106910005BD7000E0001CC6F000ECD6F000ECE6F66
:10692000000ECF6F100ED1ECE2F0E806D8A44BD0E9
:10693000B205D8A438D09D05D8A419D068C0C9F034
:1069400069C0CAF0480ECB6FD2EC03F0F36F020EB1
:10695000F36105D0640E6827000E692304D0C80EC9
:10696000685F000E695B010E01013D6F2CD09E51E6
:10697000D8B429D06CC0C9F06DC0CAF0480ECB6F36
:10698000D2EC03F0F36F020EF36105D0640E6C27B6
:10699000000E6D2304D0C80E6C5F000E6D5B010EFF
:1069A00001013E6F10D0020EB219D8A40CD09D0583
:1069B000D8A409D068C0C9F069C0CAF0480ECB6F2E
:1069C000D2EC03F0C3D73C500001F36FF46B6C5171
:1069D000F35D6D51F459D8B003D03CC06CF06D6BD1
:1069E00068510101085D0001695101010959D8B0E0
:1069F00004D008C168F009C169F0000E0001CA6F37
:106A0000400EC96FBDEC15F0E806D8A40ED0000EFC
:106A10009A6F010E0101CE6F000E0001816F000E12
:106A2000806F000E9D6F000E9E6F000ECA6F400EAD
:106A3000C96F1CEC18F0E806D8A412D0815104E10B
:106A4000510E805DD8A00CD00A0EA46F010EA16F6C
:106A5000000E0101CE6F000E0001816F000E806FED
:106A6000000ECA6F400EC96FDCEC15F0E806D8A422
:106A70002CEFAEF0815101E11BD22CEFAEF0700E85
:106A8000A419D8A41FD29B51D8A409D0010E9B6F82
:106A90007CC043F27DC044F2010E01017B6F000E09
:106AA0000001916F000E3D6EDC0EA819D8B404D021
:106AB000DC0E4AEC0FF0A86F4650D8B40DD066C07B
:106AC000BCF067C0BDF03EEC0DF0BCC066F0BDC0D0
:106AD00067F0010E01013C6F0001A505D8A404D0A8
:106AE000000E9A6F010EA06FA605D8A432D0665191
:106AF0007C1904E167517D19D8B428D0000E8D6F40
:106B0000000E8C6F000E8B6F000E8A6F000E01015D
:106B1000526F000E516F000E506F000E4F6F00014C
:106B20008905D8A405D0000E01014E6F010E4D6FEE
:106B3000010E00018F6F010E906F66C000F167C0FB
:106B400001F1010E0101A26F000EAA6F000E0001FB
:106B50009C6F0101A205D8A406D0AA51D8A403D0E5
:106B6000010E0001B46F0001B405D8B458D05BD059
:106B700066EC19F001010051021922E101510319DB
:106B8000D8A41ED0000EAA6F02C178F003C179F01C
:106B900002C17AF003C17BF07AC0BCF07BC0BDF0CB
:106BA000CCEC07F0000E0101A26F000E236F000E67
:106BB000226F000E0001B46F0A0EA46F010EA16FC8
:106BC0000101235104E1C80E225DD8A028D0000E97
:106BD0000001D76F000ED66F100ED86F020ED96F5E
:106BE0000B0E22ECD1F0010E0101AA6F000EA26F74
:106BF000000E236F000E226F000E0001B46F0A0E0C
:106C0000A46F010EA16F410E0001F46FF00EF36F3F
:106C1000330EE82EFED7F32FFCD7F42FFAD700015E
:106C2000B405D8B4A5D7000ECC6F000ECD6F000E02
:106C3000CE6F000ECF6F120ED1ECE2F0E806D8A4B2
:106C400007D076C066F077C067F0010E01013C6F97
:106C5000000E0001CC6F000ECD6F000ECE6F000E47
:106C6000CF6F130ED1ECE2F0E806D8A407D035C000
:106C700066F036C067F0010E01013C6F000E0001A6
:106C8000CC6F000ECD6F000ECE6F000ECF6F0F0ECB
:106C9000D1ECE2F0E806D8A47BD0030EB219D8A458
:106CA00041D0210EF66EFE0EF76E000EF86E080053
:106CB000F550520AD8A413D066C0C9F067C0CAF014
:106CC0005A0ECB6FD2EC03F0F36F090EF36105D0CF
:106CD0000A0E6627000E672321D05A0E55D066C0D3
:106CE000C9F067C0CAF05A0ECB6FD2EC03F0F36F55
:106CF000060EF36105D00A0E6627000E672304D046
:106D00003C0E665F000E675B675104E13E0E665DF8
:106D1000D8A004D0000E676F3D0E666F010E010112
:106D20003C6F36D0020EB219D8A409D066C0C9F0A3
:106D300067C0CAF05A0ECB6FD2EC03F0C5D7B205CC
:106D4000D8A426D066C0C9F067C0CAF0540ECB6F75
:106D5000D2EC03F00009D8A409D066C0C9F067C01E
:106D6000CAF05A0ECB6FD2EC03F0AED766C0C9F0B2
:106D700067C0CAF05A0ECB6FD2EC03F0F36F020E6D
:106D8000F36101D0A5D7140E665F000E675BC6D70E
:106D9000000E0001CC6F000ECD6F000ECE6F000E06
:106DA000CF6F100ED1ECE2F0E806D8A42CD0020E82
:106DB000B219D8B428D0B205D8A425D066C0C9F07D
:106DC00067C0CAF0540ECB6FD2EC03F00009D8A410
:106DD00013D066C0C9F067C0CAF0480ECB6FD2ECC2
:106DE00003F0F36F090EF36105D0640E6627000E01
:106DF000672306D0840E01D0E80E665F030E675B42
:106E0000010E01013C6F00016651335C675134583B
:106E1000D8B007D033C066F034C067F0010E01016E
:106E20003C6F000166516711D8A407D0000E676F50
:106E3000010E666F010E01013C6F000E0001CA6F6A
:106E4000400EC96FBDEC15F0E806D8A40AD0000EBC
:106E50009A6F010E0101CE6F000E0001816F000ECE
:106E6000806F000ECA6F400EC96F1CEC18F0E80668
:106E7000D8A412D0815104E1510E805DD8A00CD06D
:106E80000A0EA46F010EA16F000E0101CE6F000E5D
:106E90000001816F000E806F000ECA6F400EC96F37
:106EA000DCEC15F0E806D8A42CEFAEF0815108E137
:106EB000510E805DD8B02CEFAEF06E0EB2EFC1F087
:106EC0002CEFAEF0780EA419D8A483D09B51D8A48F
:106ED00009D0010E9B6F7CC043F27DC044F2010ECD
:106EE00001017B6F1E0E0001A819D8B404D01E0E3C
:106EF0004AEC0FF0A86F4650D8B408D0A4C0BCF03C
:106F00009751DFEC0BF0966F010E986FA505D8A492
:106F100002D0010EA06FA605D8B40CD01ED0790EF9
:106F200007D07A0E05D0780E03D07C0E01D0810EEA
:106F3000A46F11D09751010AD8B4F1D7030AD8B47D
:106F4000F0D7010AD8B4EFD7070AD8B4EED7010AB0
:106F5000D8B4EDD7E8D7010EA16F000ECA6F400E6E
:106F6000C96FBDEC15F0E806D8A408D0010E0101E8
:106F7000CE6F000E0001816F000E806F000ECA6F91
:106F8000400EC96F1CEC18F0E806D8A412D081514D
:106F900004E1510E805DD8A00CD00A0EA46F010E42
:106FA000A16F000E0101CE6F000E0001816F000E77
:106FB000806F000ECA6F400EC96FDCEC15F0E8065A
:106FC000D8A42CEFAEF0815102E1ACEFC1F02CEF70
:106FD000AEF0790EA419D8A479D09B51D8A409D0C9
:106FE000010E9B6F7CC043F27DC044F2010E010193
:106FF0007B6F1E0E0001A819D8B404D01E0E4AECF7
:107000000FF0A86F4650D8B408D001016F5137EC8B
:1070100014F001016F6F010E6E6F0001A605D8A478
:1070200004D0780EA46F010EA16FA2C0CCF0000EA8
:10703000CD6F000ECE6F000ECF6F140ED1ECE2F0CC
:10704000A26FA205D8A406D0A4C0A3F00A0EA46F14
:10705000010EA16F000ECA6F400EC96FBDEC15F096
:10706000E806D8A408D0010E0101CE6F000E000181
:10707000816F000E806F000ECA6F400EC96F1CEC4E
:1070800018F0E806D8A412D0815104E1510E805DB9
:10709000D8A00CD00A0EA46F010EA16F000E010142
:1070A000CE6F000E0001816F000E806F000ECA6F60
:1070B000400EC96FDCEC15F0E806D8A42CEFAEF05A
:1070C000815102E1C3EFBCF02CEFAEF07A0EA419AF
:1070D000D8A4D8D09B51D8A409D0010E9B6F7CC0F6
:1070E00043F27DC044F2010E01017B6F1E0E0001D0
:1070F000A819D8B404D01E0E4AEC0FF0A86F465061
:10710000D8B408D0A4C0BCF09751DFEC0BF0966F58
:10711000010E986FA505D8A402D0010EA06FA60598
:10712000D8B408D012D0010E03D0020E01D0030E45
:10713000B16F0BD09751010AD8B4F5D7030AD8B470
:10714000F4D7010AD8B4F3D7EED7B151B219D8B4F5
:1071500048D0000E916F010E01015F6F010E00011A
:107160008F6F010E01015B6F0001B15163ECF8F00C
:10717000B26F000E8D6F000E8C6F000E8B6F000EC5
:107180008A6F000E0101526F000E516F000E506F9A
:10719000000E4F6F000E0001AA6F000EA96F000EC7
:1071A0004A6E000E496E000E0101856F00018905CF
:1071B000D8A405D0000E01014E6F010E4D6F0001E5
:1071C0008805D8A405D0000E0101496F010E486F53
:1071D00000018705D8A405D0000E3B6E010E010109
:1071E000466FA2C0CCF0000E0001CD6F000ECE6F36
:1071F000000ECF6F140ED1ECE2F0A26FA205D8A45E
:1072000006D0A4C0A3F00A0EA46F010EA16F000E59
:10721000CA6F400EC96FBDEC15F0E806D8A408D0BF
:10722000010E0101CE6F000E0001816F000E806F14
:10723000000ECA6F400EC96F1CEC18F0E806D8A407
:1072400012D0815104E1510E805DD8A00CD00A0EFD
:10725000A46F010EA16F000E0101CE6F000E0001A0
:10726000816F000E806F000ECA6F400EC96FDCEC9C
:1072700015F0E806D8A42CEFAEF0815101E183D3DC
:107280002CEFAEF07B0EA419D8A448D09B51D8A403
:1072900009D0010E9B6F7CC043F27DC044F2010E09
:1072A00001017B6F000E0001CA6F400EC96FBDEC7B
:1072B00015F0E806D8A408D0010E0101CE6F000E2B
:1072C0000001816F000E806F000ECA6F400EC96F03
:1072D0001CEC18F0E806D8A412D0815104E1510E3C
:1072E000805DD8A00CD00A0EA46F010EA16F000E15
:1072F0000101CE6F000E0001816F000E806F000E45
:10730000CA6F400EC96FDCEC15F0E806D8A42CEF6C
:10731000AEF0815101E137D32CEFAEF07C0EA41911
:10732000D8A491D29B51D8A409D0010E9B6F7CC0E8
:1073300043F27DC044F2010E01017B6F1E0E00017D
:10734000A819D8B404D01E0E4AEC0FF0A86F46500E
:10735000D8B408D0A4C0BCF09751DFEC0BF0966F06
:10736000010E986FA505D8A402D0010EA06FA60546
:10737000D8B426D22CD2780EA46F010EA16F27D2DA
:10738000000E4E6E010E4D6E000E5A6E000E5B6EBC
:1073900013D266EC19F00001B451D8A48CD0070EBA
:1073A000D66FF6C0D7F0020E88EC14F0000ED76F3F
:1073B000000ED66F100ED86F030ED96F0A0E22EC96
:1073C000D1F0270EC26FFD0EC36F070EC46F010E02
:1073D000C56F010EC66F1E0EC76F060EC86F000E7A
:1073E000C96F000ECA6F000ECB6F000ECC6F000E7F
:1073F000CD6FF6C0CEF0BAEC00F0270EC26FFD0ED6
:10740000C36F070EC46F010EC56F010EC66F250E48
:10741000C76F060EC86F000EC96F000ECA6F000E50
:10742000CB6F000ECC6F000ECD6FF6C0CEF0BAEC75
:1074300000F0270EC26FFD0EC36F070EC46F010E62
:10744000C56F010EC66F2C0EC76F060EC86F000EFB
:10745000C96F000ECA6F000ECB6F000ECC6F000E0E
:10746000CD6FF6C0CEF0BAEC00F0270EC26FFD0E65
:10747000C36F070EC46F010EC56F010EC66F330ECA
:10748000C76F060EC86F000EC96F000ECA6F000EE0
:10749000CB6F000ECC6F000ECD6FF6C0CEF0BAEC05
:1074A00000F0000EF56F010E0101C36F000EAF6F0B
:1074B000010E0001B46F1D0E0101C265F8D0000E6F
:1074C000C26F0001F52BF505D8A439D0270EC26F85
:1074D000FD0EC36F070EC46F010EC56F010EC66FA0
:1074E000330EC76F060EC86F000EC96F000ECA6F4D
:1074F000000ECB6F000ECC6F000ECD6FF6C0CEF03D
:10750000BAEC00F0270EC26FFD0EC36F070EC46FFA
:10751000010EC56F020EC66F1E0EC76F060EC86F36
:10752000000EC96F000ECA6F000ECB6F000ECC6F3D
:10753000000ECD6FF6C0CEF0BAEC00F0B8D0020E5F
:10754000F519D8A439D0270EC26FFD0EC36F070EF0
:10755000C46F010EC56F010EC66F1E0EC76F060EFB
:10756000C86F000EC96F000ECA6F000ECB6F000E01
:10757000CC6F000ECD6FF6C0CEF0BAEC00F0270E47
:10758000C26FFD0EC36F070EC46F010EC56F020EF2
:10759000C66F250EC76F060EC86F000EC96F000EAE
:1075A000CA6F000ECB6F000ECC6F000ECD6FF6C011
:1075B000CEF0BAEC00F07BD0030EF519D8A439D088
:1075C000270EC26FFD0EC36F070EC46F010EC56F8D
:1075D000010EC66F250EC76F060EC86F000EC96F6D
:1075E000000ECA6F000ECB6F000ECC6F000ECD6F79
:1075F000F6C0CEF0BAEC00F0270EC26FFD0EC36FDE
:10760000070EC46F010EC56F020EC66F2C0EC76F3A
:10761000060EC86F000EC96F000ECA6F000ECB6F4A
:10762000000ECC6F000ECD6FF6C0CEF0BAEC00F0BD
:107630003ED0040EF519D8A43AD0270EC26FFD0E25
:10764000C36F070EC46F010EC56F010EC66F2C0EFF
:10765000C76F060EC86F000EC96F000ECA6F000E0E
:10766000CB6F000ECC6F000ECD6FF6C0CEF0BAEC33
:1076700000F0270EC26FFD0EC36F070EC46F010E20
:10768000C56F020EC66F330EC76F060EC86F000EB1
:10769000C96F000ECA6F000ECB6F000ECC6F000ECC
:1076A000CD6FF6C0CEF0BAEC00F0000EF56F4E04D0
:1076B000D8A448D0000E0101C36F000EC26F000EA7
:1076C000236F000E226F000E0001B46F000E4D6E8E
:1076D000000E0101AF6F000E556F070E0001D66F4F
:1076E000F6C0D7F0040E88EC14F0000ED76F000E31
:1076F000D66F100ED86F020ED96F0C0E22ECD1F09F
:107700007A0E0001F46FC10EF36F810EE82EFED7E2
:10771000F32FFCD7F42FFAD700D00A0E0001A46F84
:10772000010EA16F9251D8B407D0030E70ECF4F0A3
:10773000040E70ECF4F006D0010E70ECF4F0020EC2
:1077400070ECF4F0DC0E0101225D050E2359D8A087
:1077500033D0000EC36F000EC26F000E236F000EF9
:10776000226F000E0001B46F000E4D6E010E01017C
:10777000AF6F070E0001D66FF6C0D7F0040E88EC8D
:1077800014F0000ED76F000ED66F100ED86F020ED9
:10779000D96F0B0E22ECD1F07A0E0001F46FC10EFE
:1077A000F36F810EE82EFED7F32FFCD7F42FFAD714
:1077B00000D0010E0001A16F4D04D8A408D0E9D576
:1077C0009751010AD8B4D7D5030AD8B4D9D5000E39
:1077D0000001CA6F400EC96FBDEC15F0E806D8A4D1
:1077E00008D0010E0101CE6F000E0001816F000E66
:1077F000806F000ECA6F400EC96F1CEC18F0E806CF
:10780000D8A412D0815104E1510E805DD8A00CD0D3
:107810000A0EA46F010EA16F000E0101CE6F000EC3
:107820000001816F000E806F000ECA6F400EC96F9D
:10783000DCEC15F0E806D8A42CEFAEF0815101E1A4
:10784000A2D02CEFAEF0810EA419D8A4A6D09B51E3
:10785000D8A409D0010E9B6F7CC043F27DC044F2D6
:10786000010E01017B6F0001A505D8A403D0010E14
:107870000101A66F0001A605D8A44CD00101A60500
:10788000D8A448D077ECEEF00009D8B4FBD7070EA7
:107890000001C46F0D0EFCEC16F0070E0001C46F62
:1078A0000F0EFCEC16F0070E0001C46F0E0EFCEC80
:1078B00016F0070E0001C46F100EFCEC16F08DECF4
:1078C000DEF0410E0001F46FF00EF36F330EE82E80
:1078D000FED7F32FFCD7F42FFAD7020E0001C46FA6
:1078E0000D0EFCEC16F0020E0001C46F0F0EFCEC46
:1078F00016F0030E0001C46F0E0EFCEC16F0030E22
:107900000001C46F100EFCEC16F00A0E0001A46F0B
:10791000010EA16F000E0001CA6F400EC96FBDECD1
:1079200015F0E806D8A408D0010E0101CE6F000EB4
:107930000001816F000E806F000ECA6F400EC96F8C
:107940001CEC18F0E806D8A412D0815104E1510EC5
:10795000805DD8A00CD00A0EA46F010EA16F000E9E
:107960000101CE6F000E0001816F000E806F000ECE
:10797000CA6F400EC96FDCEC15F0E806D8A42CEFF6
:10798000AEF0815108E1510E805DD8B02CEFAEF021
:10799000780EB2EFC1F02CEFAEF0820EA419D8A48D
:1079A0007DD09B51D8A409D0010E9B6F7CC043F2BF
:1079B0007DC044F2010E01017B6F1E0E0001A8196B
:1079C000D8B404D01E0E4AEC0FF0A86F4650D8B4BD
:1079D00008D0A4C0BCF09751DFEC0BF0966F010EFD
:1079E000986FA505D8A402D0010EA06FA605D8B443
:1079F0000FD018D0830E0AD0840EA46F000E916FA2
:107A0000000E3D6E000E9C6F0BD0820EA46F08D04E
:107A10009751010AD8B4EED7030AD8B4EDD7F5D7F9
:107A2000010EA16F000ECA6F400EC96FBDEC15F0BC
:107A3000E806D8A408D0010E0101CE6F000E0001A7
:107A4000816F000E806F000ECA6F400EC96F1CEC74
:107A500018F0E806D8A412D0815104E1510E805DDF
:107A6000D8A00CD00A0EA46F010EA16F000E010168
:107A7000CE6F000E0001816F000E806F000ECA6F86
:107A8000400EC96FDCEC15F0E806D8A42CEFAEF080
:107A9000815102E1ACEFC1F02CEFAEF0830EA419DE
:107AA000D8A419D29B51D8A409D0010E9B6F7CC0D9
:107AB00043F27DC044F2010E01017B6F00018E058F
:107AC000D8A408D0DC0EA819D8B404D0DC0E4AEC37
:107AD0000FF00AD08E51D8A408D01E0EA819D8B421
:107AE00004D01E0E4AEC0FF0A86F4650D8B419D03F
:107AF0008E05D8A40ED070C0BCF071C0BDF03EECB5
:107B00000DF0BCC070F0BDC071F0010E0101576FE7
:107B100008D0A4C0BCF09751DFEC0BF0966F010EBB
:107B2000986F0001A505D8A404D0000E9A6F010E2D
:107B3000A06FA605D8A485D08E51D8B46ED078D0C9
:107B4000010E8E6F000E9C6F010E9A6F010E936FE7
:107B500078D0B751010A0101566F56C1B7F0000144
:107B6000B851B71901015E6F010E0001936F010E4C
:107B7000A06F000E9A6F65D09305D8A43ED07C51BB
:107B8000701904E17D517119D8B402D0010E01D0F1
:107B9000000E9C6F7051741904E171517519D8B4BD
:107BA0002ED09C05D8A42BD0000E8D6F000E8C6FAC
:107BB000000E8B6F000E8A6F000E0101526F000ED7
:107BC000516F000E506F000E4F6F00018905D8A451
:107BD00005D0000E01014E6F010E4D6F000E000129
:107BE000916F010E01015F6F010E00018F6F010E99
:107BF00001015B6F000E536F02D0000E9C6F000EF0
:107C000000019A6F0A0EA46F010EA16F9251D8A4C1
:107C100018D0060E70ECF4F014D09751010AD8B4C5
:107C20008FD7030AD8B495D7010AD8B4A5D709D0FD
:107C30009705D8A404D0000E8E6F000E9A6F010E27
:107C4000986FA2C0CCF0000E0001CD6F000ECE6F79
:107C5000000ECF6F140ED1ECE2F0A26FA205D8A4F3
:107C600006D0A4C0A3F00A0EA46F010EA16F8E056A
:107C7000D8A4D3D0000ECC6F000ECD6F000ECE6F07
:107C8000000ECF6F120ED1ECE2F0E806D8A407D0B8
:107C900076C070F077C071F0010E0101576F000ED1
:107CA0000001CC6F000ECD6F000ECE6F000ECF6FB7
:107CB000130ED1ECE2F0E806D8A407D035C070F07E
:107CC00036C071F0010E0101576F000E0001CC6F3C
:107CD000000ECD6F000ECE6F000ECF6F0F0ED1ECE9
:107CE000E2F0E806D8A45ED0030EB219D8B404D0EE
:107CF000020EB219D8A423D070C0C9F071C0CAF066
:107D00005A0ECB6FD2EC03F0F36F060EF36105D081
:107D10000A0E7027000E712304D03C0E705F000E17
:107D2000715B715104E13E0E705DD8A004D0000E6D
:107D3000716F3D0E706F010E0101576F33D0B205A8
:107D4000D8A430D070C0C9F071C0CAF0540ECB6F47
:107D5000D2EC03F00009D8A413D070C0C9F071C0F0
:107D6000CAF05A0ECB6FD2EC03F0F36F090EF36139
:107D700005D00A0E7027000E7123DDD75A0E0ED0E3
:107D800070C0C9F071C0CAF05A0ECB6FD2EC03F0CC
:107D9000F36F020EF36101D0ECD7140E705F000E8A
:107DA000715BC9D7000E0001CC6F000ECD6F000EC5
:107DB000CE6F000ECF6F100ED1ECE2F0E806D8A423
:107DC0002CD0020EB219D8B428D0B205D8A425D030
:107DD00070C0C9F071C0CAF0540ECB6FD2EC03F082
:107DE0000009D8A413D070C0C9F071C0CAF0480E01
:107DF000CB6FD2EC03F0F36F090EF36105D0640E84
:107E00007027000E712306D0840E01D0E80E705F3B
:107E1000030E715B010E0101576F000170510101EA
:107E20000A5D0001715101010B59D8B006D00AC199
:107E300070F00BC171F0010E576F0001705171119C
:107E4000D8A407D0000E716F010E706F010E0101F2
:107E5000576F000E0001CA6F400EC96FBDEC15F0E0
:107E6000E806D8A40ED0000E9A6F010E0101CE6F65
:107E7000000E0001816F000E806F000E9C6F000EDF
:107E80008E6F000ECA6F400EC96F1CEC18F0E8062A
:107E9000D8A412D0815104E1510E805DD8A00CD03D
:107EA0000A0EA46F010EA16F000E0101CE6F000E2D
:107EB0000001816F000E806F000ECA6F400EC96F07
:107EC000DCEC15F0E806D8A42CEFAEF0815101E10E
:107ED000F1D12CEFAEF0840EA419D8A4F4D19B51AB
:107EE000D8A409D0010E9B6F7CC043F27DC044F240
:107EF000010E01017B6F00018505D8B403D0840514
:107F0000D8A408D0C80EA819D8B404D0C80E4AEC1A
:107F10000FF007D01E0EA819D8B404D01E0E4AECDC
:107F20000FF0A86F4650D8B430D08551D8A40CD0EB
:107F30008451D8A409D0A4C0BCF09751DFEC0BF059
:107F4000966F010E986F21D08505D8A40ED031C050
:107F5000BCF032C0BDF03EEC0DF0BCC031F0BDC095
:107F600032F0010E0101406F10D08405D8A40DD06D
:107F70002FC0BCF030C0BDF03EEC0DF0BCC02FF007
:107F8000BDC030F0010E01013F6F0001A505D8A46E
:107F900004D0000E9A6F010EA06FA605D8A4A5D03C
:107FA0008551D8A49AD08451D8B458D096D0010E17
:107FB000856F000E846F04D0010E846F000E856FF4
:107FC000010E9A6F92D08651D8A425D0B051D8A472
:107FD00003D0AF51D8B43ED0010E0101B96F000EED
:107FE00000018F6F000E906F000E916F000E3D6EBE
:107FF000000E01015D6F000E0001B86F06C178F040
:1080000007C179F006C17AF007C17BF0010E3A6E24
:10801000010E866F1FD03A04D8B41CD0000E866FB4
:10802000000E0101B96F000E1F6F000E1E6F010ED2
:1080300000018F6F010E906F000E916F000E3D6E6C
:10804000000E01015D6F000E0001B86F0A0EA46FF3
:10805000010EA16F010E0001986F47D09751010AE0
:10806000D8B4A5D7030AD8B4A7D7010AD8B4ABD7D8
:108070003CD0000E856F31C006F132C007F101011E
:108080000451065D05510759D8A0E4D7010E3124EB
:108090002F6E000E3220306E2FC004F130C005F17B
:1080A000010E3F6FD7D7000E846F2FC004F130C090
:1080B00005F101010451065D05510759D8A0CAD741
:1080C000FF0E2F24316EFF0E3020326E31C006F1CC
:1080D00032C007F1010E406FBDD79751010AD8B4E5
:1080E000C8D7030AD8B4DFD7B5D7B051D8A403D0C6
:1080F000AF51D8B492D08605D8A47DD03A04D8A484
:1081000012D001011F5104E10A0E1E5DD8A00BD050
:10811000000E1F6F000E1E6F020E3A6E0C0E000155
:10812000916F0C0E2FD0020E3A18D8A416D0010170
:108130001F5104E1640E1E5DD8A00FD0000E1F6F0A
:10814000000E1E6F030E3A6E010E5D6F010E0001F0
:10815000B86F080E916F080E15D0030E3A18D8A408
:1081600013D001011F5104E18C0E1E5DD8A00CD06C
:10817000000E1F6F000E1E6F040E3A6E000E0001FF
:10818000916F000E3D6E37D0040E3A18D8A433D04C
:1081900001011F5104E1280E1E5DD8A02CD0000E55
:1081A0001F6F000E1E6F000E5D6F000E0001B86F96
:1081B0000101045100017A5D0101055100017B5963
:1081C000D8B009D0010E3A6E784B792B78C07AF08E
:1081D00079C07BF010D0000E866F000E0101B96FE0
:1081E000000E1F6F000E1E6F010E00018F6F010E3B
:1081F000906F010E986F00017C510201431906E156
:1082000000017D5102014419D8B407D07CC043F26B
:108210007DC044F2010E01017B6F000E0001CA6FA8
:10822000400EC96FBDEC15F0E806D8A41CD0000EB6
:10823000866F000E0101B96F000E1F6F000E1E6FDA
:10824000000E0001916F000E3D6E000E846F000E57
:10825000856F000E9A6F010E0101CE6F000E0001B6
:10826000816F000E806F000ECA6F400EC96F1CEC4C
:1082700018F0E806D8A412D0815104E1510E805DB7
:10828000D8A00CD00A0EA46F010EA16F000E010140
:10829000CE6F000E0001816F000E806F000ECA6F5E
:1082A000400EC96FDCEC15F0E806D8A42CEFAEF058
:1082B000815107E1510E805DD8B02CEFAEF0820EF7
:1082C00051D02CEFAEF06D0EA419D8A458D09B510C
:1082D000D8A409D0010E9B6F7CC043F27DC044F24C
:1082E000010E01017B6F000E0001CA6F400EC96FC5
:1082F000BDEC15F0E806D8A408D0010E0101CE6F40
:10830000000E0001816F000E806F000ECA6F400EDC
:10831000C96F1CEC18F0E806D8A412D0815104E112
:10832000510E805DD8A00CD00A0EA46F010EA16F73
:10833000000E0101CE6F000E0001816F000E806FF4
:10834000000ECA6F400EC96FDCEC15F0E806D8A429
:108350002CEFAEF0815111E1510E805DD8B02CEFC1
:10836000AEF0640EA46F010EA16F000E0101CE6F7E
:10837000000E0001816F000E806F2CEFAEF0A4059F
:10838000D8A488D00D0E946F000ECA6F800EC96FEE
:108390001CEC18F0506E0201685104E18C0E675D10
:1083A000D8A027D05050D8A424D0000E0101C16F0E
:1083B000000E0201686F000E676F0A0E0001A46FC5
:1083C000010EA16F000EBD6F070EBC6F09EC19F016
:1083D0005A0AD8A408D0000E0001BD6F080EBC6F69
:1083E00009EC19F001D00C0E0001946F010E01018F
:1083F000B06F00018205D8A406D0A4C0A3F0030E7C
:10840000A46F010EA16F000ECA6F400EC96FBDECC4
:1084100015F0E806D8A408D0010E0101CE6F000EB9
:108420000001816F000E806F000ECA6F400EC96F91
:108430001CEC18F0E806D8A410D0815104E1320EEB
:10844000805DD8A00AD0040EA46F0A0EA36F010E9F
:10845000A16F000E816F630E806F000ECA6F400E19
:10846000C96FDCEC15F0E806D8A46DD1815103E1A9
:10847000320E805DD8B067D1000E0101CE6F000EC4
:108480000001816F000E806F000E0201686F8C0E7C
:10849000676F59D1030EA419D8A42ED001012C5115
:1084A00040080001C26F01012D51D8A0E82A01083F
:1084B0000001C36F000EC56F640EC46F0EEC14F0A4
:1084C000C251426E010176514218D8B402D0010E59
:1084D000756F00018251D8A436D18305D8A433D159
:1084E000A451A319D8A403D00A0EA46F02D0A3C02C
:1084F000A4F0010EA16F27D1040EA419D8A447D06F
:1085000080514008C26F8151D8A0E82A0108C36F8A
:10851000000EC56F640EC46F0EEC14F0C251956F5F
:108520000101745100019519D8B409D0410E805D44
:10853000010E8159D8B003D0010E0101736F000EF6
:108540000001CA6F400EC96F1CEC18F0E806D8A4F1
:108550000FD0400E805D010E8159D8B004D008D0F4
:1085600077ECFDF04F6E4F50D8B4FAD79FEC19F06E
:10857000000E0001CA6F400EC96FDCEC15F0E80672
:10858000D8A4E1D0A451A319D8B4AED7B0D7050E62
:10859000A419D8A499D00B0ECB6FB80ECA6F78EC83
:1085A00010F001016051D8B403D06105D8A40CD0FB
:1085B0000001A451A319D8A403D00A0EA46F02D0BD
:1085C000A3C0A4F0010EA16F000E0001CA6F100E2F
:1085D000C96FBDEC15F0E806D8B409D0000ECA6F1B
:1085E000100EC96FDCEC15F0E806D8A40CD0AAC0B8
:1085F000CCF095C1CDF089C1CEF0000ECF6F0A0E40
:10860000D1ECE2F0AA6F000ECA6F200EC96FBDEC6C
:1086100015F0E806D8B409D0000ECA6F200EC96F55
:10862000DCEC15F0E806D8A40CD0A9C0CCF094C1BD
:10863000CDF088C1CEF0000ECF6F0B0ED1ECE2F082
:10864000A96F8205D8A406D0A4C0A3F0030EA46F1E
:10865000010EA16F000ECA6F400EC96FBDEC15F080
:10866000E806D8A408D0010E0101CE6F000E00016B
:10867000816F000E806F000ECA6F400EC96F1CEC38
:1086800018F0E806D8A410D0815104E1320E805DC4
:10869000D8A00AD0A4C0A3F0040EA46F010EA16F4D
:1086A000000E816F630E806F000ECA6F400EC96F9F
:1086B000DCEC15F0E806D8A446D0815144E1320E36
:1086C000805DD8A0D9D63FD0060EA419D8A43BD03F
:1086D000E00E0101205D2E0E2159D8A032D02F0EC0
:1086E000205D310E2159D8B013D020512E08000141
:1086F000C26F01012151D8A0E82A31080001C36FDF
:10870000000EC56F640EC46F0EEC14F0C251406EC3
:1087100001016D514018D8B402D0010E6C6F6D513B
:10872000D8A411D04050D8A40ED010EC00F003D043
:1087300077ECFDF04F6E4F50D8B4FAD79FEC19F09C
:1087400002D000011FD70001A451ACECC3F0A4512A
:1087500000EC80F0D4EFA9F0DC6F3950D8A431D010
:108760006E0E0001DC19D8B420D06F0EDC19D8B41D
:108770001CD0700EDC19D8B418D0780EDC19D8B41F
:1087800014D0790EDC19D8B410D07A0EDC19D8B414
:108790000CD07B0EDC19D8B408D07C0EDC19D8B410
:1087A00004D0810EDC19D8A406D048C0CCF0020E4B
:1087B0001BECEAF00BD048C0CCF0010E1BECEAF049
:1087C00005D048C0CCF0030E1BECEAF00A0E000105
:1087D000A419D8A4B7D2AB51D8A47CD1B105D8A4E0
:1087E0007BD08DC0CCF018C1CDF019C1CEF0020EF7
:1087F000D06F020ECF6F040ED26F040ED16F010E38
:108800002DECDCF0CCC018F1CDC019F18CC0CCF04F
:1088100016C1CDF017C1CEF0020ED06F020ECF6F91
:10882000040ED26F040ED16F020E2DECDCF0CCC022
:1088300016F1CDC017F18BC0CCF014C1CDF015C12D
:10884000CEF0020ED06F020ECF6F040ED26F040E68
:10885000D16F030E2DECDCF0CCC014F1CDC015F1BE
:108860008AC0CCF012C1CDF013C1CEF0020ED06F91
:10887000020ECF6F040ED26F040ED16F040E2DECDA
:10888000DCF0CCC012F1CDC013F1AAC0CCF010C105
:10889000CDF011C1CEF0020ED06F020ECF6F040EDC
:1088A000D26F040ED16F050E2DECDCF0CCC010F1B0
:1088B000CDC011F1A9C0CCF00EC1CDF00FC1CEF0EA
:1088C000020ED06F020ECF6F040ED26F040ED16F66
:1088D000060E2DECDCF0D1D1020EB119D8A47BD05C
:1088E0008DC0CCF018C1CDF019C1CEF0020ED06F02
:1088F000020ECF6F040ED26F040ED16F010E2DEC5D
:10890000DCF0CCC018F1CDC019F18CC0CCF016C190
:10891000CDF017C1CEF0020ED06F020ECF6F040E55
:10892000D26F040ED16F020E2DECDCF0CCC016F12C
:10893000CDC017F18BC0CCF014C1CDF015C1CEF075
:10894000020ED06F020ECF6F040ED26F040ED16FE5
:10895000030E2DECDCF0CCC014F1CDC015F18AC0B3
:10896000CCF012C1CDF013C1CEF0020ED06F020ECA
:10897000CF6F040ED26F040ED16F040E2DECDCF01D
:10898000CCC012F1CDC013F1AAC0CCF010C1CDF013
:1089900011C1CEF0020ED06F020ECF6F040ED26F57
:1089A000040ED16F050E2DECDCF0CCC010F1CDC063
:1089B00011F1A9C0CCF00EC1CDF00FC1CEF0020E66
:1089C000D06F020ECF6F100ED26F100ED16F060E49
:1089D0002DECDCF052D1030EB119D8A452D18DC0C8
:1089E000CCF018C1CDF019C1CEF0020ED06F020E3E
:1089F000CF6F040ED26F040ED16F010E2DECDCF0A0
:108A0000CCC018F1CDC019F18CC0CCF016C1CDF09E
:108A100017C1CEF0020ED06F020ECF6F040ED26FD0
:108A2000040ED16F020E2DECDCF0CCC016F1CDC0DF
:108A300017F18BC0CCF014C1CDF015C1CEF0020EF1
:108A4000D06F020ECF6F040ED26F040ED16F030EE3
:108A50002DECDCF0CCC014F1CDC015F18AC0CCF007
:108A600012C1CDF013C1CEF0020ED06F020ECF6F47
:108A7000100ED26F100ED16F040E2DECDCF0CCC0B6
:108A800012F1CDC013F1AAC0CCF010C1CDF011C1CC
:108A9000CEF0020ED06F020ECF6F040ED26F040E16
:108AA000D16F050E2DECDCF0CCC010F1CDC011F172
:108AB000A9C0CCF00EC1CDF00FC1CEF0020ED06F28
:108AC000020ECF6F040ED26F040ED16F060E2DEC86
:108AD000DCF0D3D0B105D8A47BD052C1CCF018C102
:108AE000CDF019C1CEF0020ED06F020ECF6F040E82
:108AF000D26F040ED16F010E2DECDCF0CCC018F15A
:108B0000CDC019F151C1CCF016C1CDF017C1CEF0D6
:108B1000020ED06F020ECF6F040ED26F040ED16F13
:108B2000020E2DECDCF0CCC016F1CDC017F150C117
:108B3000CCF014C1CDF015C1CEF0020ED06F020EF4
:108B4000CF6F040ED26F040ED16F030E2DECDCF04C
:108B5000CCC014F1CDC015F14FC1CCF012C1CDF095
:108B600013C1CEF0020ED06F020ECF6F040ED26F83
:108B7000040ED16F040E2DECDCF0CCC012F1CDC090
:108B800013F14AC0CCF010C1CDF011C1CEF0020EED
:108B9000D06F020ECF6F040ED26F040ED16F050E90
:108BA0002DECDCF0CCC010F1CDC011F149C0CCF0FF
:108BB0000EC1CDF00FC1CEF0020ED06F020ECF6FFE
:108BC000100ED26F100ED16F060E2DECDCF055D0CA
:108BD000020EB119D8A427D04AC0CCF010C1CDF0F4
:108BE00011C1CEF0020ED06F020ECF6F040ED26F05
:108BF000040ED16F050E2DECDCF0CCC010F1CDC011
:108C000011F149C0CCF00EC1CDF00FC1CEF0020E73
:108C1000D06F020ECF6F040ED26F040ED16F060E0E
:108C20002DECDCF02AD0030EB119D8A42AD04AC00A
:108C3000CCF010C1CDF011C1CEF0020ED06F020EFB
:108C4000CF6F040ED26F040ED16F050E2DECDCF049
:108C5000CCC010F1CDC011F149C0CCF00EC1CDF0A7
:108C60000FC1CEF0020ED06F020ECF6F040ED26F86
:108C7000040ED16F060E2DECDCF0CCC00EF1CDC091
:108C80000FF1ABC0CCF04BC2CDF04CC2CEF0020E17
:108C9000D06F020ECF6F040ED26F040ED16F0A0E8A
:108CA0002DECDCF0CCC04BF2CDC04CF284C1CCF04A
:108CB0004DC2CDF04EC2CEF0020ED06F020ECF6F7D
:108CC000040ED26F040ED16F080E2DECDCF0CCC078
:108CD0004DF2CDC04EF201014C51D8A41CD0000E73
:108CE0000001CA6F400EC96F1CEC18F0CC6F7EC03B
:108CF000CDF07FC0CEF0020ED06F020ECF6F040E0B
:108D0000D26F040ED16F070E2DECDCF0CCC07EF0DC
:108D1000CDC07FF012004CC1CCF07EC0CDF07FC042
:108D2000CEF0020E0001D06F020ECF6F200ED26F78
:108D3000200ED16F070E2DECDCF0CCC07EF0CDC044
:108D40007FF01200040EDC19D8A41BD0000ECA6FED
:108D5000400EC96F1CEC18F0CC6F7EC0CDF07FC008
:108D6000CEF0020ED06F020ECF6F100ED26F100E2B
:108D7000D16F070E2DECDCF0CCC07EF0CDC07FF0C3
:108D800012006D0EA419D8A41BD0000ECA6F400E9D
:108D9000C96F1CEC18F0CC6F7EC0CDF07FC0CEF058
:108DA000020ED06F020ECF6F040ED26F040ED16F81
:108DB000070E2DECDCF0CCC07EF0CDC07FF01200B1
:108DC000780EA419D8A41BD0000ECA6F400EC96F2C
:108DD0001CEC18F0CC6F7EC0CDF07FC0CEF0020E40
:108DE000D06F020ECF6F040ED26F040ED16F070E3C
:108DF0002DECDCF0CCC07EF0CDC07FF01200700E08
:108E0000A419D8A41BD0000ECA6F400EC96F1CEC69
:108E100018F0CC6F7EC0CDF07FC0CEF0020ED06FC8
:108E2000020ECF6F040ED26F040ED16F070E2DEC21
:108E3000DCF0CCC07EF0CDC07FF012006F0EA41924
:108E4000D8A41BD0000ECA6F400EC96F1CEC18F0DE
:108E5000CC6F7EC0CDF07FC0CEF0020ED06F020E80
:108E6000CF6F040ED26F040ED16F070E2DECDCF025
:108E7000CCC07EF0CDC07FF012006E0EA419D8A435
:108E80001BD0000ECA6F400EC96F1CEC18F0CC6FDF
:108E90007EC0CDF07FC0CEF0020ED06F020ECF6F3D
:108EA000040ED26F040ED16F070E2DECDCF0CCC097
:108EB0007EF0CDC07FF01200830EA419D8A41BD081
:108EC000000ECA6F400EC96F1CEC18F0CC6F7EC04C
:108ED000CDF07FC0CEF0020ED06F020ECF6F040E29
:108EE000D26F040ED16F070E2DECDCF0CCC07EF0FB
:108EF000CDC07FF01200650EA419D8A41BD0000EBF
:108F0000CA6F400EC96F1CEC18F0CC6F7EC0CDF05C
:108F10007FC0CEF0020ED06F020ECF6F040ED26F64
:108F2000040ED16F070E2DECDCF0CCC07EF0CDC06E
:108F30007FF01200640EA419D8A41BD0000ECA6FD3
:108F4000400EC96F1CEC18F0CC6F7EC0CDF07FC016
:108F5000CEF0020ED06F020ECF6F040ED26F040E51
:108F6000D16F070E2DECDCF0CCC07EF0CDC07FF0D1
:108F700012000B0EA419D8A41BD0000ECA6F400E0D
:108F8000C96F1CEC18F0CC6F7EC0CDF07FC0CEF066
:108F9000020ED06F020ECF6F040ED26F040ED16F8F
:108FA000070E2DECDCF0CCC07EF0CDC07FF01200BF
:108FB000820EA419D8A41BD0000ECA6F400EC96F30
:108FC0001CEC18F0CC6F7EC0CDF07FC0CEF0020E4E
:108FD000D06F020ECF6F040ED26F040ED16F070E4A
:108FE0002DECDCF0CCC07EF0CDC07FF01200840E02
:108FF000A419D8A41200000ECA6F400EC96F1CEC51
:1090000018F0CC6F7EC0CDF07FC0CEF0020ED06FD6
:10901000020ECF6F040ED26F040ED16F070E2DEC2F
:10902000DCF0CCC07EF0CDC07FF0120000017851A2
:10903000D61906E17951D719D8A402D0000E08D06C
:109040007051D61906E17151D719D8A402D0010E7A
:10905000DD6F040ED75DD8A004D0030ED76FD6699C
:1090600008D0D651D711D8A404D0000ED76F010E66
:10907000D66FD6C0C2F0D7C0C3F0030EC56FE80EDE
:10908000C46F0EEC14F0C251100FD86F030EBF6FF7
:10909000E80EBE6FD6C0BCF0D7C0BDF05DEC15F0D9
:1090A000BCC0C2F0BDC0C3F0000EC56F640EC46F7B
:1090B0000EEC14F0C251100FD96F000EBF6F640E8A
:1090C000BE6FD6C0BCF0D7C0BDF05DEC15F0BCC023
:1090D000C2F0BDC0C3F0000EC56F0A0EC46F0EEC27
:1090E00014F0C251100FDA6FD6C0BCF0D7C0BDF07B
:1090F000000EBF6F0A0EBE6F5DEC15F0BC51100F75
:10910000DB6F4304D8B404D001017951D8A429D22B
:1091100000019C05D8A425D2E80ED65D030ED759D0
:10912000D8A07DD0480EC26FE50EC36F070EC46F86
:10913000020EC56FD8C0C6F0000EC76FDD51020D1C
:10914000F350030FC86F000EC96F000ECA6F000EF8
:10915000CB6F000ECC6F000ECD6FF6C0CEF0BAEC28
:1091600000F0480EC26FE50EC36F070EC46F020E0B
:10917000C56FD9C0C6F0090EC76FDD51020DF3509F
:10918000030FC86F000EC96F000ECA6F000ECB6FC1
:10919000000ECC6F000ECD6FF6C0CEF0BAEC00F032
:1091A000480EC26FE50EC36F070EC46F020EC56F87
:1091B000DAC0C6F0120EC76FDD51020DF350030F77
:1091C000C86F000EC96F000ECA6F000ECB6F000E85
:1091D000CC6F000ECD6FF6C0CEF0BAEC00F0480EAA
:1091E000C26FE50EC36F070EC46F020EC56FDBC002
:1091F000C6F01A0EC76FDD51020DF350030FC86F92
:10920000000EC96F000ECA6F000ECB6F000ECC6F40
:10921000000ECD6FF6C0CEF0BAEC00F01200D751C0
:1092200004E1640ED65DD8A09CD0480EC26FE50E56
:10923000C36F070EC46F020EC56F000EC66F000E1F
:10924000C76FDD51020DF350030FC86F000EC96FD9
:10925000000ECA6F000ECB6F000ECC6F000ECD6FEC
:10926000F6C0CEF0BAEC00F0480EC26FE50EC36F48
:10927000070EC46F020EC56FD9C0C6F0000EC76FCF
:10928000DD51020DF350030FC86F000EC96F000EC1
:10929000CA6F000ECB6F000ECC6F000ECD6FF6C004
:1092A000CEF0BAEC00F0480EC26FE50EC36F070EA9
:1092B000C46F020EC56FDAC0C6F0090EC76FDD516C
:1092C000020DF350030FC86F000EC96F000ECA6F76
:1092D000000ECB6F000ECC6F000ECD6FF6C0CEF03F
:1092E000BAEC00F0480EC26FE50EC36F070EC46FF4
:1092F000020EC56FDBC0C6F0120EC76FDD51020D46
:10930000F350030FC86F000EC96F000ECA6F000E36
:10931000CB6F000ECC6F000ECD6FF6C0CEF0BAEC66
:1093200000F0480EC26FE50EC36F070EC46F020E49
:10933000C56F000EC66F1A0EC76FDD51020DF350D8
:10934000030FC86F000EC96F000ECA6F000ECB6FFF
:10935000000ECC6F000ECD6FF6C0CEF0BAEC00F070
:109360001200D75104E10A0ED65DD8A07DD0480E78
:10937000C26FE50EC36F070EC46F020EC56F000EFD
:10938000C66F000EC76FDD51020DF350030FC86F9B
:10939000000EC96F000ECA6F000ECB6F000ECC6FAF
:1093A000000ECD6FF6C0CEF0BAEC00F0480EC26FE2
:1093B000E50EC36F070EC46F020EC56FDAC0C6F0AC
:1093C000090EC76FDD51020DF350030FC86F000E79
:1093D000C96F000ECA6F000ECB6F000ECC6F000E6F
:1093E000CD6FF6C0CEF0BAEC00F0480EC26FE50EBD
:1093F000C36F070EC46F020EC56FDBC0C6F0120E3E
:10940000C76FDD51020DF350030FC86F000EC96F17
:10941000000ECA6F000ECB6F000ECC6F000ECD6F2A
:10942000F6C0CEF0BAEC00F0480EC26FE50EC36F86
:10943000070EC46F020EC56F000EC66F1A0EC76FFF
:10944000DD51020DF350030FC86F000EC96F000EFF
:10945000CA6F000ECB6F000ECC6F000ECD6FF6C042
:10946000CEF0BAEC00F01200480EC26FE50EC36FEA
:10947000070EC46F020EC56F000EC66F000EC76FD9
:10948000DD51020DF350030FC86F000EC96F000EBF
:10949000CA6F000ECB6F000ECC6F000ECD6FF6C002
:1094A000CEF0BAEC00F0480EC26FE50EC36F070EA7
:1094B000C46F020EC56F000EC66F090EC76FDD5177
:1094C000020DF350030FC86F000EC96F000ECA6F74
:1094D000000ECB6F000ECC6F000ECD6FF6C0CEF03D
:1094E000BAEC00F0480EC26FE50EC36F070EC46FF2
:1094F000020EC56FDBC0C6F0120EC76FDD51020D44
:10950000F350030FC86F000EC96F000ECA6F000E34
:10951000CB6F000ECC6F000ECD6FF6C0CEF0BAEC64
:1095200000F0480EC26FE50EC36F070EC46F020E47
:10953000C56F000EC66F1A0EC76FDD51020DF350D6
:10954000030FC86F000EC96F000ECA6F000ECB6FFD
:10955000000ECC6F000ECD6FF6C0CEF0BAEC00F06E
:109560001200480E0001C26FE50EC36F070EC46FF4
:10957000020EC56F000EC66F000EC76FDD51020DE3
:10958000F350030FC86F000EC96F000ECA6F000EB4
:10959000CB6F000ECC6F000ECD6FF6C0CEF0BAECE4
:1095A00000F0480EC26FE50EC36F070EC46F020EC7
:1095B000C56F000EC66F090EC76FDD51020DF35067
:1095C000030FC86F000EC96F000ECA6F000ECB6F7D
:1095D000000ECC6F000ECD6FF6C0CEF0BAEC00F0EE
:1095E000480EC26FE50EC36F070EC46F020EC56F43
:1095F000000EC66F120EC76FDD51020DF350030F40
:10960000C86F000EC96F000ECA6F000ECB6F000E40
:10961000CC6F000ECD6FF6C0CEF0BAEC00F0480E65
:10962000C26FE50EC36F070EC46F020EC56F000E4A
:10963000C66F1A0EC76FDD51020DF350030FC86FCE
:10964000000EC96F000ECA6F000ECB6F000ECC6FFC
:10965000000ECD6FF6C0CEF0BAEC00F01200D8418B
:10966000E8423F0B030D6F00CCFFDFF0DA05D8A412
:1096700058D0510EC26FFC0EC36FDF516608C46F25
:10968000010EC56F000EC66FDFC0C7F0D9C0C8F0AD
:10969000000EC96F000ECA6F010ECB6F000ECC6FAB
:1096A000000ECD6FF6C0CEF0BAEC00F0510EC26FD6
:1096B000FC0EC36FDF516608C46F010EC56F000E4C
